:020000040000fa
:080000000002040000000000f2
:020000040000fa
:100008007808000078080000b0040000ba04000076
:1000180078080000780800007808000078080000d8
:100028007808000078080000780800003890000080
:1000380078080000780800007808000094020000a2
:1000480078080000780800007808000078080000a8
:100058007808000078080000780800007808000098
:100068007808000078080000780800007808000088
:100078007808000078080000780800007808000078
:100088007808000078080000780800007808000068
:10009800780800007808000048030000780800008d
:1000a8007808000078080000780800007808000048
:1000b8007808000078080000780800007808000038
:1000c8007808000078080000780800007808000028
:1000d8007808000078080000780800007808000018
:1000e8007808000078080000780800007808000008
:1000f80078080000780800007808000078080000f8
:1001080078080000780800007808000078080000e7
:1001180078080000780800007808000078080000d7
:1001280078080000780800007808000078080000c7
:1001380078080000780800007808000078080000b7
:1001480078080000780800007808000078080000a7
:100158007808000078080000780800007808000097
:100168007808000078080000780800007808000087
:100178007808000078080000780800007808000077
:100188007808000078080000780800007808000067
:100198007808000078080000780800007808000057
:1001a8007808000078080000780800007808000047
:1001b8007808000078080000780800007808000037
:1001c8007808000078080000780800007808000027
:1001d8007808000078080000780800007808000017
:1001e8007808000078080000780800007808000007
:0801f8007808000078080000ff
:020000040000fa
:100208007808000078080000b0040000ba04000074
:1002180078080000780800007808000078080000d6
:10022800780800007808000078080000389000007e
:1002380078080000780800007808000094020000a0
:1002480078080000780800007808000078080000a6
:100258007808000078080000780800007808000096
:100268007808000078080000780800007808000086
:100278007808000078080000780800007808000076
:100288007808000078080000780800007808000066
:10029800780800007808000048030000780800008b
:1002a8007808000078080000780800007808000046
:1002b8007808000078080000780800007808000036
:1002c8007808000078080000780800007808000026
:1002d8007808000078080000780800007808000016
:1002e8007808000078080000780800007808000006
:1002f80078080000780800007808000078080000f6
:1003080078080000780800007808000078080000e5
:1003180078080000780800007808000078080000d5
:1003280078080000780800007808000078080000c5
:1003380078080000780800007808000078080000b5
:1003480078080000780800007808000078080000a5
:100358007808000078080000780800007808000095
:100368007808000078080000780800007808000085
:100378007808000078080000780800007808000075
:100388007808000078080000780800007808000065
:100398007808000078080000780800007808000055
:1003a8007808000078080000780800007808000045
:1003b8007808000078080000780800007808000035
:1003c8007808000078080000780800007808000025
:1003d8007808000078080000780800007808000015
:1003e8007808000078080000780800007808000005
:0803f8007808000078080000fd
:020000040000fa
:10040000cff020000e7f22000e01880000000000c7
:1004100000012000200288000c00070060d728009f
:100420000100200011000700000020000000e00093
:10043000020032000000020000000000c4040200bc
:10044000000000000040da000000fe004440a90067
:10045000402b20000000e0000300320000002000dc
:10046000a00188004440a800000006009101880017
:10047000800078000000eb0015003700e2804000ab
:1004800032a0b4009101ba00e280400032a0b40072
:100490009102ba00e280400032a0b4000002eb00fa
:1004a000472bde00f507b200602ce10004003a00a3
:1004b0000059eb008301e900fdff3e000400370016
:1004c0006128e100010032000082eb000400070017
:1004d0001101ba000200e000e8ff3a000000060047
:1004e0003159ba008301e9000c0032002159ba00e9
:1004f0008301e900080032000400e00003003a0034
:10050000e280400032a0b400f5ff370011d9ba00f4
:100510008301e900faff3a008100e800e180400031
:1005200032a0b40000000600841f78000000fa002a
:1005300084e0a90014002000547088000080fa00b4
:100540004f027800004006000000fa008408800096
:100550000440a0000450a10084088800046b23001c
:10056000640888000002eb003408880084e0a900d9
:1005700094e0a80011e1a8000080fa000000060045
:100580000000fa00940880000440a0000450a1007c
:100590009408880004c42900740888000002eb0055
:1005a0005408880013e1a8000080fa00000006004b
:1005b000cc00fa000002eb00040f780064708000a9
:1005c000e00f520003003200e10f5200140032002d
:1005d0002d00370040462900c890020000000000ae
:1005e000b65102000000000000027800e10f520046
:1005f0000400320060492900c89002000000000099
:10060000210037000040eb00ee7c020000000000fb
:10061000647080000402e800647088001a003700eb
:10062000b65102000000000000027800e10f520005
:1006300014003a0001003700000000008e0b020099
:100640000000000000027800040f7800f46a230024
:100650009e027800848f5200f7ff3600980b02004c
:100660000000000000027800140798000040eb0032
:10067000165202000000000094e0a90084e0a900e6
:10068000eeff3700000000000080fa0000000600c6
:10069000801f7800849fbe00861f78000200fa0049
:1006a000b4118000044f780087c0a900c4df200087
:1006b000144278000483fb0005a02000850243005b
:1006c0009e4a78000442e80004407800fcedb70040
:1006d000a4df2000144278000442e80004407800bf
:1006e000faedb7000080fa004f0378004f02be0019
:1006f0004f007800004006000200fa0097c0a900f1
:10070000a4df2000144278000482fb00040f78006c
:1007100097c0a8001e027800040078000080fa004c
:10072000000006000400fa00100798001e02900066
:10073000040f78008411800066026200e60f520008
:100740001e003a000c0037000000000095118000e8
:100750000420200004826200e00f5200fbff3a00f8
:100760001e02900014027800a41188001e0290005e
:100770000482e800140798001e029000140278001a
:10078000e00f5200f0ff3a001100370000000000b7
:10079000951180000420200004826200e00f5200c6
:1007a000fbff3a001e027800144278000402fb00ae
:1007b000a41188001e0fe8000100370000000000af
:1007c0001e02780014427800e04f5200efff3a001a
:1007d0000080fa00000006000a00fa0020079800d6
:1007e00031079800420798000002eb00040f7800e0
:1007f0003e02900014079800240037004e0290003b
:100800009e027800848f5200020031001e0fe80023
:10081000030037002e029000200037000000000087
:100820002100070000427800e04f5200f3ff320041
:100830000002eb00040f7800841180006602620061
:10084000e60f520007003a00b51180003e0290000a
:10085000050a78003e0290000482e8003407980000
:1008600007003700b4118000044278009e02900017
:10087000844a78001e0290000402e80014079800e1
:100880002e0290000402e900240798002e02900036
:10089000e00f5200e1ff3a002e02900004007800c1
:1008a0000080fa00000006000000fa0094118000a9
:1008b0000442780061426200044078000080fa003f
:1008c000000006000000fa009511800004102000ce
:1008d0000482620004f0a7000402ea000402e900b6
:1008e0004f22de0004427800044078000080fa00c5
:1008f000000006000000fa00841180006602620019
:10090000e60f520002003a00b411800003003700e5
:10091000b5118000f40f200004826200040078000a
:100920000080fa00000006000200fa00000f7800c4
:100930008411800066026200e60f520003003a0054
:100940001e027800a411880003003700f40f200075
:100950001e026200a41188000080fa000000060058
:100960000000fa0000000000000000000080fa0013
:10097000004006000000fa00000000000000000037
:100980000080fa00004006000400fa00a2010700ff
:1009900092010700a6010700e4000700088c02008e
:1009a0000000000024d7200052022000a14b2900a3
:1009b00004007800a20b020000000000968c0200e8
:1009c00000000000a402020000000000c0020200bb
:1009d0000000000001010700a516800004002200ad
:1009e00004826200e00f52003d003a00988f02003e
:1009f000000000000002be00048fbe00452c200055
:100a00000042eb00844a780030003700988f0200e3
:100a1000000000000002be003e035200ae835a00f8
:100a200004092d0035002000840f5300858f5b00e2
:100a3000260036006000b8005c8302000000000061
:100a400000c0eb00748302000000000000c0eb0057
:100a50007483020000000000e88302000000000030
:100a6000452c2000f4c0b300844a78000000000048
:100a7000988f0200000000000002be003e035200fa
:100a8000ae835a000602be000403be0024aa24005e
:100a900045002000840f5300858f5b00f4ff340075
:100aa000452c20000042eb00844a78000000000042
:100ab000a51680000400220004826200e00f5200ac
:100ac000fbff32000000fe0005003700a516800085
:100ad0000400220004826200e00f5200cbff3200cb
:100ae00072850200000000000100370000000000d5
:100af000988f0200000000000003be00e468800040
:100b0000f56880000403530085835b0014a127006f
:100b100005002000840f5300858f5b001100360014
:100b2000988f0200000000000002be00e468880008
:100b3000f568880024168000044278006142620053
:100b40000404a200614262000482fb0061026200b0
:100b500026168000e5ff2f008502630004827200e4
:100b600024168800ba8502000000000022880200d6
:100b700000000000d80202000000000050900200b7
:100b80000000000061000700f46680000567800037
:100b90000669800017698000860f5200878f5a000f
:100ba000d2ff3200f4668000056780000469880087
:100bb00015698800f4668000056780000400be00a7
:100bc000030007002c88020000000000c8ff370067
:100bd0000c00fa00881f7800400798005107980021
:100be00004c1b300244798000042eb00044f780092
:100bf000330037009e4278000582fb00e802470080
:100c000004824200144278000482fb00e3024700a1
:100c10008500780004007800906f0200000000005a
:100c20000042eb00144798000f0037002e4290005e
:100c30000483fb001e4290000482fb000402470074
:100c40003442900025d7200085024300844a780072
:100c50002e4290000442e800244798001e42900073
:100c60000442e800144798001e4290000484fb00f0
:100c70006302470004007800e00b0200000000005f
:100c800000027800840f5400e8ff39001e4278000b
:100c9000e34f52000e0032002e4290008482fb008f
:100ca00024d7200084824200e4c2b300844a780042
:100cb0002e4290000442e800244798001e4fe800ae
:100cc0001e427800e34f5200caff36000100370091
:100cd000000000002e429000ff4f520006003e0030
:100ce0002e4290008482fb0024d7200084824200a0
:100cf0000042eb00844a7800968c0200000000005d
:100d00004f0478000080fa00000006000000fa009e
:100d10000418800041d1200004007800906f020088
:100d2000000000000080fa00000006000000fa0049
:100d3000c002a900c022a900c042a900c062a90047
:100d4000c082a900c0a2a900c0c2a900c4e2a90033
:100d5000452c20000042eb00844a7800243a8000b1
:100d60000480a1000490a10004a0a100243a8800fe
:100d70000002eb00441988002c83a9002ca3a900d1
:100d8000444e2800041988004440200014198800ab
:100d900034002100241988000402200084198800ee
:100da00097c0a80004002800841188000440200097
:100db0009411880034032000c4118800d7c2a80011
:100dc000d3c2a900d782a800d382a900fa81020069
:100dd000000000000080fa00000006000800fa0091
:100de000881f78000042eb00044f78003203200097
:100df0008000eb00e0cd2000b00b020000000000fe
:100e00000acda8000aeda80062002000f14d2900db
:100e1000b0d02000a20b020000000000048c2a00c9
:100e200055f02000f466880005678800f4668000ad
:100e30000567800094678800a5678800f4ff2f008d
:100e4000f50f20001467880025678800146780006c
:100e500025678000b4678800c567880094ea2f0082
:100e600015102000346788004567880094ea2f0039
:100e70001510200054678800656788006022b8005c
:100e8000746788008567880002012000514e2900a0
:100e9000a0cf2000a20b020000000000a0cf200085
:100ea0008e7202000000000031032000e0cd20001f
:100eb000ce710200000000000002780094688800f3
:100ec0001e427800e04f520002003200e0cd2000c8
:100ed000260007000e82e80063002000040178006d
:100ee0006000b80080820200000000003303200090
:100ef000e2cd20006000200001002000808202007e
:100f0000000000009e02900034032000848f5200f5
:100f10000c003a00ae02900094688000848f52006a
:100f200008003a003e04900031032000e0cd20008c
:100f3000ce7102000000000000027800840f54000f
:100f4000070032001e427800e04f520001003200dc
:100f5000ffff370014c0b300044f7800a3ff370031
:100f60004f0478000080fa00000006000800fa0034
:100f70003007980094688000140798003e029000a3
:100f80003103200004007800ce7102000000000050
:100f9000000278002407980034032000040f780032
:100fa0006000b8005c830200000000000e027800c0
:100fb0006100200004007800ba83020000000000f5
:100fc0003e0290003103200004007800ba83020042
:100fd000000000000080fa00000006000000fa0097
:100fe000440e200004198800c4032000141988004e
:100ff00094d020002419880054002000441988004f
:10100000f4fd2f00641988000002eb0084198800a9
:101010000080fa00000006000000fa00d2c2a8001a
:1010200004f02f00041688000080fa00000006007b
:101030000000fa0021e3a8000080fa00000006008a
:101040000600fa000518800014188000848242000f
:101050002418800084824200341880008482420078
:101060004418800084824200541880008482420028
:1010700064188000848242007418800084824200d8
:101080008418800084824200941880008482420088
:10109000a418800084824200b41880008482420038
:1010a000c418800084824200d418800084824200e8
:1010b000e418800084824200f41880000482420018
:1010c00005002000048fbe001e02be00452bdd007f
:1010d0004b22de0004027300cb2ade0024079800b6
:1010e0002e029000040078000080fa000000060044
:1010f0000040da000000fe0000c0da000000060038
:101100000a00fa00e20f500022003e0074708000d6
:10111000e10f520006003200872320004623200002
:101120002423200005232000e08f530004003a0010
:1011300087222000462220002422200005222000b1
:10114000000028001500600003003a00800b7800c2
:1011500007002800958a73000540200094826200f1
:1011600001003a0014a0a0008202780006003700b7
:10117000940378000710b200fdff3200b103fb00ba
:10118000070b78008502e900e08f5200f8ff3a0073
:101190000800370034002000b4bf9f00c0bf9f008c
:1011a000d1bf9f00e2bf9f006a805700d2ff0700b7
:1011b0006fb99700020078000080fa000000060076
:1011c000889fbe008a9fbe008c1f78000006eb003f
:1011d000e00f5000e08f5800e00f5900e08f5900f9
:1011e00007003d006044b8006055b800000054009e
:1011f00081805c0002015d0083815d001c00200095
:10120000e00f5200e08f5a00e00f5b00e08f5b00c0
:1012100007003d006044b8006055b8000402540067
:1012200085825c0006035d0087835d000c00a200e0
:1012300012010700e00f5600060032006022b800dd
:101240006033b8000000520081805a0002015b0048
:1012500083815b004f0678004f05be004f04be003f
:1012600000000600889fbe008a9fbe003004be00ba
:101270002005be000404440085844c0006054d0092
:1012800087854d000898be000a90be000440e1002a
:1012900005c8e10006d0e10007d8e10002003100f6
:1012a000680040001008e8004f05be004f04be0073
:1012b000000006001000fa00889fbe008a9fbe0052
:1012c0000605be000404be003002be002003be00be
:1012d000c4b79f00d5b79f00e6b79f00f7b79f0040
:1012e0000802520089825a000a035b008b835b006c
:1012f00084bf9f0095bf9f00a6bf9f00b7bf9f0000
:101300000498be000698be00110020004fb297005e
:10131000dfb297006fb39700ffb39700b2000700ea
:10132000010039008000eb00108810004f05be005e
:101330004f04be000080fa00000006001400fa000e
:10134000889fbe008a9fbe008c9fbe007900070068
:101350000605be000404be000006eb00ccb79f00eb
:10136000bcb79f00acb79f009cb79f008cb79f0095
:101370000d0420004fb39700bfb2970086034300cf
:101380002fb29700e00f530004003d009b000700c0
:101390000f004000b3ff070003003700970007006d
:1013a0000f004000c3ff0700cfb2970095bf9f001a
:1013b000e08f52000900350065000700140020008e
:1013c000050020006033b8000000720081807200c8
:1013d0000201730083817300560007000c06e800c9
:1013e0008d0f5600e3ff3a001fba9700e00f52003e
:1013f00005003d000802be000a03be0000fe2f00eb
:101400000f00400097ff07004faa9700e00f52001f
:1014100008003a000fb497009fb497002fb59700cb
:10142000bfb59700d8b79f00e9b79f00fab79f00f4
:101430008bbf9f00460007004f06be004f05be0051
:101440004f04be000080fa0000000600881f7800ec
:1014500018002000881f7800b8ff07008f87e90078
:101460004f04780000000600801feb00b3ff070068
:101470008f87e90000000600889fbe008a9fbe009b
:101480004100070007003d0044000700180020004d
:101490004900070008003d002f0007000004eb0092
:1014a000050037000004eb004300070002003d0088
:1014b0002900070018002000e4ff0700e00f540097
:1014c00001003200410007004f05be004f04be007e
:1014d00000000600889fbe008a9fbe008c1f780017
:1014e0002900070005003d002c0007001c0020001b
:1014f0003d00070007003d00050037000006eb0037
:101500002d00070003003d006044b8006055b8009e
:1015100013000700d4ff0700e00f5600010032005f
:101520002a0007004f0678004f05be004f04be009a
:1015300000000600010007000000060090b79f00b1
:10154000a1b79f00b2b79f00c3b79f00000006007d
:1015500008000700000006006044b8006055b800ad
:101560000402540085825c0006035d0087835d00f1
:10157000000006001fb09700afb097003fb1970082
:10158000cfb1970000000600e00f5000e08f580038
:10159000e00f5900e08f5900000006006044b800d9
:1015a0006055b8000000540081805c0002015d00bd
:1015b00083815d0000000600e00f5200e08f5a00ba
:1015c000e00f5b00e08f5b00000006006022b800c7
:1015d0006033b8000000520081805a0002015b00b5
:1015e00083815b00000006000820e10009a8e100fb
:1015f0000ab0e1000bb8e100000006004f2bde004e
:1016000087037300a7b79f004f23de008582420047
:101610008502730095b79f00ffaa97004f2bde004d
:10162000040242000402730084b79f006faa97006f
:101630004f23de008582420085027300f5af9f00d4
:10164000ccff07004f18de000402420000027200c7
:10165000e4af9f00c7ff0700000040008180480002
:101660000201490083814900b4ff07000802be005f
:101670000a03be0000fe2f0000000600889fbe0087
:101680008a9fbe008c9fbe000404b8000506b80007
:101690008904460060854e000606b8000a0546002b
:1016a000e0854e000706b8008b054600040eb80022
:1016b000890446000a854e00e0854d00050eb800fd
:1016c0000a0546008b854e00060eb8008b054600c5
:1016d0000416b8000a0546008b854e000516b800b2
:1016e0008b054600041eb8008b0546000800be00ae
:1016f0000a01be004f06be004f05be004f04be00eb
:1017000000000600020ab900001bb9000200b80080
:101710008100420081004300000006000000fa0042
:1017200034088000040078000080fa000000060001
:101730000000fa0054088000040078000080fa00dd
:10174000000006000002780002003700315a7800dd
:101750000201e900e00f5100fcff3a000000060022
:101760000002780002003700015a78000201e90007
:10177000e00f5100fcff3a00000006000002780074
:10178000060037000201e90031437800065a78006c
:1017900084027800e04f5300060032008402780093
:1017a000e00f5100f7ff3a0002003700805aeb00cb
:1017b0000201e900e00f5100fcff3a0000000600c2
:1017c000000278008042eb00b4cf1200fdff3a0027
:1017d0000080ea0000004200000006000c00fa0051
:1017e000889fbe0000047800f4ff2700d4bf9f004c
:1017f0008004eb0099bf9f0088bf9f00a8bf9f0097
:10180000240c2000b4bf9f0078815700cfb0970010
:1018100070805700220007000fba9700094a78002d
:101820000fba9700080052004f04be000080fa0073
:101830000000060001002000107888002178880050
:1018400015c0b30004f02000054a7800000006002f
:1018500004f020008042eb0094cf120002003a0016
:1018600010002000f3ff0700d2e62400631c2400d0
:101870001078800021788000a2ff070094032300e5
:10188000050020000002420081824a00147888008e
:10189000257888000500780000f0a100000006000f
:1018a0002f03b000889fbe008a9fbe008c9fbe00a1
:1018b0008e1f7800e0af9f00c1af9f00b2b79f00be
:1018c0008006eb006e023700cfa897008100e80089
:1018d000c1af9f0054c2b300844f500006003a00cd
:1018e000010278000006eb0001c3b30000c2b300a0
:1018f000b7c2b300070037000000fb00efa8970055
:101900006b020700e10f40005d0232008d06e80027
:101910005b0237008402780034437800d2c2b300ff
:10192000824f53000900320005003c00804f5300f5
:1019300008003200874f53000c003a0007003700c0
:10194000814f530009003a00060037000c30a00018
:10195000f0ff37000c00a000eeff37000c10a000d5
:10196000ecff37000c20a000eaff3700620266009f
:10197000010032000c00a100680266000100320084
:101980000c20a1000602fb000403b100e90f520085
:101990000c003e00050378000002eb006a22b9004b
:1019a000b603fb000703b1000482430086027800ff
:1019b0009603fb000703b100e98f5300f7ff3600e1
:1019c000080037000002eb00a7c2b300874f5300a6
:1019d00004003a00bfb1970043027800b3b79f00fc
:1019e0008502e8000007eb00e6c2b300954f130044
:1019f0000a003a000ce0a00064435300d54f1300e6
:101a00000200320005037800080037003fb397005a
:101a100046077800b6b79f008502e8000503780006
:101a2000080037006a70b90000874300860278001a
:101a3000b603fb000703b100e98f5300f9ff36003e
:101a4000f6ff3700b6427800c6af9f00c0c6b300ad
:101a500080cf5200250032000f003c0036c6b30094
:101a600086cf52006e00320004003c00e0cf5200ee
:101a7000080232006b4353000f00370046c6b30024
:101a800086cf5200170032006543430086cf5200d4
:101a900083003a001300370036c7b30086cf5200e8
:101aa0001f00320007003c006443530086cf520001
:101ab000140032000643e80086cf520078003a0056
:101ac0001300370056c7b30086cf520079003200aa
:101ad0006343430086cf520071003a00a5c79f00c0
:101ae0000d003700a5c79f0074003700f0036600a3
:101af00005012000010032000500280005067600df
:101b0000d0ff3700a5c79f000c60a0006b00370016
:101b1000a5c79f000c50a0000c70a0006700370004
:101b2000a5c79f00bfb09700c1027800b1b79f0062
:101b300005047800e08f520001003a0028ed2000f3
:101b4000080378008002eb00010037008502e800fe
:101b5000e6c37a00e0cf5300fcff3a00850478002a
:101b6000e00f570003003200890f570001003100d9
:101b70008e0478000007eb00890f52000100360048
:101b8000090752006806660014003a000700370093
:101b9000efa8970000022000c5010700e10f4000f8
:101ba000010032008d06e8000e07e900e00f570043
:101bb000f7ff3a000087eb000800370008027800c2
:101bc0003400fb0004047800efa89700b801070078
:101bd000e10f4000010032008d06e80009027800a4
:101be0008404e900e00f5200f4ff3a00e00f5600d1
:101bf000a301320007003700efa897000002200081
:101c0000ab010700e10f4000010032008d06e80043
:101c10000e07e900e00f5700f7ff3a009801370080
:101c20003fb19700c2027800b2b79f00050078006c
:101c3000cf80de000101780082017800f0af9f00c4
:101c400081b79f0092b79f00a3b79f004800de00b6
:101c5000c80add0000807200a0c79f007003660004
:101c600009003200e04f500007003200e14f400011
:101c700005003200b0c79f006fdb9700c6c79f000a
:101c80002900200003003700efdb9700b7c79f0053
:101c90001900200038fc2f000f044400b0ff37006b
:101ca000a5c79f0028fc2f000f0444001900200046
:101cb000abff3700a5c79f000c0cb3008c02780067
:101cc000050cb2002b003a00e00f560005003d0065
:101cd0003fb097004005be004004be00b0b79f0073
:101ce00017003700f00266000f003200bfb2970005
:101cf0004501be00b5b79f00c2a79f00d3a79f00b4
:101d00000503780096029000cfaade00e5a79f00a9
:101d1000f5a79f004fa49700dfa497006fa5970039
:101d2000ffa59700060037003fb0970040047800f9
:101d3000b0b79f00cfc4de00090578008a0578009f
:101d4000e00f5400e08f5c00e00f5d00e08f5d006d
:101d500025003d003c00b3006000b8006011b800f1
:101d600008045000898458000a0559008b855900e1
:101d70001d003700e00f560005003d00bfb0970082
:101d80004105be004104be00b1b79f0016003700f8
:101d9000f00266000e003200bfb297004501be009f
:101da000b5b79f0082af9f0093af9f000003eb0089
:101db000a6af9f008003eb00b7af9f000fac97006a
:101dc0009fac97002fad9700bfad9700060037007e
:101dd0003fb0970040047800b0b79f000900200092
:101de0000a0020000b002000e00f570007003a0017
:101df0001e002000e00f5400e08f5c00e00f5d004b
:101e0000e08f5d00010032000007eb008c007800dd
:101e1000010cb200f1af9f0005042000858f500037
:101e20002c00320003003c00e08f5000080032001c
:101e30003c003700050820007fa99700850f51005e
:101e400010003200050c2000850f510035003a00cb
:101e500086e1200015c0b3003600be003601be008a
:101e60000040e10001c8e10002d0e10003d8e10038
:101e70002b0039008542e800f4cf5200f6ff3a000b
:101e80002700370015c0b30000012000010020002a
:101e90006011b8000040e10001c8e10002d0e1009b
:101ea00003d8e1001e003900460020000000d000e9
:101eb0008180d2000281d2008381d2000603e90032
:101ec000faff3a008542e800f0cf5200f1ff3a00f5
:101ed0001300370015c0b30080002000010020006f
:101ee0006011b8000040e10001c8e10002d0e1004b
:101ef00003d8e1000a003900370020000000d000bc
:101f00008180d2000281d2008381d2008703e90060
:101f1000faff3a008542e800f5cf5200f1ff3a009f
:101f2000a5c79f002fc097008002fb008e8f520034
:101f300002003d00aec79f0003003700850f570029
:101f400001003d0005077800e00f52000300320059
:101f5000e3026600010032000402e90005002400eb
:101f600085026600050032008e0f52000200340028
:101f70000e025200010037000002eb002fc1970053
:101f80008202fb008001eb00d3af9f00850f52005f
:101f90000200340085025200d5af9f006402660043
:101fa0002c003200e202660061026600e08f5200ff
:101fb00006003200b0022000e00f520001003200a3
:101fc0000080e800efa8970004003700e00f5200ff
:101fd00006003200efa8970000022000b4000700be
:101fe000e10f4000010032008d06e8005faa970073
:101ff000e00f52008d0032000802be000a03be004e
:10200000dfac9700efa8970000032000c4b79f0043
:10201000d5b79f00e6b79f00f7b79f00a400070061
:102020004fb29700dfb297006fb39700ffb39700ee
:10203000e10f4000010032008d06e8008904e9004c
:10204000f0ff3a00d9af9f000605be000404be00b1
:1020500076003700dfaa9700e08f520018003200a8
:102060006802660016003a000802be000a03be00bd
:10207000dfac9700efa8970000022000c4b79f00d4
:10208000d5b79f00e6b79f00f7b79f00880007000d
:102090004fb29700dfb297006fb39700ffb397007e
:1020a000e10f4000010032008d06e8008904e900dc
:1020b000f0ff3a00d9af9f000605be000404be0041
:1020c000e202660061026600e08f52000600320004
:1020d000b0022000e00f5200010032000080e80052
:1020e000efa8970004003700e00f52004f003200c5
:1020f000efa89700000220006d000700e10f4000ec
:102100004a0032008d06e800480037000e07e9005b
:102110007fab970007042000870f53002d0032008b
:1021200003003c00e00f5300080032003700370086
:10213000040820007fae9700840f56001200320082
:10214000040c2000840f560030003a004372dd007a
:1021500000e12000000242005403be004402be0021
:102160000800be000a01be00b8fc0700a400200061
:10217000050020006033b800bbfc070004c3b300b7
:10218000044240002000370014ec2000bfa297005a
:10219000e08f52000100320004eb2000c272dd002b
:1021a0000800be000a01be008502e90005003300f8
:1021b0008301d1000281d3008180d3000080d3004d
:1021c000f9ff37006f00600064407800a0c79f00ef
:1021d0000e0037006372b9000800be000a01be009d
:1021e000040678000c06e900050033008301d100e5
:1021f0000281d3008180d3000080d300f9ff370033
:10220000674260000443b000a4c79f00afc09700be
:102210000100fb00efa8970025000700e10f400038
:10222000060032008d06e800040037000c0178003b
:102230000202b200b2a79f008cbf9f00e00f5700c0
:10224000b2ff3a000fbe9700680666000c0032002d
:10225000dfa99700e08f51000900340003067800e1
:10226000efa897000002200011000700e10f4000d6
:10227000010032008d06e8000c06e900f8ff3a0084
:102280004faa970014407800a0c79f00e04f50006d
:102290008dfd3a000d0078004f0778004f06be0014
:1022a0004f05be004f04be002f03b1000000060022
:1022b000889fbe000104780038029000e2026200ac
:1022c0008084eb003b003200040378000620b2005b
:1022d0009802900002003a00e08f520035003a0068
:1022e0000490a0003404980080047800f90fb20034
:1022f000e08f520002003a00a8029000050c78001e
:10230000ea8f540005003a000408b20003003a00c6
:1023100088007800d0002000e5ff07001802900038
:10232000d8029000850f52000b0032000402e80032
:102330001404980018027800094a7800040ce80098
:1023400015c0b30064f02000054a7800ea8f5400fd
:1023500018003a000500370088007800094078002e
:102360001700070080047800120037003802900040
:102370000410b2000f00320018019000a800900075
:10238000480090005efb070018029000840f500088
:1023900004003200380290000403b30034049800b3
:1023a0008084eb000002eb001404980028029000e7
:1023b000040c7800090078004f04be0000000600fd
:1023c0000200fa00889fbe00a0ff9f000104780071
:1023d00038029000840278000504b2000200320046
:1023e0000000fb0035003700e202620005003a0001
:1023f0000403b30034049800150498000080eb0037
:102400002e003700d8049000e08f540006003a00f8
:1024100012002000e68057004800900038fb0700bb
:102420001904980023003700a8029000e08f5200a2
:1024300008003a0095f0200025049800050c78006b
:102440002500200055049800150498000430a000d1
:102450003404980018019000a800900048009000f3
:1024600027fb0700280290008082eb0015049800eb
:10247000affa9700054a7800040ce8002ffa97009d
:10248000ea4f52000b003a00380290000410b200ec
:102490000800320018019000a80090004800900049
:1024a00017fb07000002eb0014049800a80290003c
:1024b000050c78002ffa97000400fb004f04be00c3
:0824c0000080fa000000060094
:020000040000fa
:1024c80045720000726f0000723a0000204d000053
:1024d800535000004c5f0000527500006e4d000024
:1024e8006f64000062750000733a00002045000028
:1024f800727200006f7200002072000065610000b7
:10250800646900006e6700002041000064640000f8
:1025180069740000696f00006e6100006c200000a3
:10252800416400006472000065730000732c0000b1
:1025380020450000727200006f720000636f000097
:1025480064650000203d00002025000064000000b4
:1025580045720000726f0000723a0000204d0000c2
:10256800535000004c5f0000527500006e4d000093
:102578006f64000062750000733a00002045000097
:10258800727200006f720000207200006561000026
:10259800646900006e670000204300005243000099
:1025a8002c20000045720000726f0000726300006a
:1025b8006f640000652000003d20000025640000d5
:1025c80000450000727200006f7200003a2000009f
:1025d8004d530000504c00005f520000756e000023
:1025e8004d6f000064620000757300003a2000001f
:1025f8005772000069740000655000006f72000097
:102608007420000066610000696c000065640000c9
:102618002c20000045720000726f000072630000f9
:102628006f640000652000003d2000002564000064
:1026380000450000727200006f7200003a2000002e
:102648004d530000504c00005f52000065610000cf
:10265800644d000062500000647500003a200000dc
:102668004d530000504c00005f52000065610000af
:1026780064500000616300006b6500007420000076
:1026880066610000696c000065640000207200004b
:1026980065610000646900006e6700002046000064
:1026a800432c000020450000727200006f72000089
:1026b800636f000064650000203d000020250000d5
:1026c8006400000045720000726f0000723a00005a
:1026d800204d0000535000004c5f00005265000080
:1026e800616400004d62000050640000753a00000b
:1026f800204d0000535000004c5f00005265000060
:102708006164000050610000636b000065740000a4
:1027180020660000616900006c650000642000000c
:102728007265000061640000696e000067200000a7
:102738004643000030780000304600002f3000008b
:10274800783100003020000050440000552c000073
:1027580020450000727200006f720000636f000075
:1027680064650000203d0000202500006400000092
:102778004275000066660000657200002074000063
:102788006f6f0000207300006d6100006c6c00002a
:10279800207400006f200000726500006164000072
:1027a80020500000445500000045000072720000ef
:1027b8006f7200003a2000004d530000504c00009a
:1027c8005f52000065610000644d00006250000027
:1027d800647500003a2000004d530000504c000082
:1027e8005f520000656100006450000061630000f2
:1027f8006b6500007420000066610000696c0000d1
:1028080065640000207200006561000064690000d2
:102818006e67000020620000616c0000616e0000bd
:1028280063650000206f000066200000504400002f
:10283800552c000020450000727200006f720000e5
:10284800636f000064650000203d00002025000043
:102858006400000045720000726f0000723a0000c8
:102868002043000052430000206d000069730000ff
:102878006d61000074630000682e000020450000b0
:102888007870000065630000746500006420000033
:102898005b250000785d00005b250000785d000086
:1028a800206600006f7500006e640000205b000069
:1028b800257800005d5b0000257800005d000000c1
:1028c800436f00006c77000061790000205300001e
:1028d8006f6c000075740000696f00006e73000073
:1028e800204d00006f640000627500007320000036
:1028f8004d610000737400006572000020500000f4
:10290800726f0000746f0000636f00006c2000009d
:102918004c6900006272000061720000790d0000cd
:102928000a00000045720000726f0000722100006a
:10293800205500006e610000626c000065200000f8
:10294800746f0000206900006e690000746900005f
:10295800616c000069730000652000004d530000a1
:10296800504c00000d0a000000000000436f0000fa
:102978006c77000061790000204d00005350000082
:102988004c20000020760000352e00003432000074
:10299800202000002020000020200000202000002f
:1029a800202000002020000020200000202000001f
:1029b800202000000000000004a300000000000028
:1029c800004d000043480000504200004f41000005
:1029d80052440000000000000d0a000044480000b6
:1029e800435000002f5000006f7700006572000010
:1029f80020650000766500006e740000206f0000fe
:102a080063630000757200007265000064000000d6
:102a180001000000f4010000f401000001000000c2
:082a2800f4010000f4010000bc
:020000040000fa
:102a30000200fa00004f780044e0200014427800c1
:102a40009e4f52002100320044e0200014427800e2
:102a5000e24f42000c00320044e0200014427800b3
:102a60000482fb007e22b90084027800c4bc2000ee
:102a700004824200e2012000c1c620000400780068
:102a8000a20b0200000000001e40780004eeb70018
:102a90001e427800e24f42000e0032009e42780053
:102aa0000582fb007e22b90084027800c4bc2000ad
:102ab00004824200e201200084007800c0c62000a9
:102ac000a20b02000000000003003700000000001d
:102ad00001003700000000000080fa00000006003e
:102ae0000000fa0055e020009542780044e0200004
:102af0001442780084cf52002f00320054e02000ae
:102b000014427800e24f42001a00320087c02000d1
:102b100054e02000144278000482fb007e22b900b9
:102b200004027800fc024200c4bc2000048242007f
:102b30001443780054e02000144278000482fb0023
:102b40007e22b90084027800c4bc200004824200c6
:102b50001402780085fd2f00848242008402200048
:102b600013c0b300070178008640780005007800a4
:102b70006111070044e0200014427800044078000e
:102b800005eeb70085c82000954278006463800098
:102b900087fd2f008483430086c02000840220002c
:102ba000854178000701780011c0b3000600780065
:102bb0005111070001003700000000000080fa00fa
:102bc000000006000c00fa00e45e200014079800e4
:102bd00014708000e00f520009003a00086d0200f6
:102be000000000000002be0084027800f47f200094
:102bf0008482620004402000048242001470880035
:102c0000c20320008000eb0000c32000b00b0200d4
:102c1000000000000042eb00444798000042eb0037
:102c2000044f78004d0037001e40780080ff0700f9
:102c30001e4078000082fb006622b9008402780002
:102c4000c4502900048242009442900055479800e5
:102c50001e4078000082fb006622b9000402780062
:102c60008482e800c4502900048242009402780063
:102c7000350798001e4078000082fb006622b900ec
:102c800004027800e4024200c45029000482420099
:102c900094027800450798005e4290000482fb0091
:102ca000e00f5200010032002b0037001e009000a0
:102cb00050079800be0290004e02900084824200ad
:102cc0001e02900004824200a402b0001407980083
:102cd0009e029000e4e12000848f5200fcff3e0041
:102ce0005e40900088ecb7005e0290008402b00065
:102cf00064638800656380003e02900004824200a5
:102d00000402e80074638800756380004e0290003e
:102d10000482420084638800d40020001464880088
:102d2000846ca9006eff07009e4278000582fb00bc
:102d30006622b90084027800c4502900048242004f
:102d400014427800044078002fecb700290b0700ec
:102d50001e4fe80001003700ffff37001e427800d9
:102d6000e14f5200b0ff36000080fa00000006007c
:102d70000c00fa001007980021079800624798009d
:102d800043079800244f98000042eb00044f78005e
:102d90009a0037001e40780025ff07001464800069
:102da000ed0f520091003a004dff0700f5c22000e0
:102db000954278002e4a900084cf52008d003a0050
:102dc00084212000646188006e429000e04f520030
:102dd00008003a004e009000c0608800846ca80093
:102de00044002000146488004e029000346488007f
:102df0007c00370015708000f43f2000848f520063
:102e0000040036001570800084382100848f520041
:102e10000200360004402000147088001470800006
:102e2000c46088000402e80014708800ce0390009b
:102e3000b7608800988f0200000000000002be000a
:102e4000d4638800e5638800848ca8006e429000fb
:102e50000482fb006123b9000082eb008082eb005a
:102e60000602420087824a00360020000700200048
:102e7000860f5200878f5a005a003e0004600100fe
:102e80000300370002003700160037002d0037001e
:102e90001e029000ae029000f46088000561880078
:102ea0006e4290000414a2000482fb000402e900b8
:102eb0004f22de00044278000482fb0061026200bf
:102ec0004222dd0056618000b5ff2f0085026300bd
:102ed00004827200546188000002eb0014648800d0
:102ee000400037000e82e800940290000e82e80055
:102ef00014027800848242004e02900084824200d4
:102f0000c460800004826a00346488001e0290005d
:102f1000ae029000f4608800056188000042eb007a
:102f2000044078002eecb700d403200005002000f8
:102f300044608800556088002400200014648800e4
:102f4000280037001e029000ae02900004027800b4
:102f500084027800254290000483fb0035429000f3
:102f60000482fb004822dd000602720004037800a0
:102f70001e029000ae029000040278009443780094
:102f80008782fb00144290000482fb004822dd008f
:102f900005027200840243004e02900084824200c7
:102fa000c460800004826a00346488001e029000bd
:102fb000ae02900004027800a20020008400780095
:102fc000e0c12000a20b020000000000540020001d
:102fd0001464880011c0b30020c0b3003907070093
:102fe000000000001e4278000800370000000000ca
:102ff00001003700000000001e4fe8001e4278006c
:10300000e14f520063ff3600e4cfb3000440780084
:103010000080fa00000006000200fa00004f78006d
:103020001e427800e14f52000200360014002000da
:103030000b0037001e4078007dfe070025648000ed
:103040000400210004826200e00f520003003200fd
:10305000858ca90014002000010037000002eb005d
:10306000040078000080fa00000006000200fa0068
:10307000004f78001e427800e14f520002003600f7
:103080000002eb00080037001e40780068fe0700d1
:103090001464800067026a0004f0a7000402ea00da
:1030a0000402e9004f22de00040078000080fa00ec
:1030b000000006000200fa00004f78001e4278006f
:1030c000e14f520048003e001e40780058fe0700c5
:1030d000b4638000c463880014648000050020008d
:1030e000e600200007002000860f5200878f5a005c
:1030f00037003e0004600100120037000d00370069
:10310000100037000f003700310037000d00370086
:103110000e0037000d0037002d0037002c0037005f
:103120002b0037001800370029003700280037002f
:103130002400370006640200000000002d0a07008a
:103140002a0037002b0a07002800370011c0b300ff
:1031500010c1b300db060700d4608000e00f52000e
:103160000500320095638000a4608000848f5200c7
:10317000f6ff3a0001003700000000008400200044
:10318000146488001900370011c0b30010c1b300e7
:10319000cc060700d4608000e00f5200050032002a
:1031a00095638000a4608000848f5200f6ff3a008f
:1031b0000100370000000000c400200014648800f3
:1031c0000a003700d400200014648800070037008c
:1031d0008040eb0040c1b300ba060700050a0700b3
:1031e0000000000001003700000000000080fa002d
:1031f000000006000200fa00004f78001e4278002e
:10320000e14f520006003e001e40780008fe070015
:10321000846ca9001e407800a6ff0700010037005b
:10322000000000000080fa00000006000200fa0022
:10323000004f78001e427800e14f52000200360035
:103240000002eb000b0037001e407800f8fd07007d
:1032500023fe0700a2002000e1c12000a0c820003a
:10326000a20b020000000000b4608000a46488008b
:10327000a4c82000040078000080fa0000000600c6
:103280000200fa00004f78001e427800e14f520021
:103290000b003e001e407800e5fd070010fe070011
:1032a00095638000a4608000848f52000500320086
:1032b00011c0b30000c1b30082060700010037004f
:1032c000000000000080fa00000006000400fa0080
:1032d000204798002e429000e14f52000200360035
:1032e0000002eb001d0037002e409000d0fd0700cb
:1032f00014648000044f78001e427800e74f5200ab
:10330000050032001e427800eb4f520002003200ee
:103310000002eb001100370095638000a463800079
:10332000848f520009003900756380006463800057
:1033300084825200a66380009463800004025300dc
:10334000048242000402e90004003700a563800003
:1033500094638000048252000402e90004007800b3
:103360000080fa00000006000400fa0020479800e0
:10337000314798002e429000e14f52000200360083
:103380000002eb00440037002e409000a8fd07002b
:103390002e409000cdff070000027800040f780057
:1033a0001e027800e00f520002003a000002eb001b
:1033b000390037001e027800e10f520002003a0087
:1033c0002e409000aeff070025648000041020000e
:1033d00004826200e00f520009003a007563800029
:1033e00064638000048252000402d1009e0f5200e8
:1033f000030039002e409000a1ff0700850ca800b3
:10340000e303470085c8200095427800966380005a
:103410001400200013c0b300070178008540780035
:1034200006007800340f0700946380000402e8006f
:10343000946388009563800074638000848f5200d9
:103440000200390064638000946388001e027800e3
:10345000e10f520003003a002e40900088ff070061
:103460000c00370025648000040220000482620002
:10347000e00f520007003a0084aca800a68f0200bb
:10348000000000000002be00040278006902420051
:10349000f463880014002000040078000080fa0023
:1034a000000006000c00fa006047980041079800f1
:1034b000520798000002eb00140798006e4290003b
:1034c000e14f5200020036000002eb0061003700bd
:1034d0006e40900056fd07006e4090007bff070095
:1034e00000027800240798002e029000e00f52009e
:1034f00004003a006e40900061ff07000002eb00fc
:10350000540037002e029000040f7800ae029000a5
:103510005e029000848f5200020036005e0290002e
:10352000040f7800256480000410200004826200eb
:10353000e00f52000a003a00756380006463800067
:10354000048252008402d1002e029000848f520027
:10355000030039006e40900049ff0700850ca80069
:10356000946380009e02420074638000848f520046
:103570001600390075638000946380000482520055
:1035800014079800ce03900085c82000954278006b
:10359000966380001e02900013c0b30007017800fc
:1035a0008540780006007800d30e0700ce02900018
:1035b0001e02900004824200440798001e02900000
:1035c0001e0f12006463800094638800ce03900095
:1035d00085c8200095427800966380001e0278001e
:1035e00013c0b3000701780085407800060078001a
:1035f000c10e0700946380001e024200946388009d
:10360000ae0290005e029000848f520003003e00e4
:103610006e4090001aff07000c0037002564800000
:103620000402200004826200e00f520007003a000a
:1036300084aca800a68f0200000000000002be00bb
:103640000402780069024200f46388001e029000c0
:103650001e024200040078000080fa00000006000c
:103660000400fa00004f7800110798001e02900035
:1036700004007800e00b0200000000000002780067
:10368000040178009e0090001e40780085ff07002e
:10369000000278009e02900004824200040078003c
:1036a0000080fa00000006000600fa00404798007b
:1036b0004e429000e14f5200020036000002eb0043
:1036c0000c0037004e409000d9fc07007563800065
:1036d0006463800004825200040fe9004e409000b1
:1036e000fafe070000027800140798001e029000fe
:1036f0001e021200040078000080fa00000006009c
:103700000200fa00004f78001e4078000c0007000d
:1037100000027800e00f5200070032001e407800df
:10372000c3fc0700b4638000c463880011c0b30009
:1037300000c1b300630507000080fa000000060026
:103740000200fa00004f78001e427800e14f52005c
:10375000020036000002eb00120037001e40780025
:10376000b3fc0700b5638000c4638000848f5200ff
:1037700004003900b5638000c463800004825200f5
:103780000800370085638000c46380008482520093
:10379000b663800074638000040253000482420018
:1037a0000402e800040078000080fa00000006002f
:1037b0000600fa0020479800210798002e4090004c
:1037c000dfff070000027800040f78001e02780077
:1037d000e00f520002003a000002eb002a0037001e
:1037e0002e40900092fc07002e029000e00f520045
:1037f0000a00320085c8200095427800c763800027
:103800002e03900014002000854178000701780005
:1038100011c0b30006007800370e0700c4638000b3
:103820000402e800c4638800c563800084638000ec
:10383000848f52000200360074638000c4638800e5
:103840001e027800e10f520002003a00854ca800e9
:103850000c0037002564800004022000048262000e
:10386000e00f520007003a0084aca800a68f0200c7
:10387000000000000002be00040278000403b00053
:10388000f463880014002000040078000080fa002f
:10389000000006000a00fa0040479800310798002f
:1038a000420798000002eb00040f78004e409000a1
:1038b000a3ff070000027800140798001e02900082
:1038c000e00f520002003a000002eb005000370007
:1038d0004e40900056fc0700ce0290001e02900061
:1038e000848f5200020036001e02900044079800a8
:1038f000c56380004e029000848242008463800091
:10390000848f52001900360085638000c4638000f4
:1039100004825200040fe8003e029000e00f5200c3
:103920000d00320085c8200095427800c7638000f2
:103930003e0390001e027800854178000701780060
:1039400011c0b30006007800eb0d07003e029000a6
:103950001e024200340798004e0290001e025200e0
:103960004407980074638000c46388003e0290009e
:10397000e00f52000a00320085c82000954278000e
:10398000c76380003e0390004e029000854178009e
:103990000701780011c0b30006007800d60d0700bb
:1039a000c56380004e02900004824200c463880018
:1039b0004e0290001e024200440798009e029000b2
:1039c0004e029000848252004e029000848f52007a
:1039d00002003e00854ca8000c00370025648000e2
:1039e0000402200004826200e00f520007003a0047
:1039f00084aca800a68f0200000000000002be00f8
:103a0000040278000403b000f46388004e029000c2
:103a1000040078000080fa00000006000600fa00aa
:103a2000404798004e429000e14f5200020036009d
:103a30000002eb000b0037004e409000fcfb07003b
:103a40008563800074638000048f52004e409000b4
:103a50003bff070000027800140798001e02900048
:103a60001e021200040078000080fa000000060028
:103a70000e00fa006047980041079800520798002e
:103a8000630798006e429000e14f520003003e0031
:103a90005e029000e00f520002003a000002eb00cc
:103aa000450037006e409000e1fb07006e4090003b
:103ab00023ff07000002780014079800ee02900030
:103ac0005e029000848242001e029000848f5200a9
:103ad000040036009e0290006e02900004825200a4
:103ae00054079800c56380006e029000048f420066
:103af000846380009e0f52000500310085638000c2
:103b000074638000048252000482ea001e0f4200a7
:103b1000846380001e0252000402e800240798001b
:103b2000de0290002e029000848f52000a003e00b8
:103b300085c82000954278004e0390005e029000f8
:103b4000854178001e01780011c0b300060078009e
:103b5000690d07001700370085c8200095427800de
:103b60004e0390002e029000854178001e017800df
:103b700011c0b300060078005f0d0700de02900060
:103b80002e0290000482520085c8200095427800e1
:103b9000776380004e0090002e03900006034000e3
:103ba000854178000701780011c0b3000600780055
:103bb000510d07005e029000040078000080fa00ba
:103bc000000006000600fa00204798002107980030
:103bd000ae019000120020008e0078002e40900070
:103be000a3ff07001e427800044078000080fa001e
:103bf000000006003e00fa0020779800211f980080
:103c0000321f9800431f9800541f9800651f9800aa
:103c10002e729000e14f520003003e003e1a9000c9
:103c2000e00f520002003a000002eb0026013700cc
:103c30002e7090007efb07002e709000c0fe0700e3
:103c400000027800ce1a9000050252001407980076
:103c50009e0290003e1a9000848f520002003100b4
:103c60000082eb00180137005e1a9000e00f52004e
:103c7000060032009e0290005e1a9000848f52006f
:103c8000020036005e1a900014079800c563800099
:103c90004e1a900004824200340798008563800029
:103ca0003e029000848f520007003100856380003f
:103cb00074638000048252000482ea00be02900015
:103cc0000482420034079800be029000050f78007d
:103cd000856380003e029000048252000402e800e6
:103ce000240798004e1a900034079800be1a9000de
:103cf000750798002e1a9000040f98002e1a900055
:103d000094427800154f98002e1a90000402e800a3
:103d1000241f98000002eb00640798006e1a9000c0
:103d2000e00f52000c0032009e4a900004c6b3001f
:103d300084cf5200080036009e4a9000a4c7b3000a
:103d400084cf520004003e009e4a900004ceb3008f
:103d500004c24200144f980004c2b300244f9800dc
:103d60002e4a90008482fb002e029000848f520025
:103d7000020036002e029000244f98002e4a900038
:103d80008482fb001e029000848f520002003600e5
:103d90001e029000244f98002e4a90000482fb00df
:103da00085c820009542780072034700854178005d
:103db0001e01780011c0b30006007800ce0c070089
:103dc0002e4a90000482fb001e0f42002e4a9000f3
:103dd0000482fb00ae029000048252002407980087
:103de0002e029000e00f520004003a00746380003d
:103df000040f78000082eb00240798006e1a9000f0
:103e0000e00f5200680032000042eb00044f9800bf
:103e1000600037000e4a90000482fb000402470055
:103e2000a452900004c6b30084cf520011003600a3
:103e30000e4a90000482fb0004024700a452900046
:103e4000a4c7b30084cf52000a003e000e4a90007f
:103e50000483fb000e4a90000482fb00040247002a
:103e6000a452900004ceb30004c242008602470070
:103e7000a45298000e4a90000482fb0004024700fe
:103e8000a45290001e4a900084cf520023003a00b2
:103e90003e1a90000402e900341f98003e1a900078
:103ea000e00f520008003a00be0290007e0290002f
:103eb000848252000e4a90000482fb000482420079
:103ec0000402e800800037002e1a90009442780027
:103ed000154f98002e1a90000402e800241f980045
:103ee00014002000640798009e4a900004c6b300a6
:103ef00084cf5200240036009e4a9000a4c7b3002d
:103f000084cf520020003e009e4a900004ceb300b1
:103f100004c24200144f98001b0037007e0290003c
:103f2000341f98006e029000e00f5200160032001d
:103f30008e0a9000251f98002e1a90009442780057
:103f4000154f98002e1a90000402e800241f9800d4
:103f50009e4a900004c6b30084cf52000800360089
:103f60009e4a9000a4c7b30084cf520004003e00d4
:103f70009e4a900004ceb30004c24200144f980041
:103f80000002eb00640798000e4a90000442e8002b
:103f9000044f98008e4a90002e4a900084cf520021
:103fa0009cff3900370037000042eb00044f9800b7
:103fb000300037000e4a90000482fb0004024700e4
:103fc000a45290001e4a900084cf520017003a007d
:103fd0003e1a90000402e900341f98003e1a900037
:103fe000e00f520008003a00be0290007e029000ee
:103ff000848252000e4a90000482fb000482420038
:104000000402e800300037002e1a90009442780035
:10401000154f98002e1a90000402e800241f980003
:1040200014002000640798000f0037007e02900003
:10403000341f98006e029000e00f52000a00320018
:104040008e0a9000251f98002e1a90009442780046
:10405000154f98002e1a90000402e800241f9800c3
:104060000002eb00640798000e4a90000442e8004a
:10407000044f98008e4a90002e4a900084cf520040
:10408000ccff39002e4a90000482fb009e02900073
:1040900004825200140798009e0290003e1a90007d
:1040a000848f5200020031000082eb0006003700ce
:1040b0002e4a90000482fb00be029000048242005f
:1040c0003407980024ff3700040078000080fa00cd
:1040d000000006000800fa00004f78001147980021
:1040e0001207980023079800340798000e03e80091
:1040f000be0290002e0290009e019000120020004f
:10410000860078001e407800bafe070000027800a2
:10411000040078000080fa00000006000e00fa009b
:10412000881f78000042eb00044f78003c02370003
:104130001e4078003efa07000042eb0064479800fa
:104140000002eb00140798000002eb00240798001f
:10415000256480000420200004826200e00f5200e9
:1041600005003a00256480000440200004826200bb
:10417000e00f52000c003200843a02000000000000
:1041800000027800e00f52000700320004c1b300c3
:1041900064479800246480004a22de006142620085
:1041a0000482fb00140798002564800004022000ac
:1041b00004826200e00f52000a003200f8638000bf
:1041c000a68f0200000000000002be00040278007a
:1041d00004025400e00f520002003c0004c1b3008e
:1041e0006447980025648000040420000482620073
:1041f000e00f52000a00320008648000a68f02001f
:10420000000000000002be00040278000402540016
:10421000e00f520002003c0004c1b3006447980064
:1042200014648000eb0f52000c003a000864800018
:10423000a68f0200000000000002be000402780009
:1042400004025400e00f520004003c0014c1b3000b
:1042500064479800c400200014648800146480003f
:10426000e40f520064003a000002eb00440798009b
:104270005c0037004e0290007422b90004027800fe
:10428000f002420004c320000482420014027800bd
:10429000e00f5200570032004e0290007422b90025
:1042a00004027800f002420004c3200004824200ad
:1042b0009402780034648000848f520046003a00f3
:1042c00007fa07004e0290007422b90084027800b9
:1042d00004c3200004824200a20020008400780071
:1042e000e0c12000a20b0200000000004e0290007e
:1042f0007422b90004027800ea02420004c32000dc
:104300000482420014027800b46088004e029000db
:104310007422b90004027800ec02420004c32000b9
:10432000048242001402be0061024200e0824a00a0
:10433000846088009560880005618000f4608000da
:1043400084824200b460800084824200c4608000a5
:1043500004826a003464880024c1b3006447980072
:104360006400200014648800ce029000c4fe2f0078
:1043700004aab90004027800870220008483430065
:104380004e0290000402e8007422b9008402780012
:1043900004c3200004824200040378004e0290000f
:1043a0007422b9008402780004c320000482420011
:1043b000840278000702780013c0b3000601780079
:1043c00011c0b300050078004b0b07000002eb00a2
:1043d00044638800080037004e0290000402e800a1
:1043e000440798004e029000e20f5200a1ff3600f1
:1043f00001003700000000006e429000e04f5200c4
:10440000090032001e02900004f0a7000402ea0036
:104410000402e9004f22de00044278008440780064
:104420006e40900027020700246480007002620042
:10443000e00f52002d003a0014648000e70f520094
:104440006f013a00988f0200000000000003be00d8
:10445000d4638000e56380000402530085825b0022
:10446000e00f5200e08f5a0067013500246480009d
:1044700067026200e60f52000e003a0024648000da
:104480004322de0061426200644798001e407800cb
:1044900008fb07001e40780006fb07006e429000f4
:1044a000e04f52005a013a00e400200014648800f2
:1044b0005a0137008af9070021c0b30000c1b300d8
:1044c00000020700988f0200000000000003be00f9
:1044d00084962800950020000602420087824a0048
:1044e000d4638800e56388004c013700988f020090
:1044f000000000000003be00d4638000e56380007c
:104500000402530085825b00e00f5200e08f5a00e6
:104510004101350072f90700146480000500200095
:10452000c600200007002000860f5200878f5a0027
:10453000ef003e00046001000c0037002600370049
:10454000530037005d003700eb003700860037006e
:1045500095003700a9003700b6003700c3003700c8
:10456000c7003700a5003700d3003700ec63020016
:104570000000000000027800e00f5200e00032006e
:1045800014002000146488005461800064026200fa
:10459000e00f520008003200f460800005618000e6
:1045a0000402780011c0b3000400780038640200ef
:1045b00000000000d9003700f46080000561800031
:1045c0000402780011c0b3000400780038640200cf
:1045d00000000000d10037006a02470004007800a4
:1045e0006a6402000000000000027800e00f520040
:1045f000c5003200066402000000000000027800de
:10460000e00f5200160032005e029000ee029000b1
:10461000f46088000561880024002000146488008c
:1046200005618000f460800084824200b4608000f4
:1046300084824200c460800004826a00346488007e
:104640000042eb00044078002eecb700d4032000b9
:10465000050020004460880055608800af003700e6
:10466000988f0200000000000003be00849628001e
:10467000950020000602420087824a00d463880029
:10468000e56388000002eb0014648800a300370093
:10469000a68f0200000000000002be0004027800a5
:1046a000f4638800e0c120004880020000000000a0
:1046b00034002000146488009800370021c22000d4
:1046c000e0c120000a810200000000000002780022
:1046d000e00f52001d003a00a68f0200000000000b
:1046e0000002be0084027800f4638000048352005c
:1046f000446080005560800004027800840f5300fd
:1047000083003600e4c2200014427800e54f5200d6
:104710000b003e00e4c22000144278000442e8008e
:10472000044078002eecb7004460800055608000a3
:104730000402420085824a00446088005560880077
:1047400024002000146488007400370024c0b300e3
:10475000644798000002eb00140798005400200002
:10476000146488006d00370024c0b30064479800cb
:104770001400200014079800e4c2200014427800be
:10478000e34f52006400360044c0b3000440780098
:104790002eecb70004242400f500200044608800bb
:1047a000556088005d003700e4c2200014427800a4
:1047b000e14f520005003e0024c1b3006447980059
:1047c000140020001407980054003700246480006f
:1047d00068026200e00f52000500320044c1b300dd
:1047e0006447980014002000240798004b0037000d
:1047f00024c0b3006447980048003700e4c220009a
:1048000014427800e44f520005003e0004c1b3009a
:104810006447980014002000140798003f003700f8
:10482000840020001464880014c1b3006447980019
:104830003a003700e4c2200014427800e44f5200ee
:1048400005003e0014c1b300644798001400200026
:10485000140798003100370044c1b3006447980042
:1048600014002000240798002c00370044c1b30036
:1048700064479800140020002407980027003700a0
:10488000e4c2200014427800e44f520005003e00cc
:1048900004c1b30064479800140020001407980076
:1048a0001e00370044c1b300644798001400200084
:1048b0002407980019003700e4c220001442780051
:1048c000e44f520005003e0014c1b3006447980055
:1048d00014002000140798001000370044c1b300f2
:1048e0006447980014002000240798000b0037004c
:1048f000000000000900370000000000070037003a
:104900000000000005003700000000000300370031
:104910000000000001003700000000006e4290001f
:10492000e04f5200310032001e029000e00f5200b2
:104930002b003200e4c22000144278000442e80058
:10494000044078002eecb700446080005560800081
:104950000402420085824a00446088005560880055
:10496000a5608000a4638000048252004407980080
:10497000a5608000a4638000848f5200060031008f
:10498000756380006463800004825200ce02900050
:1049900004824200440798006660800077608000cf
:1049a0004e029000050020000402530085825b0047
:1049b0006460880075608800d56080004e029000b9
:1049c00004824200d4608800a4638000a460880050
:1049d0008040eb006e409000ba00070003003700f3
:1049e00011c0b3006e409000b60007002e02900088
:1049f000e00f520009003200fe03070007003700f5
:104a00000000000005003700000000000300370030
:104a10000000000001003700000000001e4fe80009
:104a20001e427800e14f5200c1fd36000002eb004b
:104a300044079800390037004e0290007422b900f4
:104a400004027800f002420004c320000482420005
:104a500014027800e00f520034003200a68f0200ea
:104a6000000000000002be00040378004e02900027
:104a70007422b90004027800f202420004c320004c
:104a8000048242001402780084025300c42d2000e6
:104a9000848f52001e003600ce029000c4fe2f000c
:104aa00004aab9000402780087022000848343002e
:104ab0004e0290000402e8007422b90084027800db
:104ac00004c3200004824200040378004e029000d8
:104ad0007422b9008402780004c3200004824200da
:104ae000840278000702780013c0b3000601780042
:104af00011c0b300050078007f0907000002eb0039
:104b0000446388004e0290000402e90044079800c4
:104b10004e0290000402e800440798004e02900004
:104b2000e20f5200c4ff3600010037000000000011
:104b30004f0478000080fa00000006002c00fa0004
:104b40003017980041179800521798003e139000b4
:104b5000164278000480fb00964390008783fb0098
:104b6000c83bdd008083730007027800a6439000f5
:104b70008783fb00364390000683fb004833dd004b
:104b80000703730086027800340f9800450f9800e1
:104b90004e1290001403be00560f9800670f980045
:104ba0000042eb00645f980064c0b300745f98003b
:104bb000de139000071798000e1290000400780092
:104bc00052710200000000000002780004179800f3
:104bd00076024700c100200004007800ce71020078
:104be00000000000000278000482ea001417980018
:104bf0005e109000bc3d0200000000000002780042
:104c0000241798009e1290002e129000848f52005c
:104c1000040032009c3a0200000000001400200052
:104c2000250037000000eb00728b0200000000003e
:104c30000e82e8004101200004007800fa3e0200e4
:104c4000000000000e82e80004007800290307003d
:104c50007e0290004422de006f42620025002000a8
:104c60000522dd00744f52009e4278000582fb0051
:104c7000de12900004825200740252005417980011
:104c80000e82e800be10900004007800f3010700d7
:104c900000027800e00f5200040032000e82e800ab
:104ca000de10900004007800010407009c3a020026
:104cb0000000000014002000040078000080fa00ca
:104cc000000006002a00fa00006f9800116f98009b
:104cd00083f707000e6a90000482fb006102620005
:104ce00004427800e04f520005003200856ca800b5
:104cf0008e6a9000e4cfb30004c26200046f980093
:104d000084aca90084cca90084eca900852ca9005e
:104d1000854ca900850ca90000000000843a02001f
:104d20000000000000027800e00f5200fbff32009c
:104d30000e6a90000482fb0066026200e00f5200df
:104d4000030032000002eb00040f78007600370009
:104d500095638000a4608000848f520003003a00b5
:104d60000002eb00040f78006100370095638000bb
:104d7000a4608000848f52001b0036009563800081
:104d8000a4608000048f5200d46080009e0f520007
:104d900002003100d0608000000f78006461800064
:104da0009e0f52000300310064618000040f780000
:104db000854ca80085c8200095427800a660800038
:104dc0001e02780085417800060178008040eb00e3
:104dd00060032000c8080700a46080001e02420093
:104de000a46088004200370075638000a4608000e2
:104df0000482520034179800be1290009463800021
:104e00008482420064638000048f5200d46080007a
:104e10009e0f520002003100d5608000050f78001f
:104e2000646180009e0f52000300310060618000c9
:104e3000000f7800854ca8003e1290009e0f520093
:104e4000020036001e027800341798003e129000cf
:104e500085c8200095427800a660800085417800d2
:104e6000060178008040eb0060032000a2080700e4
:104e70003e1290001e021200341798003e1290005d
:104e8000e00f52000d0032003e12900085c8200055
:104e9000954278006763800070638000a6608000a0
:104ea000060350006603b0008541780007017800d2
:104eb0008040eb00060078008f080700a4608000a7
:104ec0001e024200a4608800a56080007463800018
:104ed000848f520006003900a56080006663800060
:104ee000746380000402530004824200a4608800be
:104ef000256480000480200004826200e00f5200dc
:104f000009003200d46080009e0f5200060032007b
:104f1000646180009e0f5200030032000e6a900010
:104f20000404a000046f98001e027800e00f5200f5
:104f300005003a000e6a90000482fb0063026200e2
:104f4000e00f520021003200d46080001e025200a7
:104f5000d46088001e027800e00f52000300320087
:104f60000e6a90000434a000046f98001e6a90003e
:104f70000482fb006102620004427800e04f5200ac
:104f8000070032000042eb00044078002eecb7002e
:104f900044422f00050020004460880055608800ce
:104fa000988f0200000000000003be0044608000f3
:104fb000556080000602420087824a00d463880060
:104fc000e5638800848ca8003a0037001e6a9000d0
:104fd0000482fb0062026200e00f52001400320003
:104fe00024648000674262000442e8006742620075
:104ff0000482fb00670262002664800085ff2f00a8
:10500000850263000482720024648800646080006a
:105010007560800061025200e0825a00646088007e
:105020007560880014002000040f7800210037000c
:105030002464800070026200e00f52001d00320004
:105040001e6a90000482fb0061026200e00f5200c1
:105050000f003a00e4c2200014427800e04f5200f2
:105060000b003200e4c22000144278000442e90040
:10507000044078002eecb70044608000556080004a
:105080008502d1000482d300446088005560880006
:10509000988f0200000000000003be004460800002
:1050a000556080000602420087824a00d46388006f
:1050b000e5638800c460800024079800b460800025
:1050c0003407980064608000756080004407980091
:1050d0005507980084608000956080006407980000
:1050e000750798000e0a900004e0a10004f0a100ea
:1050f000040f98000e0a90000400a1000410a10003
:105100000420a1000430a100040f98000e6a900052
:10511000145798000002eb00340f9800666080007e
:10512000776080001e027800050020000602420021
:1051300087824a0064608800756088000e6a90006b
:105140000482fb0062026200e00f52001a0032008b
:105150000e6a90000482fb0070026200e00f5200b1
:1051600003003a006022b8006407980075079800b1
:105170005461800062026200e00f520007003200ba
:105180004e029000de02900061025200e0825a005e
:1051900044079800550798000700370064608000b6
:1051a0007560800061024200e0824a00646088000d
:1051b000756088002a2ca8000e6a90000482fb000b
:1051c0006102620004427800e04f520001003200a8
:1051d0002a0ca800b5638000c4638000848f52004d
:1051e0000900390085638000746380008482520066
:1051f000c6638000b463800004025300048242004e
:10520000140f980005003700c5638000b463800068
:10521000048252000402e900140f9800ce3a020002
:105220000000000000027800140798009e02900021
:10523000f4032000848f520003003e000002eb00c4
:1052400014079800030037001e0290000404b10008
:10525000140798009e0a90001e029000848f52004e
:10526000020036001e029000140f980064024700ee
:10527000040078009f0107009e027800748f4200ae
:105280000e0a90000440a0000450a1000460a00099
:105290000470a100040f98000e6a90000482fb00c5
:1052a00062026200e00f5200150032001e0078001a
:1052b000640f400024c0b300045f980044c0b300f2
:1052c000145f980024802100540f98000e0a90006b
:1052d0004422de006f4262000442e8006f42620036
:1052e0000482fb006f0262004422dd000e0b90007e
:1052f000f5f02f008502630004827200040f98000d
:10530000e6cd2000164378008683fb00f6cd200012
:10531000164378000683fb004833dd000703730063
:105320000602780006ce2000164378008683fb0034
:1053300016ce2000164378000683fb004833dd00bc
:105340000703730086027800640f9800750f9800b9
:10535000f46080000561800004179800151798001c
:105360000042eb004467980064c0b30054679800a3
:105370009e027800351798003e12900004007800d5
:1053800052710200000000000002780034179800fb
:105390007c024700c100200004007800ce710200aa
:1053a00000000000000278000482ea00240f980048
:1053b000e0002000083d0200000000001e0178000f
:1053c00061c0b300e0c12000c08a020000000000fc
:1053d000640247004101200004007800443f0200bd
:1053e000000000000e6a90000482fb00620262006e
:1053f000e00f520005003200780247004100200013
:1054000004007800443f0200000000002002200059
:10541000223d0200000000001e007800bc3d02009a
:10542000000000000002780014079800200320000c
:10543000083d0200000000000e82e800210020006c
:1054400004007800443f020000000000883c020095
:10545000000000000080fa00000006000a00fa00c8
:1054600030079800410798003e0290001402900017
:10547000e00f520002003a000002eb001a01370070
:10548000e4cfb30014479800ce029000254290006c
:105490000483fb00354290000482fb004822dd00bb
:1054a00006027200840278004e0290009443780055
:1054b0000783fb00144290000482fb004822dd00b9
:1054c00006027200848242003e02900014027800bc
:1054d000848242003e0290001402900004826a001e
:1054e000240798000042eb00044f78003b0037008f
:1054f0001e4078004ef5070014648000ed0f520046
:105500003000320014648000e40f520008003a00ba
:10551000356480003e02900014029000848f520097
:105520002a003a001e427800144798002a003700eb
:10553000356480002e029000848f520025003a00ce
:1055400067f507003e02900094029000c46080005e
:10555000848f520020003a003e02900094027800ae
:10556000b4608000848f52001b003a004e0390000c
:10557000964378000780fb00964390008783fb00ea
:10558000c83bdd008083730007027800a6439000cb
:105590008783fb00364390000683fb004833dd0021
:1055a0000703730086027800f660800007618000c0
:1055b000860f5200878f5a0007003a00140020001f
:1055c000c9003700000000000300370000000000a1
:1055d00001003700000000001e4fe8001e42780066
:1055e000e14f5200c2ff36001e429000e24f4200df
:1055f000170032001e4090000df5070038f5070037
:105600001e429000e24f4200110032002e02900034
:1056100034648800a2002000ce009000e0c1200089
:10562000a20b0200000000003e029000140278006d
:10563000b46088003e02900014029000c4608800ac
:1056400064638000a460880014002000a600370076
:105650003e029000e40290000420200004826200d8
:10566000e00f520002003a000002eb009e003700fb
:1056700044638000e00f5200020032000002eb00a1
:10568000990037000002eb00140798004b00370028
:105690001e0290007422b90004027800f002420059
:1056a00004c320000482420014027800e00f52007c
:1056b000460032001e0290007422b90004027800f5
:1056c000f002420004c320000482420094027800e9
:1056d0003e02900014029000848f52002f003a0086
:1056e0001e0290007422b90004027800ea0242000f
:1056f00004c3200004824200940278003e0290001d
:1057000014027800848f520026003a001e02900096
:105710007422b9008402780004c32000048242008d
:105720001403be004e009000104278000481fb007c
:10573000904090008180fb00c808dd0082807000ee
:1057400001027800a04090008180fb003040900072
:105750000080fb004800dd0001007000800278003e
:10576000840f5300858f5b0010003a00a68f020063
:10577000000000000002be00040378001e0290003a
:105780007422b9008402780024c4200004824200fc
:10579000060a78000002eb0053003700000000000a
:1057a0000300370000000000010037000000000087
:1057b0001e0290000402e800140798001e029000e8
:1057c000e20f5200b2ff3600010037000000000077
:1057d0000042eb00044f78003f0037001e40780085
:1057e00093f407002464800068026200e00f520016
:1057f00035003200baf40700c56080003e02900018
:1058000014029000848f520031003a001e02900072
:105810007422b9008402780004c32000048242008c
:10582000a2002000ce00900004007800a20b02002d
:10583000000000003e029000140378001e02900059
:105840007422b90084027800a4c3200004824200bc
:10585000060a78003e029000b402900024029000f4
:105860001e0390007433b90086037800c6c320007d
:1058700006834300048bbe003e0290001403900098
:105880001e0290007422b9008402780004c4200033
:1058900004824200060a7800a68f02000000000081
:1058a0000002be00040378001e0290007422b900ba
:1058b0008402780024c4200004824200060a780092
:1058c0000002eb0008003700000000000100370074
:1058d000000000001e4fe8001e427800e14f520019
:1058e000beff36000002eb00040078000080fa00e2
:1058f000000006000200fa00000f78001e02780087
:1059000014027800040078005271020000000000c8
:10591000000278009e027800840a78001e02780057
:105920001402900004007800527102000000000090
:10593000000278009e027800940298001e0278000f
:10594000b4029000240290000400be006e710200b8
:10595000000000000002be001e037800240398002f
:10596000350398001e027800d40290004402900093
:105970000400be006e710200000000000002be00c4
:105980001e03780044039800550398001e02780017
:1059900074029000040078005271020000000000c0
:1059a000000278009e027800f40298001e0278003f
:1059b000040a900004007800527102000000000008
:1059c000000278009e027800840a98001e02780087
:1059d000140a9000040078005271020000000000d8
:1059e000000278009e027800940a98000080fa0075
:1059f000000006000000fa00881f780038f4070055
:105a0000c46080003464880064638000946388000c
:105a100064638000a463880074638000b4638800ba
:105a200074638000c463880024648000680262009c
:105a3000e00f520002003200440020000100370055
:105a4000d400200014648800840ca900842ca900d0
:105a5000844ca900848ca90084aca90084cca90042
:105a600084eca900850ca900852ca900854ca9000f
:105a7000856ca900858ca8002a0ca9002a2ca900f5
:105a80002a6ca9002a8ca90064638000a4608800a5
:105a9000c8c02000986c02000000000000027800de
:105aa000040c7800c8c02000986c020000000000c0
:105ab00000027800140498000082eb004461880022
:105ac00014002000d46088004f0478000080fa00a1
:105ad000000006000400fa00881f7800c0002000c3
:105ae000728b020000000000e83e0200000000008f
:105af00000427800044f78001e4278008482fb0048
:105b0000040f20000482620042a2de0004427800fa
:105b1000744f52001e427800e04f520002003a00db
:105b2000842120005e003700710020000000eb009f
:105b3000fa3e02000000000046003700e83e020086
:105b40000000000000427800144798001e429000b8
:105b5000e04f5200480032001e429000e14f5200d8
:105b60003b0032001e429000e24f520023003a00f8
:105b70001e427800e24f5200410036000002eb0066
:105b800014079800e83e0200000000000042780080
:105b9000144798001e429000e44f52000b003a0058
:105ba0000e82e8000404e800e83e02000000000065
:105bb00000427800044c78000e84e800e83e0200c1
:105bc0000000000000427800044c78009e02900023
:105bd00074212000848f52002b0036009e0290001a
:105be000445b2000848f520002003600445b20009a
:105bf0002b0037001e029000290037001e4278005b
:105c0000e14f520022003600e83e02000000000092
:105c100000427800144798001e4290009e4278008f
:105c200084cf52001c0039001e4290000482fb0009
:105c3000840078000000eb00fa3e02000000000043
:105c40009e4278001e42900004cf520001003700af
:105c5000000000009e4278000582fb000402ea007a
:105c60004f22de00044278001e4fe900e04f520050
:105c7000b2ff3a00090037000000000007003700bb
:105c8000000000000500370000000000030037009e
:105c90000000000001003700000000008421200007
:105ca000040078004f0478000080fa00000006002d
:105cb0002200fa00700f9800011798007e0a9000e9
:105cc000d44a9000055798007e0a90004403900043
:105cd000d403900046079800570798007e0a90006a
:105ce00024039000b4039000160f9800270f98002b
:105cf000840ca900842ca900844ca9002464800091
:105d000070026200e00f520009003a00988f020012
:105d1000000000000003be008496280095002000cb
:105d20000602420087824a00d4638800e563880047
:105d300014648000e40f520003003200e50f5200ab
:105d40002c003200780037000e5290000482fb00d5
:105d500064026200e00f52000200320025ff0700db
:105d60002e0437000e5290000482fb007002620085
:105d7000e00f5200090032004e029000de02900057
:105d800064608800756088008040eb0040c0b3000c
:105d9000ccfb070017ff0700200437000e529000cd
:105da0000482fb0062026200e00f52000f0032002a
:105db0001e0a9000ae0a900061024200e0824a0092
:105dc000846088009560880042ff07000002780028
:105dd0006461880011c0b30020c1b300b9fb0700a3
:105de00064002000146488000c04370001ff0700e1
:105df0000a0437000e5290000482fb006402620025
:105e0000e00f5200f2033a000e5290000482fb00b1
:105e100070026200e00f52001700320066608000de
:105e2000776080004e029000de029000840f5300e5
:105e3000858f5b0010003200666080007760800014
:105e4000160f9800270f98004e029000de02900077
:105e5000646088007560880011c0b30040c0b30062
:105e600098fb07001e0b9000ae0b90006660880048
:105e700077608800e90337000e5290000482fb002f
:105e800062026200e00f5200d30332001e0a90004b
:105e9000ae0a900061024200e0824a0084608800fd
:105ea000956088007e0a900074029000d46088009b
:105eb00008ff070000027800646188000e5290001d
:105ec0000482fb0070026200e00f520010003200fa
:105ed00011c0b30000c1b3007afb070074002000ba
:105ee00014648800988f0200000000000003be00c8
:105ef00084962800950020000602420087824a000e
:105f0000d4638800e5638800848ca900c30337004c
:105f100011c0b30020c1b3006afb07006400200079
:105f200014648800bd0337008e1390006707980043
:105f30000e5290000482fb0061026200044278006d
:105f4000e04f5200030032006e0290000402e800ad
:105f5000640798000e5290000482fb006202620007
:105f6000e00f5200030032006e0290000402e800cd
:105f700064079800b5638000c4638000848f52007a
:105f800009003900856380007463800084825200b8
:105f9000c6638000b46380000402530004824200a0
:105fa0003407980005003700c5638000b4638000a3
:105fb000048252000402e9003407980084608000e3
:105fc000956080001e0b9000ae0b90000402530001
:105fd00085825b00340f9800450f98003e0a9000c0
:105fe000540f98000002eb00740798006e029000b6
:105ff000e00f5200350032003e029000e00f5200e8
:10600000480032003e0a9000ce0a9000e00f520095
:10601000e08f5a000a0035003e0290006123b8006c
:106020003e0a9000ce0a9000840f5300858f5b00db
:106030000300360014002000740798001400370095
:106040006e0290006123b8003e0a9000ce0a9000d4
:106050000602420087824a00e00f5200e08f5a0099
:106060000b003400be0290006e02900004825200c9
:106070006123b9003e0a9000ce0a9000840f5300bd
:10608000858f5b0002003500140020007407980023
:106090003e0290006123b8003e0a9000ce0a9000b4
:1060a000840f5300858f5b001e003400de0a9000d1
:1060b0006e02900004824200e00f5200190034008a
:1060c0001400200074079800160037003e0a900064
:1060d000ce0a9000e00f5200e08f5a0003003a0011
:1060e00014002000740798000e0037003e0a90004c
:1060f000ce0a9000e00f5200e08f5a0009003500f0
:106100003e0290006123b8003e0a9000ce0a900043
:10611000840f5300858f5b000200360014002000be
:10612000740798007e029000e00f520009003a00c8
:106130000e5290000482fb0064026200e00f5200e5
:1061400027033a0011c0b30000c1b300ddfa070015
:10615000320337000e5290000482fb006602620098
:10616000e00f52000200320022fe07002b0337002e
:106170000e5290000482fb0070026200e00f520099
:1061800019033200146480006123b800a4ff2f00bb
:10619000f5ff2f000602420087824a0066002000b9
:1061a00007002000860f5200878f5a005b013e00d7
:1061b00004600100060037001e0037001d00370094
:1061c0001c0037001b0037001a0037004801370059
:1061d00066608000776080004e029000de029000d2
:1061e000840f5300858f5b001000320066608000d2
:1061f00077608000160f9800270f98004e029000dd
:10620000de029000646088007560880011c0b300f1
:1062100040c0b300abfa07001e0b9000ae0b90001d
:106220006660880077608800fc02370074002000f8
:106230001464880095638000a4608000048252008a
:10624000240798002e029000e00f520006003d0047
:10625000756380006463800004825200ae02900087
:106260000482420024079800666080007760800006
:106270002e02900005002000041f430005974b00ec
:106280004e039000de0390001e02be000402530085
:1062900085825b00048fbe001e02be00e00f52002c
:1062a000e08f5a00140034005461800061026200e3
:1062b000e00f5200060032001e03be001400200052
:1062c00005002000840f5300858f5b00040032001e
:1062d0008040eb0000c1b3007afa0700cf0237001c
:1062e0004e029000de02900061025200e0825a00ed
:1062f000440798005507980066608000776080002a
:10630000a5608000a463800004825200cfa2de005a
:10631000041f530005975b00a5608000a463800004
:10632000848f520006003100756380006463800032
:1063300004825200050020001e1f12001e971a0042
:106340004e029000de0290001e1f52001e975a005f
:106350001e02be00e00f5200e08f5a0050003400d1
:106360007563800064638000048252000500200091
:10637000be0f5200ae8f5a00490039002a6ca900a6
:106380002a8ca900850ca900a76380002707980024
:10639000a56380001e02780004824200a463880086
:1063a000a56080002e029000848f520011003900f9
:1063b000a5608000a4638000848f52002300310018
:1063c0006660800077608000a5638000a460800024
:1063d00004825200050020000602420087824a0023
:1063e0006460880075608800a4638000a4608800f1
:1063f00016003700a560800076638000646380002b
:10640000040253000482420024079800a563800020
:106410002e029000848f52000c00360066608000cf
:1064200077608000a56380002e02900004825200f5
:10643000050020000602420087824a00646088004e
:1064400075608800a4638000a4608800a563800054
:1064500074638000848f520006003900a5638000b9
:10646000666380007463800004025300048242006b
:10647000a4638800a560800074638000848f52004c
:1064800030003900a560800066638000746380007e
:106490000402530004824200a460880029003700ef
:1064a000a5638000a4608000848f52002500320024
:1064b0005461800068026200e00f52002000320048
:1064c0005461800070026200e00f52001b00320035
:1064d0006660800077608000a5608000a463800013
:1064e00004825200cfa2de000402530085825b00ca
:1064f0006460880075608800a5608000a4638000e7
:10650000848f52000a00310066608000776080004e
:10651000756380006463800004825200cfa2de00b5
:106520000402530085825b00646088007560880007
:10653000a4638000a4608800854ca8002a8ca80071
:106540002a6ca800a563800094638000848f5200a9
:106550001d003a002564800004802000048262004f
:10656000e00f52000b003a00988f0200000000007c
:106570000003be0084962800950020000602420019
:1065800087824a00d4638800e5638800848ca90070
:106590000d00370066608000776080004e0290003a
:1065a000de029000840f5300858f5b0006003a00e6
:1065b0005461800061026200e00f5200020032006c
:1065c000848ca900856ca9007e0a90007403900059
:1065d000ce03900064608000756080000402780043
:1065e0000482530004024300640f9800d4608000ca
:1065f000e00f520004003a006e0a9000e00f5200d3
:1066000001003200852ca8006e0a9000d46088003a
:1066100014648000e80f520018003a0066608000a1
:10662000776080004e029000de029000840f5300dd
:10663000858f5b003b003a0054618000610262007c
:10664000e00f520039003200988f02000000000075
:106650000003be00444b2c0045002000060242000f
:1066600087824a00d4638800e5638800848ca80090
:106670009400200014648800310037001464800006
:10668000e90f52000e003a000e5290000482fb0007
:1066900061026200e00f520026003a004e039000b3
:1066a000de03900066608800776088008040eb0021
:1066b00040c1b30083f90700cefc0700d7013700c3
:1066c00014648000ea0f52001c003a0066608000eb
:1066d000776080004e029000de029000840f53002d
:1066e000858f5b00c2013a00c2fc0700cb01370076
:1066f000646080007560800061034200e0834a00ae
:106700004e029000de029000840f5300858f5b00e4
:10671000b9013a00b7fc0700c001370000000000d3
:1067200007003700000000000500370000000000ef
:1067300003003700000000000100370000000000e7
:106740000e5290008482fb0004022000048262004a
:10675000e00f5200aa013a0014648000eb0f5200cf
:10676000a901320014648000ea0f5200a80132002f
:1067700014648000ec0f5200a70132000e1290004a
:10678000e00f5200220132005e0a9000e00f52003a
:1067900080003c007e0a9000640290004422de00eb
:1067a0006f4262000482fb004222dd008402780016
:1067b0005e0a90000482520004007800728b02008e
:1067c000000000008e1290005e0a900004824200d9
:1067d000041798008e1290003e029000848f5200a1
:1067e00002003600be039000071798008660800004
:1067f000976080000e129000050020000602420003
:1068000087824a008460880095608800b5638000b4
:106810000e1290008482420084638000848f5200b4
:106820002000360085638000b4638000048252003b
:106830000402e8002407980085c8200095427800eb
:10684000b66380002e0290008041eb000081eb00d7
:106850008540780006007800270207008e1290001d
:106860002e0290000482520085c8200095427800d4
:10687000766380008041eb000081eb00854078006a
:10688000060078001c020700756380000e1390005c
:106890002e0290000402530004824200b463880078
:1068a0000d00370085c8200095427800b66380004f
:1068b0000e1290008041eb000081eb0085407800d3
:1068c000060078000c020700b56380000e129000ed
:1068d00004824200b463880044618000e10f4200fa
:1068e000cb00320044618000840278000e129000d8
:1068f0000482520044618800e560800044618000a9
:1069000004824200240798002e029000e00f5200fb
:1069100003003d000082eb0044618800bc003700aa
:1069200044618000e00f5200b9003c0086608000a6
:10693000976080002e0290000500200006024200b1
:1069400087824a008460880095608800b563800073
:106950002e02900004824200b4638800b563800078
:1069600084638000848f520007003600b563800086
:106970008663800074638000040253000482ea008e
:1069800004824200b46388000082eb004461880006
:106990009f0037005e0a9000e00f52009c00340018
:1069a0008e1290005e0a9000848242003e029000a7
:1069b000848f520004003600be0290005e0a9000f0
:1069c00004825200041798007e0a9000640290002e
:1069d0004422de006f4262000482fb004222dd009e
:1069e00004007800728b020000000000b563800094
:1069f0005e0a9000848242000e129000848242005f
:106a000084638000848f52003300360085638000e9
:106a1000b4638000848252005e0a90000402ea009f
:106a2000048242000402e800240798002e0290002d
:106a3000e00f52001700350085c82000954278000d
:106a4000b66380005e0a9000040343002e029000ab
:106a50008041eb000081eb00854078000600780063
:106a6000a50107008e1290002e02900004825200b1
:106a700085c8200095427800766380008041eb0055
:106a80000081eb0085407800060078009a0107003d
:106a90001c00370085c8200095427800b66380004e
:106aa0005e0a9000040343008763800074638000e3
:106ab000048253000482ea00040343000e12900093
:106ac0008041eb000081eb008540780006007800f3
:106ad000890107000b00370085c820009542780027
:106ae000b66380005e0a9000040343000e1290001b
:106af0008041eb000081eb008540780006007800c3
:106b00007d01070044618000e10f420005003a006a
:106b10005e0a9000446188000e129000e4608800d4
:106b20003b00370044618000840278005e0a9000d8
:106b3000848f52001c003600de0a90000e12900076
:106b4000848242004461800004037800e460800095
:106b500004024300848f520006003e00de0a9000cb
:106b60000e1290008482420044618000848f5200a3
:106b7000030031008e129000e560880007003700a6
:106b80004461800084027800e460800084824200d6
:106b90005e0a900004825200e46088005e0a900061
:106ba000446188001a003700de0a90000e1290003f
:106bb000848242004461800004037800e460800025
:106bc00004024300848f52001100360044618000ab
:106bd00084027800e4608000848242005e0a9000b3
:106be000848f52000a003900e56080005e0b90003f
:106bf0000e1290000403430044618000040353001c
:106c0000e46080000402530004824200e4608800d3
:106c10006e029000e00f52001c00320014648000ed
:106c2000e70f520002003200b4638000c4638800a2
:106c3000256480000408200004826200e00f5200f6
:106c40000500320011c0b30000c1b3001df80700f9
:106c5000a3ef07000d00370084eca8002564800036
:106c60000404200004826200e00f520007003a0092
:106c700084cca800a68f0200000000000002be0025
:106c80000402780078024200046488000e529000ea
:106c90000482fb006102620004427800e04f52006f
:106ca0005e003200846080009560800061034200d5
:106cb000e0834a006e0290006120b8001e0a900036
:106cc000ae0a90000002420081824a00840f530005
:106cd000858f5b0051003a008460800095608000e1
:106ce00061024200e0824a0084608800956088006a
:106cf000146480006123b800a4ff2f00f5ff2f006b
:106d00000602420087824a00360020000700200069
:106d1000860f5200878f5a0028003e000460010051
:106d20000300370008003700100037001e0037004e
:106d3000c40020001464880011c0b30010c1b30067
:106d4000e0f7070035003700b40020001464880025
:106d5000a68f0200000000000002be0004027800be
:106d60000403b000046488001500370066608000ea
:106d7000776080004e029000de029000840f530086
:106d8000858f5b0005003a008040eb0000c1b30036
:106d9000ccf7070017fb070020003700a4002000f5
:106da00014648800060037008040eb0000c1b30087
:106db000c4f707000ffb07001800370000000000b1
:106dc00011c0b30000c1b300bef7070013003700c5
:106dd0000000000011003700000000000f00370025
:106de000000000000d003700000000000b0037001d
:106df0000000000009003700000000000700370015
:106e0000000000000500370000000000030037000c
:106e10000000000001003700000000000080fa00c0
:106e2000000006000e00fa00604798004107980035
:106e300052079800434f98006e429000e14f520075
:106e4000020036000002eb00a80037006e40900000
:106e5000f7ee07004e029000e00f520002003a00e9
:106e6000140020004407980085638000646380005c
:106e7000048252000402e90024079800ce02900028
:106e80005e029000848242002e029000848f5200a5
:106e9000020036000002eb009400370010ef0700fc
:106ea0004e4a90000482fb0063026200e00f520031
:106eb00003003a004e4a90003440b300444f98001b
:106ec0005e02900014079800ce0290005e029000cf
:106ed00004824200ae02900004825200240798000f
:106ee0004e4a90000482fb0062026200e00f5200f2
:106ef000100032004e4a90000482fb0061026200e2
:106f000004427800e04f5200060032002e0290004a
:106f10000402d1009e0290000482420014079800ef
:106f2000040037009e0290002e029000048242006e
:106f300014079800656380001e02900004824200de
:106f40000402e80024079800b4638000040f78006e
:106f500044618000e10f42000d0032004461800076
:106f600084027800e4608000048242001e0f420028
:106f7000846380009e0f520005003100856380000d
:106f800074638000048252000482ea001e0f4200f3
:106f9000c46380009e0f520010003100c563800062
:106fa0002e029000848f5200230031004e4a900040
:106fb0000482fb0064026200e00f52000200320013
:106fc0000002eb00490037002e029000c4638800e5
:106fd0002e029000b463880017003700c46380005d
:106fe0009e0f520010003600756380002e02900044
:106ff000848f5200100031004e4a90000482fb0042
:1070000064026200e00f5200020032000002eb0056
:10701000360037002e029000c46388002e029000d4
:10702000b4638800040037002e029000c463880017
:107030002e029000b4638800c46380009e0f52004b
:107040001b0036004e4a90000482fb00640262007e
:10705000e00f520016003200746380001e0212001e
:1070600086c82000164378007763800085c820001a
:1070700095427800864178000701780085407800c5
:107080002e0090001c000700b5638000c4638000e0
:10709000848f520006003100b56380007463800065
:1070a0002e0390000402530004824200b46388005f
:1070b0002e0290007463880064638000a4608800de
:1070c00064638000a4638800646380009463880024
:1070d00014648000e70f520003003a0011c0b300af
:1070e00000c1b300f7f60700140020000400780088
:1070f0000080fa00000006000a00fa00000f780085
:107100002147980022079800634798004407980099
:107110006e4290000482fb00e00f52001d0032001e
:10712000e10f52003e003a002e4290000482fb0024
:10713000e00f52000a003200e10f520035003a0021
:10714000ae0290001e0278004e019000850078008b
:1071500004007800a20b0200000000000c003700c1
:107160001e027800e10f4200030032001e0078008a
:10717000083d0200000000002e029000ce009000aa
:1071800004007800443f02000000000000000000fe
:10719000230037002e4290000482fb00e00f5200d3
:1071a0000e003200e10f52001c003a002e02900047
:1071b000e10f4200030032002e009000223d020049
:1071c000000000001e027800ce009000040078004d
:1071d000fa3e0200000000000c0037004e01900053
:1071e000ae0090001e0078002c3e0200000000005f
:1071f00000000000b23e0200000000000002780023
:10720000e00f5200fbff3200000000000000000011
:1072100003003700000000000100370000000000fc
:107220000080fa00000006000200fa00d922a8003f
:10723000c662a900ca62a900d7c2a800d3c2a90029
:107240000042eb0004407800d2edb7000002eb00f2
:1072500004128800b4132000141288000002eb000e
:107260002412880004002800041288007c03070010
:10727000e4e92000b46e88000002eb00a46e8800f0
:10728000d80da800d82da900d84da9008000eb008a
:107290000000eb00ab050700e1e920004000200002
:1072a000a8050700e1ff250060002000a5050700f4
:1072b0000100260060012000a20507001100260041
:1072c000800120009f050700b4d020001442780000
:1072d000e04f520015003a00c4d02000144278005c
:1072e000e44f520011003a00d5d0200095427800ba
:1072f00034cab30084cf52000c003a00e4d020001e
:1073000014427800e04f520008003a00f4d0200008
:1073100014427800e04f520004003a0004d12000eb
:1073200014427800e04f520013003200b5d0200024
:1073300095427800c4d020001442780084c27200c4
:10734000d4d020001442780084c27200e4d020001f
:107350001442780084c27200f4d0200014427800f5
:1073600084c2720004d120001442780004c272006a
:10737000e04f520028003a00400620002605070092
:1073800000027800040f78000e02780014427800a2
:10739000044078000bedb7000e0278000402e8000c
:1073a00014427800044078000cedb700200620005d
:1073b0001905070000027800040f78000e0278001b
:1073c00014427800044078000dedb7000e027800fa
:1073d0000402e80014427800044078000eedb70083
:1073e000000620000c05070000027800040f78005a
:1073f0000e02780014427800044078000fedb700c8
:107400000e0278000402e80014427800044078007c
:1074100010edb700270037008e027800b4d02000ae
:1074200014427800844a78000e0278008402e80052
:10743000c4d0200014427800844a78001e027800ec
:1074400084007800400620003e0507008e02780088
:10745000d4d0200014427800844a78000e027800cc
:107460008402e800e4d0200014427800844a7800c6
:107470001e027800840078002006200031050700f5
:107480008e027800f4d0200014427800844a7800fc
:107490000e0278008402e80004d120001442780033
:1074a000844a78001e0278008400780000062000dc
:1074b00024050700115e200040c0b300f00507005e
:1074c00011002000e00120006a0507000080fa009a
:1074d000000006000000fa00a0012000ce04070012
:1074e00000027800051020000502620004f0a700e9
:1074f0000402ea000402ea004f22de0004007800e1
:107500000080fa00000006000000fa00e001200000
:10751000c1040700000278006202620004f0a700c4
:107520000402ea000402e9004f22de0004007800b1
:107530000080fa00000006000200fa0084dd20004e
:107540001442780061426200e04f520010003a009d
:10755000d80da800b46e8000048fe900b56e8000dd
:10756000e4e92000848f520002003a00e4ff250085
:10757000040f780001102000e00120003d05070005
:107580009e00780060002000ee0407000100370034
:10759000000000000080fa00000006000200fa006f
:1075a000800020009c04070000027800040f78008f
:1075b000a46e80009e027800848f52000500360081
:1075c000a46e80009e025200141625000482420020
:1075d00003003700a46e80001e0252000482e900fe
:1075e000040078000080fa00000006001a00fa008b
:1075f000881f7800300f9800410f9800c0012000cc
:1076000085040700000278000504200005026200de
:10761000e00f520042003a00d86e8000a68f0200b0
:10762000000000000002be00040278008402540042
:10763000841e2000848f520037003600a5ff07000b
:1076400000027800e00f520007003200a68f02000f
:10765000000000000002be0004027800d413b00055
:10766000d46e88002c003700541680004322de00c0
:10767000614262000404a200614262000482fb00d5
:10768000610262004322dd005616800075ff2f0064
:10769000850263000482720054168800a68f0200df
:1076a000000000000002be0004047800986c020094
:1076b00000000000000278000400780001002000b3
:1076c00002002000030020006408200005002000c4
:1076d0006033b800e0080200000000000203be00b2
:1076e0000002be000400be000601be00f4ff2f0031
:1076f000050020006033b800260a020000000000e8
:107700000203be000002be0004027800040244002e
:10771000440fb000d46e88000002eb005500370023
:1077200084dd20001442780061426200e04f520084
:107730000a003a0080ff0700c0012000360407005d
:10774000000278000504200005026200e00f5200ec
:1077500002003a000002eb0046003700b46e8000e1
:10776000a46e8800a46e800084007800a008200029
:10777000740407000e027800620120008400780083
:1077800040c0b300980207002e0a90000400780061
:10779000527102000000000000027800240f9800df
:1077a0009e027800f4ff2500848f520015003e00f1
:1077b0000e0278001442780061426200e04f5200ed
:1077c00010003a007e429000e04f52000d003a0057
:1077d000be0290000408200004826200e00f520004
:1077e00008003a002e02900070026200e00f520082
:1077f00004003a009e029000245f2000848f520013
:1078000002003600000000000000fe001e027800aa
:10781000b46e88003e0a9000ee024700620020002d
:107820008500780004007800a20b02000000000030
:10783000ce0a900000c2eb00844a78005e529000ad
:10784000e84f520009003a004e529000e04f5200bb
:10785000030032004e529000e64f520003003a00ff
:107860004e529000ce0a9000844a7800d80da900ac
:1078700014002000040078004f0478000080fa0013
:10788000000006000800fa00100798004147980021
:10789000320798004e429000e04f520002003a003a
:1078a000840020000100370084602000040f78006d
:1078b0008000eb0080082000220407003e029000b8
:1078c0006e02420084007800200020001d040700a2
:1078d0001e029000620020008400780020c0b300e7
:1078e0001602070062002000b1d0200020c0b300c3
:1078f000120207000e0278002200200084007800a7
:1079000020c0b3000d0207000080fa00000006004e
:107910000200fa00c0012000bf0307000002780047
:107920000580200005026200e00f52001b003200bb
:1079300001802000c00120008004070020042000f6
:10794000b503070000027800040f7800a0012000b2
:10795000b103070000027800054020000502620024
:10796000e00f5200050032005101200040042000c9
:10797000f40307001e00a0000500370021012000cd
:1079800040042000ef030700e4ff2f001e0f6200f9
:107990009e00780020042000ea030700a0012000d8
:1079a0009d03070000027800051020000502620018
:1079b000e00f52000300320021002000e00120000f
:1079c0002c0407000080fa00000006000400fa0002
:1079d00010079800a56e80001e02900004824200ed
:1079e000760f4200f4ff25009e027800848f52003b
:1079f00002003600e4e92a001e0f42009e007800d3
:107a0000a0082000cf0307000080fa000000060055
:107a10000400fa0010079800800820007e03070089
:107a200000027800040f78009e009000800820007b
:107a3000c40307001e027800040078000080fa00ea
:107a4000000006000400fa0010079800a0082000bb
:107a50007103070000027800040f78009e00900078
:107a6000a0082000b70307001e0278000400780079
:107a70000080fa00000006000600fa0010079800d7
:107a800021079800a56e80001e029000048242002b
:107a9000760f4200f4ff25009e027800848f52008a
:107aa00002003600e4e92a001e0f420084dd2000b7
:107ab0001442780062426200e04f5200040032003b
:107ac00001002800e0062000ea030700010037005b
:107ad00000000000e00120004f03070000027800d2
:107ae0000502200005026200e00f5200f9ff3a0093
:107af0009e007800a000200092030700ae009000d6
:107b0000c00020008f030700c1012000e001200019
:107b10000a04070001022000e0012000d50307004d
:107b200000000000e00120003b0307000002780095
:107b30000502200005026200e00f5200f9ff3a0042
:107b400084dd20001442780062426200e04f52005f
:107b50000300320001002800e0062000f7030700c0
:107b6000000120002c0307000002780004007800c8
:107b70000080fa00000006000200fa00000f780002
:107b800084dd20001442780062426200e04f52001f
:107b90000400320001002800e0062000b5030700c1
:107ba0000100370000000000e00120001a03070078
:107bb000000278000502200005026200e00f52007a
:107bc000f9ff3a00a0082000130307000002780024
:107bd00084007800a00020005a0307009e0078006f
:107be000c000200057030700c1012000e001200071
:107bf000d203070001022000e00120009d030700de
:107c000000000000e00120000303070000027800ec
:107c10000502200005026200e00f5200f9ff3a0061
:107c200084dd20001442780062426200e04f52007e
:107c30000300320001002800e0062000bf03070017
:107c400000012000f4020700000278000400780020
:107c50000080fa00000006000800fa0010079800f3
:107c600021079800320798001e029000e10f4200a1
:107c70000a003a0080082000e702070000027800ae
:107c8000140798009e0290003e0290000482420079
:107c900084007800800820002a0307002e0290004c
:107ca000e10f420010003a00a0082000da020700ad
:107cb0000002780024079800ae0290003e02900077
:107cc000048f4200f4ff25009e027800848f52004a
:107cd00002003600e4e92a001e0f42009e007800f0
:107ce000a00820001703070084dd2000144278005c
:107cf00062426200e04f520004003200010028009e
:107d0000e00620005b0307000100370000000000d0
:107d1000e0012000c00207000002780005022000f8
:107d200005026200e00f5200f9ff3a00ae00900039
:107d3000a0002000030307009e009000e000200048
:107d400000030700be009000c0002000fd020700f5
:107d500001032000e0012000460307000080fa0034
:107d6000000006000200fa00e0012000aa0207005d
:107d700000027800050220000502620004f0a7005e
:107d80000402ea00040fe9001e0278004f22de0020
:107d9000040f78001e027800e00f52000800320045
:107da00084dd20001442780062426200e04f5200fd
:107db0000300320001002800e00620005f030700f6
:107dc0001e027800040078000080fa00000006001f
:107dd0000200fa00120020008e00780040c0b300bc
:107de000010107001e427800044078000080fa007c
:107df000000006000600fa0010079800210798000e
:107e00001e029000e00f5200050032002e0190008b
:107e10009e00900040c0b300f30007000e00370042
:107e2000a00820007c02070000027800ae0290004b
:107e3000050f4200f4ff25009e027800848f520057
:107e400002003600e4e92a001e0f42009e0078007e
:107e5000a0082000bb0207002e029000040078005a
:107e60000080fa00000006000200fa00004f7800cf
:107e7000120020008e00780020c0b300af00070081
:107e80000080fa00000006000400fa00000f7800ed
:107e9000110798001e0190009e00780020c0b300da
:107ea000a60007000080fa00000006000000fa00ab
:107eb00011002000e0012000200307000000000066
:107ec000a0012000540207000002780005002200f3
:107ed00005026200e00f5200f9ff3a0000000000c6
:107ee000e00120004c0207000002780025822800f3
:107ef00005026200e00f5200f9ff3a00d82da800f9
:107f0000d84da900c00120004302070000027800fc
:107f1000e00f520001003d007003070001802000c7
:107f20000040eb005603070001002c00e006200093
:107f3000020307000080fa00000006000000fa00bb
:107f40000100220010c1b3004d0307000080fa00b9
:107f5000000006000000fa00d82da90001002c0046
:107f6000e0062000c30207000040eb0025030700e5
:107f7000000278000580200005026200e00f520038
:107f800003003200010021000040eb003c03070029
:107f90008000eb0010c1b3003903070000000000af
:107fa000a00120001c02070000027800052021002b
:107fb00005026200e00f5200f9ff320011002000bc
:107fc000e0012000ab0207000080fa00000006007c
:107fd0000400fa0020479800e00620000e02070087
:107fe00000027800f50f2f0005026200040f7800f0
:107ff0000e0278000403e8000e0278000402e80094
:1080000014427800844278002e4290006f42620051
:1080100004c27200044b78001e02780084007800cd
:10802000e0062000470207000080fa00000006007a
:108030000200fa00e0062000f701070000027800c5
:10804000040f78000e0278000402e8001442780061
:108050006f426200044078000080fa0000000600d1
:108060000000fa00d7e2a900d3e2a9002000200016
:108070008c91020000000000db22a800d922a90098
:10808000d7e2a8000042eb0004407800d2edb70030
:108090008002200001002000c891020000000000c2
:1080a000d922a800412321006001200025020700f9
:1080b00060012000d801070000027800452321005c
:1080c000850f5200f7ff3a0001012000e006200072
:1080d000680207000042eb0004407800d2edb700d0
:1080e00000000000a0012000cb0107000002780082
:1080f00005a021008502620004a02100848f5200a7
:10810000f8ff3a003000200001002000c891020072
:108110000000000060012000bf010700000278009d
:10812000e00f5200dfff3a00100020008c910200a7
:10813000000000000080fa00000006000a00fa00bb
:10814000404798003107980042079800b404800027
:108150004d22de00614262000482fb001407980099
:1081600097a0a90024c3b300044f78004e429000aa
:108170000482fb0062026200e00f52000200320043
:10818000a4c2b300044f78004e4290000482fb006a
:1081900064026200e00f520002003200e4c2b30049
:1081a000044f78004e019000be0090001e40780001
:1081b000540107001e0290000442780061426200f0
:1081c0000482fb00610262004d22dd00b6048000e3
:1081d000f5ff2d008502630004827200b40488005c
:1081e0000080fa00000006000a00fa0040479800ec
:1081f00031079800420798004e029000e00f5200ad
:1082000026003200b40480004d22de00614262008c
:108210000482fb001407980097a0a90004c3b300d0
:10822000044f78004e4290000482fb00620262001c
:10823000e00f52000200320084c2b300044f780005
:108240004e4290000482fb0064026200e00f520084
:1082500002003200c4c2b300044f78004e01900007
:10826000be0090001e407800e20007001e02900051
:1082700004427800614262000482fb0061026200f5
:108280004d22dd00b6048000f5ff2d00850263005d
:1082900004827200b404880001003700000000006e
:1082a0000080fa00000006000600fa00404798002f
:1082b000b40480004d22de00614262000482fb00b3
:1082c000040f780097a0a900d7c2a9004e429000e1
:1082d0000482fb00441288000412800062026200e3
:1082e000e00f5200fcff3a000412800061026200bd
:1082f000e00f5200f8ff3200441280000442780080
:1083000024479800d7c2a8001e02780004427800d3
:10831000614262000482fb00610262004d22dd00c6
:10832000b6048000f5ff2d00850263000482720010
:10833000b40488000080fa00000006000800fa007b
:108340004047980031079800b40480004d22de00b9
:10835000614262000482fb00040f780097a0a9002c
:10836000d7c2a9004e4290000482fb00441288004c
:108370000412800062026200e00f5200fcff3a002b
:108380000412800061026200e00f5200f8ff320028
:108390008e82e8004412800004427800844a78000b
:1083a00066024700144278000482fb0044128800f1
:1083b0000412800062026200e00f5200fcff3a00eb
:1083c0000412800061026200e00f5200f8ff3200e8
:1083d0008e82e8004412800004427800844a7800cb
:1083e000660247000402e800144278000482fb00a1
:1083f000441288000412800062026200e00f520002
:10840000fcff3a000412800061026200e00f52009b
:10841000f8ff32000e82e8008402e8004412800077
:1084200004427800844a7800d7c2a8001e0278006f
:1084300004427800614262000482fb006102620033
:108440004d22dd00b6048000f5ff2d00850263009b
:1084500004827200b40488001e02900004007800b8
:108460000080fa00000006000c00fa006047980047
:108470004207980053079800b40480004d22de00a4
:10848000614262000482fb00040f780097a0a900fb
:10849000d7c2a9006e4290000482fb0044128800fb
:1084a0000e82e800e30242000042eb00844a7800ba
:1084b0000412800062026200e00f5200fcff3a00ea
:1084c0000412800061026200e00f5200f8ff3200e7
:1084d0008e82e8004412800004427800844a7800ca
:1084e00068024700144278000482fb0044128800ae
:1084f0000412800062026200e00f5200fcff3a00aa
:108500000412800061026200e00f5200f8ff3200a6
:108510008e82e8004412800004427800844a780089
:10852000680247000402e800144278000482fb005d
:10853000441288000412800062026200e00f5200c0
:10854000fcff3a000412800061026200e00f52005a
:10855000f8ff32000e82e8008402e8004412800036
:1085600004427800844a7800680247000482e800e8
:10857000144278000482fb00441288000412800038
:1085800062026200e00f5200fcff3a000412800019
:1085900061026200e00f5200f8ff32000e82e80034
:1085a0008482e8004412800004427800844a780003
:1085b000d7c2a8001e02780004427800614262001f
:1085c0000482fb00610262004d22dd00b6048000df
:1085d000f5ff2d008502630004827200b404880058
:1085e0001e029000ae0290000400be000080fa005f
:1085f000000006000a00fa00404798003107980082
:1086000042079800b40480004d22de0061426200ff
:108610000482fb00040f780097a0a900d7c2a9002c
:108620004e4290000482fb00441288000412800035
:1086300062026200e00f5200fcff3a000412800068
:1086400061026200e00f5200f8ff32004412800025
:108650000442780024479800110037000002eb0024
:10866000441288000412800062026200e00f52008f
:10867000fcff3a000412800061026200e00f520029
:10868000f8ff32004412800004427800be029000dd
:10869000844a78003e0290000402e8003407980003
:1086a0004e02900004f0a7000402ea000402ea006f
:1086b0004f22de0004427800ce0290008502e900dd
:1086c00045079800e04f5200e4ff3a00d7c2a800e7
:1086d0001e02780004427800614262000482fb00be
:1086e000610262004d22dd00b6048000f5ff2d001e
:1086f0008502630004827200b40488000080fa00de
:10870000000006000a00fa00404798003107980070
:1087100042079800b40480004d22de0061426200ee
:108720000482fb00040f780097a0a900d7c2a9001b
:108730004e4290000482fb00441288000412800024
:1087400062026200e00f5200fcff3a000412800057
:1087500061026200e00f5200f8ff32004412800014
:108760000442780024479800120037003e0290002f
:10877000144278000482fb00441288003e029000fc
:108780000402e800340798000412800062026200cc
:10879000e00f5200fcff3a00041280006102620008
:1087a000e00f5200f8ff32004412800004427800cb
:1087b000244798004e02900004f0a7000402ea004b
:1087c0000402ea004f22de0004427800ce0290004c
:1087d0008502e90045079800e04f5200e3ff3a00a8
:1087e000d7c2a8001e0278000442780061426200ed
:1087f0000482fb00610262004d22dd00b6048000ad
:10880000f5ff2d008502630004827200b404880025
:108810000080fa00000006000a00fa0040079800f5
:108820004e0290008442780004ceb30004cf620070
:1088300004c6b3009e42780084cf52002a003e0056
:1088400024dd2000144278009e42780084cf52003c
:108850001c0032001e427800e04f520003003a0034
:1088600000ccb30090fe07001400370004c2b30030
:108870009e42780084cf520003003a0020ccb3001f
:1088800089fe07000d00370004c4b3009e42780043
:1088900084cf520003003a0040ccb30082fe0700b0
:1088a0000600370004c6b3009e42780084cf520011
:1088b00002003a0060ccb3007bfe07001e40780047
:1088c000d2edb7004e029000044278007f42620071
:1088d0008000eb000440780098fe0700000278005a
:1088e00014079800130037004e0290000500200086
:1088f0000401be0000c2b300dbfe07000002be00a0
:1089000024079800350798008e82e800640247002b
:108910000402e80014427800844a78000e82e800dd
:108920008402e800640247000482e80014427800f0
:10893000844a78001e029000040078000080fa004b
:10894000000006000a00fa0030079800410798006e
:108950003e0290008442780004ceb30004cf62004f
:1089600004c6b3009e42780084cf52002b003e0024
:1089700024dd2000144278009e42780084cf52000b
:108980001c0032001e427800e04f520003003a0003
:1089900000ccb30044fe07001400370004c2b3004b
:1089a0009e42780084cf520003003a0020ccb300ee
:1089b0003dfe07000d00370004c4b3009e4278005e
:1089c00084cf520003003a0040ccb30036fe0700cb
:1089d0000600370004c6b3009e42780084cf5200e0
:1089e00002003a0060ccb3002ffe07001e40780062
:1089f000d2edb7004e0390003e0290000442780092
:108a0000ff42620004c4b30004c272008600780012
:108a10000440780049fe0700140037008e82e80009
:108a20003e02900004427800844a78000e82e800fa
:108a30008402e8006802470014427800844a780003
:108a40000e82e8008482e800680247000402e80021
:108a500014427800844a78001e029000ae02900012
:108a60000401be0020c2b3007ffe07000080fa00b0
:108a7000000006000600fa00100798002107980081
:108a80001e0290008442780004ceb30004cf62003e
:108a900024dd2000144278009e42780084cf5200ea
:108aa0001c0032001e427800e04f520003003a00e2
:108ab00000ccb300fcfd07001400370004c2b30073
:108ac0009e42780084cf520003003a0020ccb300cd
:108ad000f5fd07000d00370004c4b3009e42780086
:108ae00084cf520003003a0040ccb300eefd0700f3
:108af0000600370004c6b3009e42780084cf5200bf
:108b000002003a0060ccb300e7fd07001e40780089
:108b1000d2edb7001e02900004427800ff426200ce
:108b200004c8b30004c27200ae0090000440780094
:108b300002fe07000080fa00000006000600fa00ae
:108b400010079800210798001e02900084427800c8
:108b500004ceb30004cf620024dd2000144278006c
:108b60009e42780084cf52001c0032001e427800e2
:108b7000e04f520003003a0000ccb300cafd0700ea
:108b80001400370004c2b3009e42780084cf520024
:108b900003003a0020ccb300c3fd07000d003700ee
:108ba00004c4b3009e42780084cf520003003a0010
:108bb00040ccb300bcfd07000600370004c6b3007c
:108bc0009e42780084cf520002003a0060ccb3008d
:108bd000b5fd07001e407800d2edb7001e029000e0
:108be00004427800ff42620004cab30004c272006b
:108bf000ae00900004407800d0fd07000080fa002d
:108c0000000006000400fa00204798002e42900061
:108c10008482fb000410200004827200840078002b
:108c20004005200047ff070011002000200520001c
:108c300044ff070000000000a0062000f6fe070029
:108c4000000278006102620004427800e04f5200a6
:108c5000f9ff3a008000eb002005200039ff0700f3
:108c600080062000ecfe070000027800040f780068
:108c70001e027800040078000080fa000000060060
:108c80000400fa00004f7800110798001e42780097
:108c90008482fb00041020000482720084007800ab
:108ca0004005200027ff07009e009000600620007e
:108cb00024ff070000000000a0062000d6fe0700e9
:108cc000000278006102620004427800e04f520026
:108cd000f9ff3a000080fa00000006000600fa00e2
:108ce00020072000ccfe070000027800040f780067
:108cf0001e027800e00f520003003d000100280032
:108d0000200720008dff0700a0012000c2fe070001
:108d10000002780014079800640247001200200047
:108d200084007800d0c1b30032fe0700ce4290002c
:108d300004c8b30004c26a004447980064024700b4
:108d40001200200084007800d0c5b3006dfe07003b
:108d5000a0012000b0fe0700000278009e029000f3
:108d600085026a000410200004826200e00f5200b5
:108d70000300320001802000c00120003dff0700f9
:108d80001e027800e00f520003003d0001002800a1
:108d90002007200037ff07000080fa0000000600cf
:108da0000400fa0020479800f46f8000e00f5200a2
:108db0000c003a0014002000f46f88000042eb0021
:108dc000044f78000400370000c2eb000440780034
:108dd00024edb7001e4fe8001e427800e04f52001d
:108de000f9ff320044d2200014427800e14f4200e3
:108df0000800320044d22000144278000440780079
:108e0000305f02000000000000c2eb000440780068
:108e100024edb70014002000346988000042eb0004
:108e20000440780028edb700288da800282da80060
:108e30000080fa00000006000200fa00004f7800ef
:108e400044d2200014427800e14f42000800320072
:108e500044d220001442780004407800305f0200c1
:108e60000000000000c2eb000440780024edb700d1
:108e70000002eb00346988000080fa000000060060
:108e80000200fa00004f780034698000e00f5200c1
:108e900003003a001400200034698800280da9005e
:108ea0000080fa00000006000200fa00004f78007f
:108eb0003469800004f0a7000402ea000402ea001a
:108ec0004f22de00040078000080fa000000060057
:108ed0000200fa00004f780044698000614262009d
:108ee0000482fb00040078000080fa000000060005
:108ef0000200fa00004f78004469800062026200bc
:108f0000e00f520003003200282da90014002000b9
:108f1000010037000002eb00040078000080fa0036
:108f2000000006000200fa00004f7800446980004b
:108f30004322de00614262000482fb0004007800ec
:108f40000080fa00000006000000fa00b569800009
:108f5000f40f200084826200e4cd200014427800e7
:108f6000604262000542720004407800deecb70007
:108f7000b4698000c822de00f4cd200014427800dd
:108f8000604262000542720004407800dfecb700e6
:108f9000c5698000f40f20008482620004ce2000a6
:108fa000144278006042620005427200044078007a
:108fb000e0ecb700c4698000c822de0014ce2000b7
:108fc000144278006042620005427200044078005a
:108fd000e1ecb7000080fa00000006000200fa0091
:108fe0000042eb00044f78003e02370034698000f5
:108ff00005002000c600200007002000860f520058
:10900000878f5a0036023e00046001001b023700c1
:109010000b0037001900370053003700710037008c
:109020009000370093013700c3013700d8013700a3
:10903000c1013700d6013700bf013700d401370026
:1090400034042000430420000041eb006000b8001d
:10905000985b0200000000000042780004407800a5
:1090600024edb70044d2200014427800e14f4200c2
:10907000040232002400200034698800c403200068
:109080000500200074698800856988000042eb00b3
:10909000044078004aedb700280da900284da9002a
:1090a0006a3a02000000000000027800e00f52005f
:1090b000f601320044d220001442780004407800c7
:1090c0009e5f02000000000000027800b512200040
:1090d000850f5200ef013600446980004422de0013
:1090e000614262000404a200614262000482fb004b
:1090f000610262004422dd0046698000f5fe2f0017
:1091000085026300048272004469880044d2200012
:10911000144278000482fb007822b90084027800af
:1091200004b0200004824200a2002000f10f2000c1
:1091300004007800b00b0200000000008000eb008b
:1091400010c0b3006b030700988f020000000000fe
:109150000002be0054698800656988003400200060
:1091600034698800de01370044d2200014427800c0
:1091700004407800586102000000000000027800fe
:10918000950f2000850f52000f003e00988f0200bf
:10919000000000000003be00546980006569800083
:1091a0000403530085835b0074842e0015002000a7
:1091b000840f5300858f5b00b80136002400200027
:1091c00034698800c6013700286da800ca0107006d
:1091d00000427800e24f5200b2013a004400200001
:1091e0003469880044d2200014427800044078009a
:1091f0009e5f0200000000000002780015102000b1
:10920000850f5200a901360044d220001442780094
:109210000482fb007822b9008402780004b02000a8
:1092200004824200a2002000f10f20000400780018
:10923000b00b0200000000008000eb0030c0b30063
:109240002c030700988f0200000000000002be00ff
:1092500054698800656988005400200034698800da
:109260009f01370044d22000144278000440780067
:10927000586102000000000000027800950f2000f5
:10928000850f52000f003e00988f02000000000082
:109290000003be0054698000656980000403530028
:1092a00085835b0074842e0015002000840f53001a
:1092b000858f5b007f013600240020003469880020
:1092c000870137008c010700004278000482fb0010
:1092d000e50f520003003200e60f5200e1003200b9
:1092e0007f01370044d22000144278000440780007
:1092f000305f02000000000000c2eb000440780074
:1093000024edb700988f0200000000000002be00ac
:109310005469880065698800640020003469880009
:10932000282da800280da800546a80006102620060
:10933000e00f520022003200b5698000f40f2000d7
:1093400084826200e4cd2000144278006042620012
:109350000542720004407800deecb700b46980007a
:10936000c822de00f4cd2000144278006042620082
:109370000542720004407800dfecb700c569800048
:10938000f40f20008482620004ce20001442780092
:10939000604262000542720004407800e0ecb700d1
:1093a000c4698000c822de0014ce20001442780078
:1093b000604262000542720004407800e1ecb700b0
:1093c000546a800064026200e00f52002200320002
:1093d000f5698000f40f20008482620024ce200012
:1093e0001442780060426200054272000440780036
:1093f000e2ecb700f4698000c822de0034ce200021
:109400001442780060426200054272000440780015
:10941000e3ecb700056a8000f40f2000848262004c
:1094200044ce20001442780060426200054272007f
:1094300004407800e4ecb700046a8000c822de0033
:1094400054ce20001442780060426200054272004f
:1094500004407800e5ecb700546a800062026200c4
:10946000e00f520022003200d5698000f40f200086
:109470008482620064ce2000144278006042620060
:109480000542720004407800e6ecb700d469800021
:10949000c822de0074ce20001442780060426200d0
:1094a0000542720004407800e7ecb700e5698000ef
:1094b000f40f20008482620084ce200014427800e1
:1094c000604262000542720004407800e8ecb70098
:1094d000e4698000c822de0094ce200014427800a7
:1094e000604262000542720004407800e9ecb70077
:1094f000546a800068026200e00f520020003200cf
:10950000146a8000256a8000f60f2000860362003e
:10951000a6ce200016437800604363000743730023
:1095200006407800eaecb700c823de00b6ce200083
:1095300016437800604363000743730006407800d9
:10954000ebecb700f60f200086836200c6ce200049
:1095500016437800604363000743730006407800b9
:10956000ececb700c82ade00d4ce2000144278000c
:10957000604262000542720004407800edecb700e2
:10958000e4ce20001442780060426200044078007b
:10959000eeecb700f4ce2000144278006042620086
:1095a00004407800efecb70004cf200014427800ac
:1095b0006042620004407800f0ecb70014cf200055
:1095c000144278006042620004407800f1ecb70079
:1095d000546a800070026200e00f520020003200e6
:1095e000346a8000456a8000f60f2000860362001e
:1095f000e6ce200016437800604363000743730003
:1096000006407800eeecb700c823de00f6ce20005e
:1096100016437800604363000743730006407800f8
:10962000efecb700f60f20008683620006cf200023
:1096300016437800604363000743730006407800d8
:10964000f0ecb700c82ade0014cf200014427800e6
:10965000604262000542720004407800f1ecb700fd
:109660000300370024002000346988000000000057
:109670009b003700988f0200000000000003be002e
:1096800054698000656980000403530085835b0092
:1096900034422f0005002000840f5300858f5b00ab
:1096a00086003600766980008769800014002000fb
:1096b00005002000840f5300858f5b000f003600eb
:1096c000566980006769800044422f000500200031
:1096d0000602420087824a00546988006569880052
:1096e000746980008569800061025200e0825a003e
:1096f0007469880085698800790037003404200087
:10970000430420000041eb006000b800985b0200b9
:1097100000000000004278000440780024edb7000b
:1097200044d2200014427800e14f4200650032002c
:10973000740020003469880044d22000144278006c
:10974000044078009e5f02000000000000027800e4
:1097500015102000850f52005c003600110020001b
:1097600030c0b300e3010700284da900988f020024
:10977000000000000002be0054698800656988008e
:10978000346980000402e80034698800540037001e
:1097900044d220001442780004407800586102004e
:1097a0000000000000027800950f2000850f520095
:1097b00015003e00988f0200000000000003be006c
:1097c00054698000656980000403530085835b0051
:1097d00074842e0015002000840f5300858f5b00d9
:1097e0003c003600346980000402e80034698800d7
:1097f00034698000ec0f520038003600240020004d
:1098000034698800360037003b00070000427800ca
:109810000482fb00e50f520003003200e60f520005
:10982000120032002e00370044d22000144278008b
:1098300004407800305f02000000000000c2eb002e
:109840000440780024edb700988f0200000000006b
:109850000002be0054698800656988006400200029
:1098600034698800282da800030037002400200058
:109870003469880000000000190037000000000073
:10988000170037000000000015003700000000003e
:109890001300370000000000110037000000000036
:1098a0000f003700000000000d003700000000002e
:1098b0000b00370000000000090037000000000026
:1098c000070037000000000005003700000000001e
:1098d0000300370000000000010037000000000016
:1098e0001e4fe8001e427800e04f5200bffd3200dc
:1098f0000080fa00000006000c00fa000042eb00b5
:109900006447980064024700040078008861020000
:10991000000000004e429000e24f52004c013a001d
:10992000c0012000885f0200000000000042eb0040
:10993000044f78000f0037006402470004007800ed
:1099400088610200000000009e4078000182fb0058
:10995000c502200084824200f4cd2000048242002f
:10996000944278004e42900084cf52004e013a005b
:109970001e4fe8001e427800e54f5200eeff360011
:109980004469800064026200e00f520008003a005f
:1099900000012000885f020000000000410020005c
:1099a00060d32000bc610200000000004a0da80046
:1099b000000f2000885f0200000000000002eb00a2
:1099c00014079800640247000400780088610200d0
:1099d0000000000000027800e00f520003003a008f
:1099e0001400200014079800190137004e4290001f
:1099f0000482fb0035032000850f5200c4003200b2
:109a000035032000850f520007003c00e30f520091
:109a10003e003200e60f52006a003200e10f5200b1
:109a20001d003200f100370065032000850f520051
:109a300099003200f50f2000850f5200b10032006e
:109a400055032000850f5200e8003a0064024700e9
:109a50000400780088610200000000004e4290007f
:109a6000e14f520012013a006602470004007800fc
:109a70008861020000000000446980006402620006
:109a8000e00f5200ec0032006e429000e24f5200b4
:109a9000eb003a001101370064024700040078002f
:109aa00088610200000000004e429000e44f520026
:109ab00001013a004469800064026200e00f520034
:109ac0000c0032000042eb00044f78000500370024
:109ad0006402470004007800886102000000000072
:109ae0001e4fe8001e427800e34f5200f8ff360098
:109af000d400370041002000e0d32000bc61020008
:109b0000000000004a4da800ce0037006502470063
:109b10000400780088610200000000005e429000ae
:109b2000e34f5200e60036004469800064026200a0
:109b3000e00f52000c0032000042eb00044f7800ae
:109b400005003700640247000400780088610200c5
:109b5000000000001e4fe8001e427800e34f520054
:109b6000f8ff36000500370041002000a0d3200098
:109b7000bc610200000000004a2da8005e42900077
:109b800064425200544798000400370064024700c2
:109b90000400780088610200000000005e4290002e
:109ba0008482fb008502ea00cf2ade00854278002d
:109bb0000442e90054479800e0cf5200f3ff3a0016
:109bc000a0003700650247000400780088610200a9
:109bd000000000005e429000e34f5200ba003600e1
:109be0004469800064026200e00f520008003a00fd
:109bf0004100200020d42000bc61020000000000d1
:109c00004a6da8005e42900064425200544798009a
:109c10005e429000e34f520012003600446980001b
:109c200064026200e00f520010003a004100200080
:109c300060d42000bc610200000000004a8da80032
:109c40005e4290006442520054479800080037007a
:109c500064024700040078008861020000000000f0
:109c60000300370000000000010037000000000082
:109c70005e4290008482fb008502ea00cf2ade006b
:109c8000854278000442e90054479800e0cf520032
:109c9000efff3a006b0037006402470004007800d1
:109ca00088610200000000004e429000e44f520024
:109cb00087003a006802470063024200040078000f
:109cc0008861020000000000680247000482e8008a
:109cd000040078008861020000000000680247006c
:109ce0000402e8000400780088610200000000001f
:109cf000680247000400780088610200000000004c
:109d00005000370014002000140798004d00370061
:109d1000640247000400780088610200000000002f
:109d20004e429000e44f52006b003a0044698000bc
:109d300064026200e00f52000c0032000042eb00af
:109d4000044f7800050037006402470004007800e3
:109d500088610200000000001e4fe8001e427800eb
:109d6000e34f5200f8ff360036003700e4d22000ff
:109d700063024200040078008861020000000000d5
:109d8000e4d220000482e800040078008861020028
:109d900000000000e4d220000402e8000400780083
:109da0008861020000000000e4d220000400780076
:109db00088610200000000007669800087698000e9
:109dc0007469800085698000cb28dd004522de00b3
:109dd00004827000c52ade000402530085825b0005
:109de000746988008569880016003700650247009d
:109df00004007800886102000000000004003700c1
:109e0000640247000400780088610200000000003e
:109e10005e4290008482fb008502ea00cf2ade00c9
:109e2000854278000442e90054479800e0cf520090
:109e3000f3ff3a0003003700000000000100370084
:109e4000000000001e029000e00f5200ddfe320014
:109e50006e429000e24f520006003a004e0290001f
:109e6000de02900094698800a5698800284da8004a
:109e70000900370096698000a76980004e029000b3
:109e8000de029000840f5300858f5b0002003200d9
:109e90000042eb00644798000862020000000000e6
:109ea0006e42900010003700000000000b003700e9
:109eb0000000000009003700000000000700370024
:109ec000000000000500370000000000030037001c
:109ed00000000000010037000000000008620200de
:109ee000000000000042eb00044078000080fa000f
:109ef000000006000a00fa00604798004107980039
:109f000010c0b300d45f02000000000010c0b30016
:109f1000d45f02000000000060c0b300d45f020004
:109f2000000000000040eb00d45f020000000000d1
:109f300020c1b300d45f02000000000030c2b300b3
:109f4000d45f02000000000040c3b300d45f0200f1
:109f50000000000060c5b300d45f020000000000f4
:109f60000040eb00d45f0200000000000040eb0066
:109f7000d45f0200000000004469800070026200ab
:109f8000e00f5200020032000042eb0001003700f7
:109f900004c8b30004407800d45f02000000000051
:109fa0000040eb00d45f0200000000006e42900011
:109fb000e34f520008003a004e029000e00f5200ba
:109fc000050032004100200060d320000460020040
:109fd000000000000c0037000040eb00d45f0200de
:109fe000000000000040eb00d45f02000000000011
:109ff0000040eb00d45f0200000000000040eb00d6
:10a00000d45f0200000000000042eb00044f780023
:10a01000040037000040eb00d45f020000000000a5
:10a020001e4fe8001e427800eb4f5200f9ff360049
:10a0300061002000b0d02000046002000000000099
:10a040000042eb00044f7800040037000040eb00b2
:10a05000d45f0200000000001e4fe80094ccb30063
:10a060009e42780084cf5200f8ff360030c6b3001d
:10a07000d45f02000000000020c8b300d45f0200db
:10a080000000000030c5b300d45f020000000000f3
:10a0900030c6b300d45f02000000000050c3b3001c
:10a0a000d45f02000000000010c0b300d45f0200c3
:10a0b000000000006e409000d45f0200000000002d
:10a0c0006e429000e14f520001003a00284da90075
:10a0d0006e429000e34f520020003a004e02900082
:10a0e000e00f52001d003a0060c3b300d45f0200cd
:10a0f0000000000040c0b300d45f02000000000078
:10a1000024d3200063024200144278000440780007
:10a11000d45f02000000000024d320000482e80085
:10a120001442780004407800d45f02000000000070
:10a1300024d320000402e800144278000440780090
:10a14000d45f02000000000024d3200014427800f5
:10a1500004407800d45f02000000000070c3b30028
:10a16000d45f02000000000040c0b300d45f0200d2
:10a170000000000010c0b300d45f02000000000027
:10a1800030c0b300d45f02000000000060c0b30024
:10a19000d45f020000000000c0c0b300d45f020022
:10a1a000000000006e429000e34f520003003a00ae
:10a1b0004e029000e00f5200080032006e42900004
:10a1c000e14f52000f003a00b4698000c569800079
:10a1d000e00f5200e08f5a000a00320020c3b300a3
:10a1e000d45f02000000000040c0b300d45f020052
:10a1f000000000004100200060d320000460020045
:10a200000000000000c0eb00d45f0200000000006e
:10a21000030037000040eb00d45f020000000000a4
:10a22000155e8000b4122000848f5200f9ff3600c2
:10a23000e6cd2000164378008683fb00f6cd200093
:10a24000164378000683fb004833dd0007037300e4
:10a250000602780006ce2000164378008683fb00b5
:10a2600016ce2000164378000683fb004833dd003d
:10a2700007037300860278001407980025079800ea
:10a280004e029000e00f520014003a00e4cd20008e
:10a29000144278006042620004407800deecb700af
:10a2a000f4cd20001442780060426200044078003f
:10a2b000dfecb70004ce2000144278006042620058
:10a2c00004407800e0ecb70014ce2000144278007f
:10a2d0006042620004407800e1ecb7005e6002007a
:10a2e000000000001e029000ae029000f60f200059
:10a2f00086036200e6cd20001643780060436300c9
:10a300000743730006407800deecb700c823de0088
:10a31000f6cd2000164378006043630007437300c6
:10a3200006407800dfecb700f60f2000868362005d
:10a3300006ce200016437800604363000743730095
:10a3400006407800e0ecb700c82ade0014ce2000fa
:10a3500014427800604262000542720004407800b6
:10a36000e1ecb7000080fa00000006000000fa00ef
:10a37000fd030700f47902000000000000027800ed
:10a38000040078000080fa00000006000000fa00d7
:10a39000fe7902000000000000027800040078004e
:10a3a0000080fa00000006000a00fa00404798000a
:10a3b00031079800420798000042eb0024479800bc
:10a3c0000e82e800be0190000e017800ce009000e1
:10a3d0004e409000fa7c020000000000000278006d
:10a3e000e00f520002003a002e4290000c003700ad
:10a3f0001e027800be0290000482420034079800da
:10a400001e027800ce029000048252004407980099
:10a410004e029000e00f5200e9ff3a002e429000f9
:10a42000044078000080fa00000006006e02fa0086
:10a43000c42620000e024200004a78006520200059
:10a440008e8242000042eb00844a78000e82e800cf
:10a45000c52620008e824200120020008400780071
:10a4600015407800d0ff07000042780065202000ea
:10a470008e824200844a7800642020000e0242004e
:10a4800014427800e04f5200170032006420200090
:10a490000e024200144278008482fb0074202000e7
:10a4a0000e024200851f780045262900851f78008e
:10a4b00004007800ee0b020000000000e487570063
:10a4c000742020000e024200c52620008e82420029
:10a4d0000401780011c0b30015407800607e0200ce
:10a4e00000000000b80037002e429000c526200072
:10a4f0008e8242009540780004407800087a02007d
:10a500000000000000027800e10f5200030032005a
:10a510002e429000e04f52009a003a000e82e8006e
:10a52000c52620008e824200840078001540780005
:10a530000801070000427800652020008e8242005a
:10a54000844a7800642020000e0242001442780001
:10a55000e04f520005003200642020000e0242004d
:10a5600014427800ea4f520090003a006420200024
:10a570000e02420014427800e04f52003d003a00c3
:10a580002e4292000482fb000402e8008e82e80062
:10a5900004824200c52620008e8242002200200054
:10a5a00084007800154078007fff070000427800a3
:10a5b000652020008e824200844a780064202000ba
:10a5c0000e02420014427800e04f520017003200a1
:10a5d000642020000e024200144278008482fb00b6
:10a5e000742020000e024200851f7800c52a290031
:10a5f000851f780004007800ee0b020000000000c8
:10a60000e4875700742020000e024200c526200077
:10a610008e8242000401780011c0b300154078001a
:10a62000607e020000000000120037000e82e80089
:10a63000c52620008e8242008400780015407800f4
:10a640009d03070000027800e10f5200090032006c
:10a65000652020008e82420074c0b300844a7800d6
:10a66000c42620000e02420014407800427e020000
:10a6700000000000642020000e0242001442780016
:10a68000e04f520005003200642020000e0242001c
:10a6900014427800ea4f520046003a00351020007c
:10a6a0008e8242000e82e800c62620000e03430080
:10a6b0000501780084007800164078004800070003
:10a6c0002e429000e04f52003c0032003420200027
:10a6d0000e024200144278000482fb006302420032
:10a6e000040f7800642020000e0242003710200082
:10a6f0008e834300452020008e824200c626200023
:10a700000e03430087017800050178009e00780061
:10a7100016407800c27d02000000000000027800b0
:10a72000e00f520027003a00642020000e02420091
:10a73000144278008482fb00742020000e02420044
:10a74000851f7800552e2900851f780004007800a9
:10a75000ee0b020000000000e48757007420200088
:10a760000e024200c52620008e82420004017800bd
:10a7700011c0b30015407800607e020000000000a8
:10a7800011003700652020008e82420064c0b300b3
:10a79000844a7800c42620000e024200144078004b
:10a7a000427e0200000000000700370000000000a9
:10a7b0000500370000000000030037000000000023
:10a7c0000100370000000000642020000e0242005b
:10a7d00014427800044078000080fa00000006006f
:10a7e0000800fa00204798002107980032079800d7
:10a7f0000042eb00044f78002e02900014429000bb
:10a800000482fb006123b9000082eb008082eb0030
:10a810000602420087824a00f6002000070020005e
:10a82000860f5200878f5a002d003e000460010001
:10a830000f0037000e0037001400370013003700f8
:10a84000190037001f0037002500370024003700ab
:10a850002300370022003700210037002000370096
:10a860001f0037001e0037000f00370015003700ab
:10a870003e019000ae0090002e409000dc000700ea
:10a8800000427800044f7800180037003e01900025
:10a89000ae0090002e409000d701070000427800e3
:10a8a000044f7800110037003e019000ae00900088
:10a8b0002e4090003401070000427800044f7800d9
:10a8c0000a0037003e019000ae0090002e4090003c
:10a8d0002602070000427800044f7800030037008a
:10a8e00014c0b300044f7800000000001e4278003e
:10a8f000e04f52000c0032002e0290009442900073
:10a9000004c8b30004c27200be02900094429800d2
:10a910003e0290009e42780025429800be029000c0
:10a9200024c0b30084429a002e02900014427800a2
:10a93000be029000844a7800be0090002e40900035
:10a940003a0307000042eb00044078000080fa0060
:10a95000000006006e00fa0020ef980061379800b2
:10a960000042eb00044f78006e3290000402e800d1
:10a9700012002000840078002ee890008afe070074
:10a9800000427800044f78001e427800e04f5200e9
:10a99000110032001e4278008482fb0066024700ec
:10a9a000851f7800d5312900851f780004007800c4
:10a9b000ee0b020000000000e4875700660247002b
:10a9c0000401780011c0b3002ee89000607e020000
:10a9d00000000000820037006e32900014429000a8
:10a9e0000482fb006123b9000082eb008082eb004f
:10a9f0000602420087824a00f6002000070020007d
:10aa0000860f5200878f5a0039003e000460010013
:10aa10000f0037000e0037000d0037000c00370024
:10aa20000b0037000a0037003100370030003700d4
:10aa30002f0037002e0037002d0037002c00370084
:10aa40002b0037002a0037000600370005003700ca
:10aa500044002000140798002400200024079800d8
:10aa6000290037006e3290000482e8005200200076
:10aa7000840078002ee890004bfe0700004278002a
:10aa8000044f78001e427800e04f520007003a0061
:10aa90006e329000644290000482fb00140798001c
:10aaa0007400200024079800170037001e42780029
:10aab0008482fb0066024700851f78006536290006
:10aac000851f780004007800ee0b020000000000f3
:10aad000e4875700660247000401780011c0b30004
:10aae0002ee89000607e02000000000006003700a3
:10aaf000a4c0b300044f78002ee89000427e02000c
:10ab000000000000000000001e427800e04f5200ec
:10ab100033003a009e02900004102000848f5200ff
:10ab20000b00360084c0b300044f7800c23b2900fc
:10ab300011c0b3002ee89000607e0200000000000b
:10ab40002ee89000427e0200000000002400370042
:10ab5000ee3290002e029000048242001e0190000e
:10ab6000840078002ee890000ffe07000042780075
:10ab7000044f78001e427800e04f5200100032006f
:10ab80001e4278008482fb0066024700851f780021
:10ab9000953d2900851f780004007800ee0b020027
:10aba00000000000e48757006602470004017800b7
:10abb00011c0b3002ee89000607e0200000000008b
:10abc0002e029000844278001e0290000442780019
:10abd00004c242000442e900ee32900084429a002e
:10abe0001e427800044078000080fa000000060051
:10abf0000c00fa006047980041079800520798003f
:10ac00004e029000244290000482fb004822dd00a6
:10ac1000140798004e029000344290000482fb001a
:10ac20009e02900004827200140798004e02900069
:10ac3000444290000482fb004822dd002407980073
:10ac40004e029000544290000482fb00ae0290003d
:10ac500004827200240798002e029000e00f520038
:10ac600043003200ae02900004042000848f5200a2
:10ac70003f003e004e029000144390004e029000b0
:10ac8000944278002e0290009e01900006417800c8
:10ac9000ee40900005407800207a0200000000009d
:10aca00000027800e10f52002e003a005e02900090
:10acb00063024200ce02900095439000ce029000c5
:10acc00015437800840278002e0290009e019000c7
:10acd00007417800ee40900006407800f87a0200c4
:10ace0000000000000427800044f78001e42780007
:10acf000e04f520018003a004e02900014429000bb
:10ad0000de029000944298002e0290004322de0062
:10ad100004427800de029000a44298002e029000c7
:10ad200067026200e00f5200050032005e029000f0
:10ad3000244290000442e800de029000a442980001
:10ad40005e0290002442900004c2e800de029000ff
:10ad500084429a000800370044c0b300044f7800d2
:10ad60000500370024c0b300044f7800020037000c
:10ad700034c0b300044f78001e42780004407800cd
:10ad80000080fa00000006001200fa00404f980010
:10ad900071079800020f98000042eb00044f780002
:10ada00014002000340798007e0290002442900096
:10adb0000482fb004822dd00440798007e029000d8
:10adc000344290000482fb00ce02900004827200a4
:10add000440798007e02900014429000ef4f52000a
:10ade0002b003a007e029000444290000482fb0057
:10adf0004822dd00340798007e0290005442900003
:10ae00000482fb00be0290000482720034079800a6
:10ae10003e029000e00f520004003200be0290009b
:10ae200004042000848f52000300360034c0b300b5
:10ae3000044f7800300037003e0290004322de00cd
:10ae4000244798003e02900067026200e00f520023
:10ae5000030032002e4290000442e800244798008c
:10ae60007e029000e44290002e42900084cf520077
:10ae70000300320034c0b300044f78001e003700d6
:10ae80007e02900067024200240798001a003700f3
:10ae90007e02900044429000e04f520007003a00ca
:10aea0007e02900054429000e04f520003003a00ae
:10aeb0000042eb00244f98000d0037007e02900006
:10aec00044429000e14f420007003a007e029000a9
:10aed00054429000e04f520003003a0014c0b30007
:10aee000244f98000200370034c0b300044f7800ac
:10aef0006a024700240798001e427800e04f520083
:10af000039003a007e029000144390007e029000c7
:10af1000944278003e029000ce01900006417800f5
:10af2000ce48900005407800207a02000000000022
:10af300000027800e10f520029003a007e029000e2
:10af4000944390007e02900014437800ae0290007b
:10af50003e029000ce01900007417800ce4890005c
:10af6000064078007a7c0200000000000042780071
:10af7000044f78001e427800e04f520015003a005e
:10af800014c0b300144798000b0037001e42900015
:10af90008482fb001e4290000482fb007e0390002e
:10afa00066427a000e0b900004f37a001e42900075
:10afb0000442e800144798001e429000e54f5200fa
:10afc000f2ff36008e0a900054c0b30084429a000b
:10afd0000500370044c0b300044f7800020037007a
:10afe00024c0b300044f78001e427800044078006b
:10aff0000080fa00000006000c00fa00604798008c
:10b0000041079800520798004e0290002442900099
:10b010000482fb004822dd00140798004e029000d5
:10b02000344290000482fb009e0290000482720071
:10b03000140798004e029000444290000482fb00e6
:10b040004822dd00240798004e02900054429000f0
:10b050000482fb00ae029000048272002407980074
:10b060002e029000e00f52003a003200ae02900033
:10b0700004022000848f520036003e004e029000f1
:10b08000144390004e029000944278002e029000eb
:10b090009e01900006417800ee4090000540780047
:10b0a000207a02000000000000027800e10f520048
:10b0b00025003a005e02900063024200ce0290003a
:10b0c00095439000ce0290001543780084027800ea
:10b0d0002e0290009e01900007417800ee40900003
:10b0e00006407800f87a0200000000000042780074
:10b0f000044f78001e427800e04f52000f003a00e3
:10b100004e02900014429000de029000944298009b
:10b110002e0290000442780004424200de029000b9
:10b12000a44298005e0290002442900004c2e8000d
:10b13000de02900084429a000800370044c0b30049
:10b14000044f78000500370024c0b300044f780096
:10b150000200370034c0b300044f78001e4278006c
:10b16000044078000080fa00000006000e00fa009b
:10b17000004f980051079800620798000042eb00ca
:10b18000044f780044c0b300244798001400200006
:10b19000240798005e029000244290000482fb0085
:10b1a0004822dd00340798005e029000344290008f
:10b1b0000482fb00be0290000482720034079800f3
:10b1c0005e02900014429000f04f520022003a00bc
:10b1d0005e029000444290000482fb004822dd00a1
:10b1e000240798005e029000544290000482fb0005
:10b1f000ae02900004827200240798002e02900094
:10b20000e00f520004003200ae029000040420005f
:10b21000848f52000300360034c0b300044f78001e
:10b220000d0037002e0290000402420084027800d4
:10b230005e029000644290000482fb00848f520002
:10b240000300320034c0b300044f7800020037001e
:10b2500074c0b300244798001e427800e04f5200ab
:10b260003d003a005e029000144390005e029000a0
:10b27000944278002e029000be01900006417800b2
:10b280008e48900005407800207a020000000000ff
:10b2900000027800e10f52002d003a00de0290001b
:10b2a0002e4290000482fb0004824200de029000e5
:10b2b00095439000de0290001543780084027800e8
:10b2c0002e029000be019000074178008e48900049
:10b2d000064078007a7c02000000000000427800fe
:10b2e000044f78001e427800e04f520015003a00eb
:10b2f00014c0b300144798000b0037001e429000a2
:10b300008482fb001e4290000482fb005e039000da
:10b3100066427a006e03900004f37a001e429000a9
:10b320000442e800144798001e429000e54f520086
:10b33000f2ff3600ee02900054c0b30084429a003f
:10b340000500370044c0b300044f78000200370006
:10b3500024c0b300044f78001e42780004407800f7
:10b360000080fa00000006000a00fa006022b8001f
:10b37000048fbe00480037001e02be00240798005c
:10b380003507980084c0b300044f980016003700ba
:10b390002e0290006102620004427800e04f5200e9
:10b3a0000b0032002e029000be0290008503d100f7
:10b3b0000483d30014002a000500200004026b005f
:10b3c00085826b0024079800350798000600370037
:10b3d0002e029000be0290008502d1000482d300ac
:10b3e00024079800350798000e4a90000482fb005d
:10b3f0000402ea004f22de00044278008e4a9000e8
:10b400008542e900054f9800e04f5200e0ff3a0006
:10b410002e039000be03900004f02f0005002000d2
:10b42000060078000703780084037800050278009e
:10b43000070060000402630005002000c022dd0058
:10b44000040020000403be006102b800040373007e
:10b4500085837300c838dd004832de000482700046
:10b46000c83ade0004427800059020009e82420027
:10b47000844a78002e029000044278000580200063
:10b480009e824200844a78001400200005002000bb
:10b490001e0f42005e974a00f40f200005002000b6
:10b4a0001e03be00840f5300858f5b00b2ff360081
:10b4b0000080fa00000006007000fa0040ef9800db
:10b4c0007137980000c2eb00044f780000c2eb0017
:10b4d000144798007e329000044292000442e80033
:10b4e000344798000042eb002447980017003700cb
:10b4f0002e4290000482fb00fe329000e5427a006a
:10b500001e42900004c26a000482fb000500200075
:10b510002407980035079800ae02900004802000b0
:10b5200004824200144278001e426a0014479800c8
:10b53000ae0290000490200004824200144f780074
:10b540002e4290000442e80024479800ae4290004a
:10b550003e42900084cf5200e5ff39003e42900009
:10b560000482fb00fe329000e5427a001e42900009
:10b5700084cf520009003a003e4290000482fb0052
:10b580000402e800fe32900065427a009e4f5200ad
:10b5900002003a0014002000210037003e429000d3
:10b5a0000482fb000402e800fe32900065427a004b
:10b5b0000480fb003e4290000482fb00fe329000bb
:10b5c00065427a008483fb001e4278000483fb00fe
:10b5d0001e4290008482fb0068024700801f7800b2
:10b5e000871f7800861f7800851f7800e5422900b4
:10b5f000851f780004007800ee0b020000000000b8
:10b60000ea875700680247000401780011c0b300c0
:10b610004ee89000607e0200000000000002eb0097
:10b62000040078000080fa00000006000a00fa001a
:10b63000604798004107980000c2eb00044f780073
:10b6400000c2eb00144798004e02900004429200a2
:10b650000442e800344798000042eb002447980079
:10b66000150037002e4290000482fb00ce029000ad
:10b67000e5427a001e42900004c26a000482fb0088
:10b6800024079800ae02900004802000048242004b
:10b69000144278001e426a0014479800ae029000df
:10b6a0000490200004824200144f78002e42900043
:10b6b0000442e80024479800ae4290003e429000c9
:10b6c00084cf5200e7ff39003e4290000482fb0025
:10b6d000ce0290001e43900086727a003e42900097
:10b6e0000482fb000402e800ce0290001e437800b2
:10b6f00086727a000080fa00000006000200fa005c
:10b700000042eb00044f7800030037001e40780031
:10b71000d30107001e4fe8001e427800e74f520099
:10b72000faff3600ca2ba8000080fa0000000600cd
:10b730000e00fa002007980031079800024f980089
:10b74000530798006407980004b02000140798007d
:10b750000042eb00044f78007b0037001e0290008f
:10b7600064029000e00f520073003a001e02900045
:10b770005e009000600298005e029000e00f5200b0
:10b780000f003a004570800004002200848f5200b0
:10b7900004003e0045708000f4ff2000848f5200ba
:10b7a00002003e00040021004470880044708000c4
:10b7b0009e029000e40298000402e80044708800b1
:10b7c0000e4a9000e04f5200050032002e02900019
:10b7d000be029000e00f5200e08f5a000a003a00cb
:10b7e0001e029000a2002000f10f2000040078004b
:10b7f000b00b0200000000001e0290005500200067
:10b8000075029800450037000e4a90000482fb0044
:10b810006123b9000082eb008082eb000602420047
:10b8200087824a003600200007002000860f520061
:10b83000878f5a0038003e00046001000300370083
:10b840000200370018003700270037001e02900062
:10b850002e039000be039000068abe000e4a9000a0
:10b860000414a2000482fb000402e9004f22de005f
:10b87000044278009e0290000482fb006102620094
:10b880004822dd00a50b9000f6ef2f000683630031
:10b8900004027300a40a98001e0290001500200004
:10b8a000750298001d0037001e0290002e039000c4
:10b8b000be039000068abe009e0290000042eb008c
:10b8c000c45298001e039000d403200005002000fd
:10b8d000040b9800150b98001e0290002500200014
:10b8e000750298000d0037002e0290008402780047
:10b8f0001e029000a200200085007800040078005d
:10b90000a20b0200000000001e0290005500200063
:10b910007502980001003700000000001e02900030
:10b92000ee039000570298001e407800c0ebb7006d
:10b930001e427800080037001e0290007802420084
:10b94000140798001e4fe8001e427800e74f52008f
:10b9500082ff360000c2eb00044078000080fa004d
:10b96000000006000600fa00881f78000042eb0085
:10b97000044f7800220137009e4278000582fb00c8
:10b980007822b90004027800ee02420004b02000e0
:10b990000482420014027800e50f52000c013200cc
:10b9a0009e4278000582fb007822b90004027800ec
:10b9b000ee02420004b0200004824200140278002b
:10b9c000e40f5200040132009e4278000582fb0021
:10b9d0007822b90004027800ee02420004b0200090
:10b9e0000482420014027800050020003600200086
:10b9f00007002000860f5200878f5a00f8003e0093
:10ba00000460010036003700020037006c00370088
:10ba100088003700ec63020000000000000278009c
:10ba2000e00f5200f00032009e4278000582fb00d9
:10ba30007822b90084027800e4b020000482420039
:10ba40008002eb00050a78009e4278000582fb0028
:10ba50007822b90004027800f402420004b0200009
:10ba600004824200140278004822de006142620033
:10ba7000e04f52000d0032009e4278000582fb002c
:10ba80007822b9008402780004b0200004824200c9
:10ba90001402be000402780011c0b3000400780054
:10baa0003864020000000000d40037009e42780095
:10bab0000582fb007822b9008402780004b02000df
:10bac000048242001402be000402780011c0b300d8
:10bad000040078003864020000000000c70037004e
:10bae0000e82e800040078006a6402000000000092
:10baf00000027800e00f5200bd0032000664020030
:10bb00000000000000027800e00f52002300320025
:10bb10001e4278000483fb001e029000ae029000db
:10bb20007833b9008603780006b02000068343000e
:10bb3000048bbe009e4278000582fb007822b9008b
:10bb400084027800e4b02000048242002500200036
:10bb5000050a78009e4278000582fb007822b90031
:10bb60008402780044b12000848242000042eb004d
:10bb7000844a78009e4278000582fb007822b90052
:10bb80008402780004b1200004834200d403200022
:10bb900005002000048bbe00980037009e4278000c
:10bba0000582fb007822b90084027800e4b020000e
:10bbb0000482420015002000050a78008f0037003b
:10bbc0001e4278000484fb00a68f020000000000e3
:10bbd0000002be00040378007842b90084027800b5
:10bbe00064b1200004824200060a78009e42780078
:10bbf0000582fb007822b9008402780004b020009e
:10bc00000482420004007800488002000000000026
:10bc10009e4278000582fb007822b90084027800f9
:10bc2000e4b020000482420035002000050a7800bc
:10bc3000720037009e4278000582fb007822b9002e
:10bc400004027800e402420004b0200004834200b1
:10bc50009e4278000582fb007822b90084027800b9
:10bc600004b02000048242008600780004007800be
:10bc70000a8102000000000000027800e00f52007c
:10bc80004a003a00a68f0200000000000002be0039
:10bc9000040378009e4278000582fb007822b900f8
:10bca00004027800f602420004b020000482420040
:10bcb00014027800040353009e4278000582fb00c2
:10bcc0007822b90004027800f002420004b020009b
:10bcd000048242001402be0004027800840f530064
:10bce000450036009e4278000582fb007822b900ac
:10bcf00004027800f402420004b0200004824200f2
:10bd000014427800e54f52001f003e001e427800aa
:10bd10008483fb00783ab90004027800f402420000
:10bd200004b0200004824200144278000443e8007a
:10bd3000783ab9008402780044b1200004824200bd
:10bd4000064a78009e4278000583fb009e427800f8
:10bd50000582fb007822b90004027800f00242005c
:10bd600004b02000048242001402be00040242001b
:10bd700085824a007833b9008603780006b1200036
:10bd800006834300048bbe009e4278000582fb00c0
:10bd90007822b90084027800e4b0200004824200d6
:10bda00025002000050a7800140037009e42780024
:10bdb0000582fb007822b90084027800e4b02000fc
:10bdc0000482420055002000050a78000b0037006d
:10bdd00000000000090037000000000007003700e5
:10bde00000000000050037000000000003003700dd
:10bdf0000000000001003700000000001e4fe800b6
:10be00001e427800e74f5200dbfe36004f047800f8
:10be10000080fa00000006000200fa00004f7800df
:10be20009e4278000582fb007822b9000402780067
:10be3000ee02420004b020000482420014027800a6
:10be400065026a0004f0a7000402ea000402e900a7
:10be50004f22de00040078000080fa000000060097
:10be60000200fa00004f78001e427800e74f5200af
:10be700019003e009e4278000582fb007822b9003e
:10be800084027800c4b02000048242008002eb00eb
:10be9000050a78009e4278000582fb007822b900ee
:10bea0008402780004b02000048342006022b800bd
:10beb000048bbe009e4278000582fb007822b90008
:10bec00084027800e4b02000048242004500200093
:10bed000050a780001003700000000000080fa0029
:10bee000000006000200fa00000f7800a502200002
:10bef0001e82420004007800083d0200000000009d
:10bf00001e027800345e88000080fa0000000600ff
:10bf10000200fa00000f78009e027800688242005a
:10bf200004007800728b0200000000001e027800fe
:10bf3000445e88000080fa00000006000200fa005b
:10bf4000004f7800843a02000000000000027800f0
:10bf5000e00f520002003a000002eb000f00370031
:10bf600064e02000144278009e4f52000600320028
:10bf70001e40780006eeb7000002eb00145e880059
:10bf80000000eb00d7ff07001e407800c0ebb700b1
:10bf9000145e8000055c20000482520004007800da
:10bfa0000080fa00000006000200fa00004f78004e
:10bfb000355e8000f45b2000848f52000200360062
:10bfc0000002eb000d0037001e407800343f0200f5
:10bfd00000000000345e80000402e800345e880047
:10bfe000355e8000145e8000848f520002003600af
:10bff000345e8000145e8800140020000400780085
:10c000000080fa00000006000600fa001007980001
:10c0100021079800345e8000055c2000048f5200e8
:10c020002e0290009e027800848f520002003100a0
:10c030001e02780024079800355e80002e029000d2
:10c0400004824200345e8800355e8000145e800009
:10c05000848f520002003600345e8000145e880037
:10c06000ae0090001e009000443f0200000000005f
:10c070002e029000040078000080fa000000060004
:10c080000200fa00000f78001e0278000400780019
:10c09000e00b02000000000000027800840078003d
:10c0a0001e007800d8ff0700000278001e02420040
:10c0b000040078000080fa00000006001c00fa006e
:10c0c00004bc2000144278000482fb007822b900ee
:10c0d0008402780004b02000048f4200145e8000c7
:10c0e00068024200140798001e0278006402900063
:10c0f0000400780052710200000000000002780085
:10c10000340798001e027800540290000400780062
:10c1100052710200000000000002780044079800fd
:10c120001e00900052710200000000000002780022
:10c13000540798000002eb0064079800e6cd200049
:10c14000164378008683fb00f6cd20001643780066
:10c150000683fb004833dd00070373000602780006
:10c1600006ce2000164378008683fb0016ce200002
:10c17000164378000683fb004833dd000703730095
:10c180008602780074079800050f98001e02780058
:10c190001403be00160f9800270f98000042eb0012
:10c1a0006457980014c1b300745798009e03900020
:10c1b000470f98004e0a9000040078005271020068
:10c1c0000000000000027800440f98006e02470053
:10c1d000c100200004007800ce71020000000000c1
:10c1e000000278000482ea0064079800e000200062
:10c1f000083d0200000000001e0278001e019000b1
:10c2000011c1b30004007800c08a020000000000e1
:10c21000660247008100200004007800443f0200cd
:10c220000000000020022000223d0200000000006b
:10c2300000027800240798001e009000bc3d020018
:10c240000000000000027800540f98005e0a900081
:10c25000e00f520002003a000082eb00540f9800f9
:10c260002e009000223d020000000000800220000d
:10c27000083d0200000000007a0247002100200073
:10c2800004007800443f020000000000883c0200e7
:10c29000000000000002eb00145e880000c2eb000a
:10c2a0000440780006eeb7000080fa0000000600a7
:10c2b0000200fa00004f78001e407800c0ebb70083
:10c2c00074e02000144278009e4f520002003200b9
:10c2d0000002eb000b003700a4bc200014427800e1
:10c2e00061426200e04f520003003200ca0ba90015
:10c2f0000000eb0006ff0700255e8000445e800022
:10c3000004825200040078000080fa000000060059
:10c310000200fa00000f7800455e8000245e800075
:10c32000848f52000600310075e0200095427800ad
:10c3300004bc20001442780084cf52000200320076
:10c340000002eb0009003700e83e02000000000098
:10c35000004278009e027800844a7800445e8000a3
:10c360000402e800445e8800140020000400780005
:10c370000080fa00000006000600fa00100798008e
:10c3800021079800455e8000245e8000848f520063
:10c390000600310075e020009542780004bc2000c2
:10c3a0001442780084cf5200020032000002eb00f9
:10c3b00014003700255e8000445e8000048f520028
:10c3c0002e0290009e027800848f520002003100fd
:10c3d0001e02780024079800ae0090001e00900016
:10c3e000fa3e0200000000000002780024079800d6
:10c3f000455e80002e02900004824200445e880068
:10c400002e029000040078000080fa000000060070
:10c410000000fa00a4bc20001442780062426200ce
:10c42000e04f520008003a009c3a02000000000071
:10c430000002eb00245e880000c2eb00044078009c
:10c4400007eeb700ca2ba8000080fa000000060023
:10c450002000fa00500f9800610f9800720f9800aa
:10c460000002eb00245e88000e82e80081002000bc
:10c4700004007800fa3e0200000000001e02900056
:10c4800004007800527102000000000000027800f1
:10c49000140798002e0290000400780052710200e8
:10c4a0000000000000027800240798003e0290007f
:10c4b00004007800527102000000000000027800c1
:10c4c00068025200340798004e029000e00f5200bc
:10c4d000390032005e0b9000164278000480fb00a9
:10c4e000964390008783fb00c83bdd008083730088
:10c4f00007027800a64390008783fb003643900034
:10c500000683fb004833dd000703730086027800d2
:10c5100054079800650798006e0a90001402be0048
:10c5200074079800050f98000042eb00245798000c
:10c5300014c1b300345798007e089000200f980073
:10c540002e0a9000040078005271020000000000e2
:10c5500000027800240f98006a024700c100200002
:10c5600004007800ce710200000000000002780094
:10c570000482ea00340f98000000eb00728b020086
:10c58000000000007e089000bc3d0200000000009a
:10c5900000027800440f9800be0a90004e0a9000f6
:10c5a000848f5200040032009c3a02000000000018
:10c5b0000002eb00150037000e82e8006e099000c3
:10c5c000de089000040078001300070000427800a5
:10c5d000044f78001e427800e14f420004003a0008
:10c5e0009c3a0200000000000002eb000700370048
:10c5f0001e40780007eeb7003e029000245e8800df
:10c60000ca0ba800ca2ba90014002000040078005f
:10c610000080fa00000006000a00fa0020079800d7
:10c6200031079800420798003e029000944278003b
:10c630000580fb00944290008582fb00c82add0043
:10c640008082720005037800a44290008582fb007e
:10c65000344290000482fb004822dd000502720093
:10c6600084037800deccbf008080fb00dfccbf00fd
:10c670000080fb004800dd0001007000000278002f
:10c68000e0ccbf008080fb00e1ccbf000080fb005d
:10c690004800dd000100700080027800840f530024
:10c6a000858f5b0002003a0000c2eb0047003700b4
:10c6b00000c2eb001447980004b020001407980053
:10c6c0000042eb00044f7800280037001e02900063
:10c6d000e40290002e02900014029000848f520019
:10c6e0001e003a001e029000d40290002e0290001c
:10c6f00014027800848f520016003a001e02900047
:10c700001403be003e009000104278000481fb003c
:10c71000904090008180fb00c808dd00828070009e
:10c7200001027800a04090008180fb003040900022
:10c730000080fb004800dd000100700080027800ee
:10c74000840f5300858f5b0002003a001e42780080
:10c750001e0037009e427800154798001e02900088
:10c7600078024200140798001e4fe8001e4278002d
:10c77000e74f5200d5ff36001e429000e14f4200c5
:10c78000110032001e4290000482fb007822b900a2
:10c790008402780004b0200004824200140798004c
:10c7a0001e029000a2002000be009000040078004d
:10c7b000a20b0200000000002e02900094027800fc
:10c7c0001e029000550298001e429000044078001e
:10c7d0000080fa00000006000000fa0044da2000a1
:10c7e0001442780061426200e04f520002003200c1
:10c7f0000002eb0002003700a40da8001400200086
:10c80000040078000080fa00000006000000fa0032
:10c81000a4de200014427800e14f420008003200fc
:10c82000a4de20001442780004407800305f02004b
:10c830000000000000c2eb0004407800eaedb70001
:10c8400074002000646f8800a40da90044da200061
:10c85000144278000482fb000402d10061426200ad
:10c860000482fb00040078000080fa00000006004b
:10c870000400fa00000f780021479800a1d9200099
:10c880001e007800126e0200000000000002780016
:10c89000e00f520004003200a42da8007400200014
:10c8a000646f8800090037001e007800a06c8800c3
:10c8b0000002eb00b46c88000002eb00646f88009b
:10c8c0002e40900098edb700a42da9000080fa003a
:10c8d000000006001c00fa00500f9800646f8000f2
:10c8e000050020007600200007002000860f52007f
:10c8f000878f5a0082033e00046001000700370062
:10c900000c0037001b0037004c0037005c0037007c
:10c91000b00037007c0237006d0237000042eb00a8
:10c9200004407800a5edb7000042eb000440780019
:10c93000a6edb700a0ce2000488002000000000055
:10c9400054da2000144278000442e80004407800e1
:10c95000a5edb700988f0200000000000002be00a5
:10c96000446d8800556d880024002000646f8800a5
:10c9700063033700e1d92000a0ce20000a81020025
:10c980000000000000027800e00f520015003a009d
:10c99000988f0200000000000003be00446d80007c
:10c9a000556d80000403530085835b0044422f00d3
:10c9b00005002000840f5300858f5b00470336007d
:10c9c00054da200014427800e24f52000200360090
:10c9d000640020000100370014002000646f88000c
:10c9e00047033700a6ce2000164378008683fb005d
:10c9f000b6ce2000164378000683fb004833dd00e6
:10ca00000703730006027800c6ce200016437800a4
:10ca10008683fb00d6ce2000164378000683fb00f9
:10ca20004833dd000703730086027800d46c880069
:10ca3000e56c880034002000646f8800a4d92000d1
:10ca40006123b800540320008001eb0042c0b30012
:10ca50000600be00985b0200000000000042780063
:10ca600004407800eaedb700a4de2000144278000c
:10ca7000e14f42001b03320044002000646f880035
:10ca8000a4de200014427800044078009e5f02007b
:10ca90000000000000027800e00f52001303320093
:10caa000047080000402e8000470880014e0200094
:10cab0001442780004407800d45f020000000000b7
:10cac00004e020001442780004407800d45f0200a3
:10cad0000000000010c0b300d45f0200000000009e
:10cae0000040eb00d45f0200000000000040eb00bb
:10caf000d45f02000000000010c0b300d45f020049
:10cb0000000000000040eb00d45f020000000000c5
:10cb10000040eb00d45f0200000000000040eb008a
:10cb2000d45f0200000000000040eb00d45f020070
:10cb3000000000000040eb00d45f02000000000095
:10cb40000040eb00d45f020000000000a46c8000f5
:10cb5000e00f520004003200a46c80000400780052
:10cb6000eb02070003003700b46c8000040078007b
:10cb7000e70207000040eb00d45f02000000000065
:10cb800084d920001442780004407800d45f020069
:10cb9000000000000040eb00d45f02000000000035
:10cba00010c0b300d45f0200000000005e6002000d
:10cbb00000000000988f0200000000000002be008c
:10cbc000446d8800556d880054002000646f880013
:10cbd000cb023700a4de2000144278000440780025
:10cbe000586102000000000000027800e00f5200cf
:10cbf0000f003a00988f0200000000000003be0002
:10cc0000446d8000556d80000403530085835b00f4
:10cc100044422f0005002000840f5300858f5b00e5
:10cc2000b402360064002000646f8800b40237004c
:10cc3000640247000402e8000400780088610200f2
:10cc400000000000640247000400780088610200d0
:10cc500000000000ae02900004708000848f52003b
:10cc6000030032000862020000000000a402370046
:10cc700064024700630242000400780088610200f9
:10cc800000000000640247000482e800040078000d
:10cc90008861020000000000640247006502420053
:10cca0000400780088610200000000006402470070
:10ccb0006402420004007800886102000000000065
:10ccc00064024700670242000400780088610200a5
:10ccd0000000000064024700660242000400780081
:10cce00088610200000000006402470069024200ff
:10ccf0000400780088610200000000006402470020
:10cd00006802420004007800886102000000000010
:10cd1000640247006b024200040078008861020050
:10cd200000000000640247006a024200040078002c
:10cd3000886102000000000013003700ba020700fb
:10cd40000e82e8000402e800040078008861020016
:10cd5000000000000e82e8000400780088610200f4
:10cd6000000000000e82e8000402e80004007800e1
:10cd700088610200000000000e82e80004007800d4
:10cd80008861020000000000ce02900005027800d9
:10cd900004f0a7000402ea000402ea004f22de00c9
:10cda000044278008502e90045079800e04f5200f0
:10cdb000e2ff3a005d0037009b0207007002470067
:10cdc0000402e8000400780088610200000000000e
:10cdd0007002470004007800886102000000000033
:10cde000700247006302420004007800886102007c
:10cdf00000000000700247000482e8000400780090
:10ce000088610200000000007002470067024200d3
:10ce100004007800886102000000000070024700f2
:10ce200066024200040078008861020000000000f1
:10ce30007002470065024200040078008861020029
:10ce40000000000070024700640242000400780005
:10ce50008861020000000000700247006902420081
:10ce600004007800886102000000000070024700a2
:10ce7000680242000400780088610200000000009f
:10ce80000e0a9000e10f520018003a001e0a9000ae
:10ce9000e10f520017003a004e0a9000e40f5200d2
:10cea00016003a00a42da800a0d920008861020035
:10ceb00000000000b0d920008861020000000000de
:10cec000c0d920008861020000000000d0d92000f5
:10ced0008861020000000000f10037000e007800b9
:10cee000886102000000000005003700000000001b
:10cef00003003700000000000100370000000000c0
:10cf0000ce0a90000502780004f0a7000402ea00af
:10cf10000402ea004f22de00044278008502e900a4
:10cf2000450f9800e04f5200ecff3a00de029000ff
:10cf30000502780004f0a7000402ea000402ea00f7
:10cf40004f22de00044278008502e9005507980070
:10cf5000e04f520098ff3a005d00370032020700b0
:10cf6000700247000402e8000400780088610200b3
:10cf70000000000070024700040078008861020091
:10cf800000000000700247006302420004007800c5
:10cf90008861020000000000700247000482e8007f
:10cfa0000400780088610200000000007002470061
:10cfb000670242000400780088610200000000005f
:10cfc0007002470066024200040078008861020097
:10cfd0000000000070024700650242000400780073
:10cfe00088610200000000007002470064024200f5
:10cff0000400780088610200000000007002470011
:10d00000690242000400780088610200000000000c
:10d010007002470068024200040078008861020044
:10d02000000000000e0a9000e10f520018003a00c4
:10d030001e0a9000e10f520017003a004e0a9000bd
:10d04000e40f520016003a00a42da800a0d9200039
:10d050008861020000000000b0d920008861020051
:10d0600000000000c0d9200088610200000000001c
:10d07000d0d920008861020000000000880037003d
:10d080000e007800886102000000000005003700f3
:10d09000000000000300370000000000010037001e
:10d0a00000000000ce0a90000502780004f0a700fe
:10d0b0000402ea000402ea004f22de000442780083
:10d0c0008502e900450f9800e04f5200ecff3a005e
:10d0d000ee0290000502780004f0a7000402ea00c6
:10d0e0000402ea004f22de00044278008502e900d3
:10d0f00065079800e04f520098ff3a005d00370046
:10d10000c9010700700247000402e800040078002b
:10d1100088610200000000007002470004007800ef
:10d1200088610200000000007002470063024200b4
:10d1300004007800886102000000000070024700cf
:10d140000482e8000400780088610200000000000a
:10d150007002470067024200040078008861020004
:10d1600000000000700247006602420004007800e0
:10d170008861020000000000700247006502420062
:10d18000040078008861020000000000700247007f
:10d190006402420004007800886102000000000080
:10d1a00070024700690242000400780088610200b2
:10d1b000000000007002470068024200040078008e
:10d1c00088610200000000000e0a9000e10f52008a
:10d1d00018003a001e0a9000e10f520017003a00b2
:10d1e0004e0a9000e40f520016003a00a42da80049
:10d1f000a0d920008861020000000000b0d9200002
:10d200008861020000000000c0d92000886102008f
:10d2100000000000d0d9200088610200000000005a
:10d220001f0037000e007800886102000000000037
:10d230000500370000000000030037000000000078
:10d240000100370000000000ce0a900005027800bf
:10d2500004f0a7000402ea000402ea004f22de0004
:10d26000044278008502e900450f9800e04f520023
:10d27000ecff3a00fe0290000502780004f0a700df
:10d280000402ea000402ea004f22de0004427800b1
:10d290008502e90075079800e04f520098ff3a00b8
:10d2a0000862020000000000a4de200014427800a2
:10d2b00004407800305f02000000000000c2eb0074
:10d2c00004407800eaedb70074002000646f880025
:10d2d00044da20001442780062426200e04f5200bb
:10d2e00003003a006022b800d46c8800e56c880026
:10d2f000d46c8000e56c80005e0b9000048bbe0057
:10d3000014002000ff00370064da20001442780087
:10d31000e14f5200050036005e0b90006022b8001d
:10d32000048bbe0014002000f600370064da2000f1
:10d33000144278000442e80004407800a6edb700eb
:10d34000e6ce2000164378008683fb00f6ce200050
:10d35000164378000683fb004833dd0007037300a3
:10d360000602780006cf2000164378008683fb0073
:10d3700016cf2000164378000683fb004833dd00fb
:10d380000703730086027800e00f5200e08f5a0016
:10d39000da003200a4ce2000144278008482fb0020
:10d3a000b4ce2000144278000482fb004822dd0045
:10d3b0000502720004037800c4ce200014427800f5
:10d3c0008482fb00d4ce2000144278000482fb004b
:10d3d0004822dd000502720084037800eeccbf0015
:10d3e0008080fb00efccbf000080fb004800dd0028
:10d3f0000100700000027800f0ccbf008080fb00cc
:10d40000f1ccbf000080fb004800dd00010070008f
:10d410008002780004026b0085826b00f60f20000a
:10d4200086036200a6ce20001643780060436300a6
:10d430000743730006407800eaecb700c823de001b
:10d44000b6ce2000164378006043630007437300a4
:10d4500006407800ebecb700f60f200086836200f0
:10d46000c6ce200016437800604363000743730074
:10d4700006407800ececb700c82ade00d4ce2000cd
:10d480001442780060426200054272000440780055
:10d49000edecb700e4ce2000144278008482fb005b
:10d4a000f4ce2000144278000482fb004822dd0004
:10d4b000050272000403780004cf200014427800b3
:10d4c0008482fb0014cf2000144278000482fb0009
:10d4d0004822dd000502720084037800eaccbf0018
:10d4e0008080fb00ebccbf000080fb004800dd002b
:10d4f0000100700000027800ecccbf008080fb00cf
:10d50000edccbf000080fb004800dd000100700092
:10d510008002780004026b0085826b00f60f200009
:10d5200086036200e6ce2000164378006043630065
:10d530000743730006407800eeecb700c823de0016
:10d54000f6ce200016437800604363000743730063
:10d5500006407800efecb700f60f200086836200eb
:10d5600006cf200016437800604363000743730032
:10d5700006407800f0ecb700c82ade0014cf200087
:10d580001442780060426200054272000440780054
:10d59000f1ecb700a4ce2000144278008482fb0096
:10d5a000b4ce2000144278000482fb004822dd0043
:10d5b0000502720004037800c4ce200014427800f3
:10d5c0008482fb00d4ce2000144278000482fb0049
:10d5d0004822dd000502720084037800eeccbf0013
:10d5e0008080fb00efccbf000080fb004800dd0026
:10d5f0000100700000027800f0ccbf008080fb00ca
:10d60000f1ccbf000080fb004800dd00010070008d
:10d610008002780004026b0085826b00f60f200008
:10d6200086036200a6ce20001643780060436300a4
:10d630000743730006407800eaecb700c823de0019
:10d64000b6ce2000164378006043630007437300a2
:10d6500006407800ebecb700f60f200086836200ee
:10d66000c6ce200016437800604363000743730072
:10d6700006407800ececb700c82ade00d4ce2000cb
:10d680001442780060426200054272000440780053
:10d69000edecb7000042eb0004407800a5edb700c8
:10d6a000a4de200014427800e14f4200080032005e
:10d6b000a4de20001442780004407800305f0200ad
:10d6c0000000000000c2eb0004407800eaedb70063
:10d6d00014002000646f880009003700000000007b
:10d6e00007003700000000000500370000000000c0
:10d6f00003003700000000000100370000000000b8
:10d700000002eb00040078000080fa000000060030
:10d710000600fa00200798002e029000040f7800ff
:10d7200001003700000000001e02780094427800db
:10d73000254798001e0fe8002e429000e04f52004f
:10d7400010003200ae429000e4c2b30084cf520019
:10d750000c003200ae429000f4c2b30084cf5200fd
:10d7600008003200ae429000c4c2b30084cf520021
:10d7700004003200ae429000e4c3b30084cf5200f4
:10d78000e9ff3a001e027800844278002e029000e1
:10d790000442780004c252000442e9003447980071
:10d7a0003e409000d45f0200000000003e42900026
:10d7b0000482fb00840078002e00900004600200c8
:10d7c00000000000000278000402e800ae029000b1
:10d7d00004824200240798002e429000e04f52003d
:10d7e0000c003200ae429000f4c2b30084cf52006d
:10d7f00008003200ae429000c4c2b30084cf520091
:10d8000004003200ae429000e4c3b30084cf520063
:10d81000c4ff3a000040eb00d45f020000000000ab
:10d820000080fa00000006000200fa000e007800f6
:10d83000886102000000000000027800e00f520042
:10d84000150032001e4278008482fb00040c200088
:10d8500084826200040c2000848f520004003a008d
:10d860000e00780088610200000000000d00370003
:10d870001e427800e04f5200090032001e4278003c
:10d880000482fb00840078000000eb00bc61020011
:10d8900000000000e5ff3700000000000100370035
:10d8a000000000000080fa00000006000a00fa00f4
:10d8b0003007980041079800746f8000856f8000e2
:10d8c00014079800250798003e029000ce029000b1
:10d8d000e00f5200e08f5a0004003a0014002000cc
:10d8e0000500200034079800450798003e0290008c
:10d8f000ce029000746f8800856f88000042eb00b4
:10d90000044f780002003700090007001e4fe800ae
:10d910001e427800ef4f5200fbff36001e029000bf
:10d92000ae0290000400be000080fa000000060075
:10d930000200fa000042eb00044f78002b00370091
:10d94000746f8000856f80008500d1000480d30053
:10d95000766f8000876f8000140020000500200093
:10d960000601780007037800840378000502780038
:10d97000070161000402630005002000c022dd00f1
:10d98000040020000403be006112b8000403730009
:10d990008583730060031300e0831b0014002000e4
:10d9a00005002d0006017800070378008403780045
:10d9b00005027800070161000402630005002000f1
:10d9c000c022dd00040020000403be006112b80084
:10d9d0000403730085837300060268008782680071
:10d9e000746f8800856f88001e4fe8001e42780023
:10d9f000ee4f5200d2ff3600746f8000856f8000ba
:10da000004027800040078000080fa00000006009c
:10da10001a00fa00881f7800041980004407980053
:10da20001419800054079800241980006407980096
:10da3000240880007407980014088000040f9800e0
:10da40000002eb000419880004f029002419880062
:10da5000f403200014198800440e280004198800db
:10da600004002800240888000082eb0014088800c5
:10da70000042eb00044f78006022b80024079800b1
:10da8000350798000002eb0014079800a8ff070074
:10da90000002780005002000340f9800450f980020
:10daa00001003700000000000060fe0000000000e0
:10dab000250480000400220004826200e00f52006e
:10dac000fbff320004088000140f98000002eb00f6
:10dad0000408880085a0a90095ff070000027800cf
:10dae000240f98001e0a9000050020002e039000cd
:10daf000be0390000602420087824a002407980075
:10db0000350798002e039000be039000f43f2200da
:10db1000450f2000840f5300858f5b000b003600fb
:10db20003e0c900082ff07000002780004026c00a7
:10db3000340f98004e0c90007dff07000002780023
:10db400004026c00440f9800240037009e029000ed
:10db50001e0a9000848f520002003a00000000006c
:10db6000d1ff37009e0290001e0a9000848252006e
:10db70002e0a900004824200050020000400be002e
:10db80004aff07001e0a9000140798003e0a900002
:10db9000ce0a90000402420085824a00340f9800a9
:10dba000450f980062ff070000027800050820007a
:10dbb00005026200e00f5200030032003e0a9000ae
:10dbc0000400a000340f98001e4fe8001e427800a9
:10dbd000e04f5200b3ff3a00000000000002eb00eb
:10dbe000041988006e029000241988005e029000db
:10dbf000141988004e029000041988007e029000db
:10dc0000240888000e0a9000140888003e0a90003c
:10dc1000ce0a90000400be004f0478000080fa0095
:10dc2000000006000c00fa00400798005107980019
:10dc30000042eb00044f78000042eb0014479800cc
:10dc40006022b8002407980035079800700037005c
:10dc50001e429000e34f52007b003e00ae42900017
:10dc600004cdb30004c24200244798001e4278004d
:10dc7000e04f520005003a002e429000e94f52005a
:10dc8000580036000002eb00a20037001e42780068
:10dc9000e34f520028003a002e429000e24f42002b
:10dca000020032000002eb009a0037002e039000c1
:10dcb000be0390005450200025002000840f530024
:10dcc000858f5b00020036000002eb0091003700f8
:10dcd0001e4290008483fb006e42900045062000a7
:10dce00005a2b90004027800044378005e42900067
:10dcf0006a22b9000402780004427800844243009a
:10dd00004e42900004c24200de0290008782420030
:10dd1000844a78001e4290000442e80014479800ac
:10dd20000042eb00044f78006022b80024079800fe
:10dd300035079800360037002e429000e24f42002f
:10dd400023003a002e039000be03900054502000a0
:10dd500025002000840f5300858f5b0002003600f1
:10dd60000002eb006b0037001e4290008483fb0032
:10dd70006e4290004506200005a2b900040278001a
:10dd8000044378005e4290006a22b90004027800e1
:10dd900004427800844243004e42900004c2420094
:10dda000de02900087824200844a78001e42900082
:10ddb0000442e800144798000042eb00044f78004a
:10ddc0006022b8002407980035079800100037003b
:10ddd0002e429000e94f5200020036000002eb0094
:10dde0004c0037001e4fe8002e039000be03900049
:10ddf000483add00c832de00850272004832dd009c
:10de000024079800350798002e4290004447980058
:10de10004e02900094427800254798002e429000d0
:10de20000482fb000402ea004f22de000442780074
:10de3000ce0290008502e80045079800e04f5200ae
:10de400083ff3a0001003700000000002e429000de
:10de5000e04f520017003200ae429000f4c2b3000f
:10de600084cf5200130032002e429000ed4f52003a
:10de7000100032002e429000ea4f52000d00320096
:10de8000ae42900004c2b30084cf520009003200b9
:10de90002e429000e94f520006003200ae42900040
:10dea000a4c3b30084cf5200020032000002eb0092
:10deb000180037002e039000be039000545020003d
:10dec00025002000840f5300858f5b000200360080
:10ded0000002eb000f0037006e4290004506200064
:10dee00005a2b90004027800044378005e42900065
:10def0006a22b90004027800044278008442430098
:10df00004e42900004c24200de029000b4429800eb
:10df100014002000040078000080fa0000000600d1
:10df20000c00fa0040079800510798000002eb002f
:10df3000240798004e029000e00f52002d0032009e
:10df40000042eb00044f780004712200140798008f
:10df500024003700ce0290001e029000110009003c
:10df60008482d80000027800340798003e029000b6
:10df7000e00f520003003a002e029000e00f520022
:10df8000110032003e029000044278000443b000c9
:10df9000de029000844a78005e0290000402e800ed
:10dfa00054079800be0290001e02900004aab90017
:10dfb00004027800ce0290000482520044079800c8
:10dfc00014002000240798009e029000a400200066
:10dfd000110009008482d80000027800140798001c
:10dfe0001e4fe8001e427800e44f5200d9ff360071
:10dff00006003700de02900004c3b300844a7800b4
:10e000005e0290000402e80054079800de029000cf
:10e010000042eb00844a78000080fa00000006000d
:10e020000200fa00000f78009e42900064c4b30022
:10e0300084cf5200040036009e42900004ceb3000c
:10e0400004c24200144798009e42780064c4b300a2
:10e0500084cf5200040036009e42780004ceb30004
:10e0600004c24200044f78009e42900094c3b30063
:10e0700084cf5200050036009e42900094ccb3003d
:10e0800004c2420014479800040037009e429000ea
:10e0900004cdb30004c24200144798009e427800a9
:10e0a00094c3b30084cf5200050036009e4278002e
:10e0b00094ccb30004c24200044f7800040037003f
:10e0c0009e42780004cdb30004c24200044f7800a1
:10e0d0001e4290000482fb004422dd00844278004e
:10e0e0001e42780004c27200044078000080fa00ea
:10e0f000000006000200fa00004f78009e427800ff
:10e100000582fb004422de00044f78001e427800a6
:10e11000e94f52000300360075c3b3001ec242002f
:10e120000200370005c3b3001ec24200044078005d
:10e130000080fa00000006000200fa00004f78009c
:10e140001e4278006f4f62001e427800e94f520075
:10e150000300360075c3b3001ec242000200370040
:10e1600005c3b3001ec24200044078000080fa00dc
:10e17000000006000600fa0010079800210798002a
:10e180001e029000144f78002e02900094427800f6
:10e19000154798002d00370004c6b3009e42780052
:10e1a00084cf520006003600a4c7b3009e42780018
:10e1b00084cf520002003e0004ceb3001e4f420046
:10e1c0009e42900004c6b30084cf5200080036007f
:10e1d0009e429000a4c7b30084cf520004003e00ca
:10e1e0009e42900004ceb30004c24200144798003f
:10e1f0001e4290009e42780084cf520002003600fa
:10e2000014c0b300240037001e4290009e427800e4
:10e2100084cf52000200310000c2eb001e00370024
:10e220001e0290000402e800140798002e029000dd
:10e230000402e800240798001e029000144f7800a2
:10e240002e02900094427800154798001e427800f4
:10e25000e04f5200030032001e429000e04f520097
:10e26000cdff3a001e4290009e42780084cf5200bb
:10e270000200360014c0b300070037001e429000b1
:10e280009e42780084cf52000200310000c2eb00b1
:10e29000010037000042eb00044078000080fa00e3
:10e2a000000006000600fa00200798002e029000e9
:10e2b000140798003e429000044f78002e429000d0
:10e2c000344798001e427800244798001e029000b0
:10e2d000040078000080fa00000006000400fa0044
:10e2e000008fbe000e0378000e0278009442780082
:10e2f0000e0278003442900004c26a00044b780099
:10e300000e0378000e027800b44290000e027800ee
:10e310001442780004c26a00344398000e03780067
:10e320000e027800944278000e0278003442900089
:10e3300004c26a00044b78000e0378000e027800d5
:10e34000944290000e0278002442900004c26a00b9
:10e35000144398000e0378000e027800a442900047
:10e360000e0278001442900004c26a002443980010
:10e370000e0378000e027800944290000e0278009e
:10e380002442900004c26a00144398001e02be009a
:10e390000400be000080fa00000006000c00fa0035
:10e3a00040079800510798005e0290000402d100d7
:10e3b000040f78004e029000140798006022b80005
:10e3c00024079800350798000c0037002e039000b2
:10e3d000be0390001e029000140278000500200089
:10e3e0000602420087824a002407980035079800f9
:10e3f0001e0290000482e800140798001e027800b4
:10e4000004f0a7000402ea000402ea004f22de0042
:10e41000044278001e0fe900e04f5200ebff3a0083
:10e420005e0290006102620004427800e04f5200f8
:10e430000a0032002e039000be0390001e029000de
:10e44000144278000482fb0005002000060242000e
:10e4500087824a0024079800350798002e02900012
:10e460006123b8003e029000050020000602420031
:10e4700087824a002407980035079800ae02900072
:10e480003e02900004824200240798002e02900071
:10e490000482ea00040078000080fa000000060010
:10e4a0000600fa00200798002e029000040f780062
:10e4b00010003700ae42900004c6b30084cf520073
:10e4c0000b003400ae429000a4c7b30084cf5200ca
:10e4d00007003c001e027800144278008442780055
:10e4e00004ceb30004c242009e027800844a780041
:10e4f0001e0fe8001e02780094427800254798001d
:10e500002e429000e04f5200eaff3a002e029000a7
:10e51000040078000080fa00000006000400fa0001
:10e52000100798001e029000ef0242000042eb002c
:10e53000844a78001e02900004007800d8ff07008b
:10e540000042eb00044f7800140037009e42780030
:10e550000582fb009e029000048242001442780073
:10e56000e04f52000c003a00070037009e4278004e
:10e570000582fb009e0290008482420004c2b30028
:10e58000844a78001e4fe8001e427800ee4f520089
:10e59000f6ff3600040037001e4fe8001e427800e8
:10e5a000ee4f5200e9ff36000080fa00000006003e
:10e5b0000800fa00100798002107980062479800a9
:10e5c000130037001e029000144f78001e029000c6
:10e5d0000402e800140798001e427800e04f520041
:10e5e00002003a000002eb00150037006e42900076
:10e5f0009e42780084cf520005003a001e0290002f
:10e600000402e900140798001e0290000c00370075
:10e610002e02900004f0a7000402ea000402ea00bf
:10e620004f22de0004427800ae0290008502e9002d
:10e6300025079800e04f5200e2ff3a000002eb008d
:10e64000040078000080fa00000006000c00fa00c8
:10e650004007980051079800ce0290000042eb005e
:10e66000844a78005e0290000402e900ce02900025
:10e670000482420024079800ae0290000042eb00a2
:10e68000844a78000002eb001407980068025700e3
:10e69000040f78001d0037002e029000144278000d
:10e6a000e04f5200030032005e0290001407980011
:10e6b000210037001e8fe9001e02780094027800c6
:10e6c00035079800de0290001e02900084825200fe
:10e6d0004e0390001e0290000402430005017800e2
:10e6e000be00900004007800be0b02000000000095
:10e6f0003e009000e00b02000000000000027800e5
:10e700009e02900004824200140798004eba9700bf
:10e7100004f0a7000402ea000402ea004f22de002f
:10e7200004427800ceba97008502e90045bf9f00f9
:10e73000e04f5200d8ff3a001e029000040078001b
:10e740000080fa00000006000e00fa004007980062
:10e7500051079800620798006022b80024079800cb
:10e76000350798006e0290004322de00044f7800c7
:10e770006e02900067026200e00f5200010032005a
:10e780001e4fe8000042eb001447980034003700a9
:10e790001e4290000482fb00de0290008482420050
:10e7a0000042eb00844a78000042eb0024479800c6
:10e7b000250037001e4290000482fb00de0290001c
:10e7c000048342001e4290000482fb00de0290009f
:10e7d0000482420014427800844278002e029000a5
:10e7e000ce03900004824300144278008483fb002f
:10e7f0002e4290000482fb00043add0004427800bf
:10e8000004c27200044b78002e029000be029000f9
:10e8100061024200e0824a00240798003507980010
:10e820006e0290006123b8002e029000be0290009c
:10e83000840f5300858f5b000d0036002e42900040
:10e840000442e800244798002e429000e74f52000f
:10e85000d8ff36001e4290000442e800144798009a
:10e860001e4290009e4f5200c9ff39000100370040
:10e87000000000000080fa00000006000c00fa0012
:10e880003007980041079800520798000042eb00bb
:10e89000044f78000042eb00144798000042eb0060
:10e8a000244798002b00370014c0b3004447980059
:10e8b0000042eb0034479800220037001e429000cf
:10e8c0000482fb00ce029000048342009e42780046
:10e8d0000582fb00be029000048242009442780050
:10e8e0004e42900004c262008482fb003e429000cf
:10e8f0000482fb0004aade0004427800044b780086
:10e900001e4290000442e800144798004e429000d6
:10e9100004424200444798002e4290000442e8001e
:10e92000244798002e4290008482fb005e029000f3
:10e93000848f52000d0031003e4290000442e800f6
:10e94000344798003e429000e74f5200dbff36000c
:10e950001e4fe8002e4290008482fb005e02900071
:10e96000848f5200d0ff3900010037000000000002
:10e970000080fa00000006000c00fa002007980052
:10e980003107980042079800530798000042eb00b7
:10e99000144798000042eb00244798000042eb0027
:10e9a000044f7800230037002e4290000482fb00c1
:10e9b000be029000848242001e4290000482fb004e
:10e9c000040242002e039000040243001402780067
:10e9d0004822de0004427800844a78002e429000eb
:10e9e0000442e800244798002e4290000482fb0075
:10e9f000be029000848242001e4290000482fb000e
:10ea0000040242002e039000040243001402780026
:10ea100004427800844a78002e4290000442e800c4
:10ea2000244798001e4290000442e80014479800d2
:10ea30001e4fe8001e4278000483fb000700200000
:10ea40004e029000de029000840f5300858f5b0021
:10ea5000d5ff39000080fa00000006000c00fa0023
:10ea60002007980031079800420798005307980044
:10ea70000042eb00144798000042eb002447980046
:10ea80000042eb00044f7800660037002e429000f1
:10ea90000482fb00be029000048042001e429000ef
:10eaa0000482fb004222dd00ae029000048242009c
:10eab0001403be0004f02f0005002000860078003b
:10eac00007037800840378000502780087806000df
:10ead0000402630005002000c022dd0004002000c5
:10eae0000403be00610ab800040373008583730049
:10eaf000c838dd004832de0004827000c83ade000b
:10eb000004427800044878002e4290000442e80055
:10eb1000244798002e4290000482fb00be02900021
:10eb2000048342001e4290000482fb004222dd006a
:10eb3000ae029000048242001402be00044278003b
:10eb4000044b78002e4290000442e80024479800cd
:10eb50002e4290000482fb00be029000048342001b
:10eb60001e4290000482fb004222dd00ae029000b3
:10eb7000048242001402be00482ade000500200084
:10eb800004427800044b78002e4290000442e800d2
:10eb9000244798002e4290000482fb00be029000a1
:10eba000048042001e4290000482fb004222dd00ed
:10ebb000ae029000048242001403be000400200054
:10ebc000f50f2000860078000703780084037800a2
:10ebd00005027800878060000402630005002000c1
:10ebe000c022dd00040020000403be00610ab8005a
:10ebf0000403730085837300403ade0005002000a3
:10ec000004427800044878002e4290000442e80054
:10ec1000244798001e4290000442e80014479800e0
:10ec20001e4fe8001e4278000483fb00070020000e
:10ec30004e029000de029000840f5300858f5b002f
:10ec400092ff39000080fa00000006001000fa0070
:10ec500040079800510798006207980073079800d2
:10ec60000042eb00144798000042eb002447980054
:10ec70000042eb00044f7800610037001e42900014
:10ec80000482fb004222dd00ce029000848242001a
:10ec900064024700420020008500780004007800ec
:10eca000a20b0200000000002e4290000482fb0034
:10ecb000de029000048042002e039000be0390000c
:10ecc00004f02f000500200086007800070378007c
:10ecd00084037800050278008780600004026300e6
:10ece00005002000c022dd00040020000403be0057
:10ecf000610ab8000403730085837300c838dd001f
:10ed00004832de0004827000c83ade000442780017
:10ed1000044878002e4290000442e80024479800fe
:10ed20002e4290000482fb00de0290000483420029
:10ed30002e029000be02900004427800044b78003e
:10ed40002e4290000442e800244798002e42900092
:10ed50000482fb00de029000048342002e02900039
:10ed6000be029000482ade00050020000442780020
:10ed7000044b78002e4290000442e800244798009b
:10ed80002e4290000482fb00de02900004804200cc
:10ed90002e039000be03900004002000f50f200019
:10eda0008600780007037800840378000502780065
:10edb000878060000402630005002000c022dd009f
:10edc000040020000403be00610ab80004037300bd
:10edd00085837300403ade0005002000044278007d
:10ede000044878002e4290000442e800244798002e
:10edf0001e4290000442e800144798001e4fe800ad
:10ee00001e4278000483fb00070020006e02900081
:10ee1000fe029000840f5300858f5b0097ff39003e
:10ee20000080fa00000006000c00fa00200798009d
:10ee30003107980042079800530798000042eb0002
:10ee4000144798000042eb00244798000042eb0072
:10ee5000044f7800110037002e4290000482fb001e
:10ee6000be029000848242001e4290000482fb0099
:10ee70002e0390000402430014427800844a780074
:10ee80002e4290000442e800244798001e42900061
:10ee90000442e800144798001e4fe8001e42780024
:10eea0000483fb00070020004e029000de02900069
:10eeb0000402420085824a00840f5300858f5b0064
:10eec000e5ff39000080fa00000006000c00fa009f
:10eed00020079800310798004207980053079800d0
:10eee0000042eb00144798000042eb0024479800d2
:10eef0000042eb00044f7800280037002e429000bb
:10ef00000482fb0004024200be02900084824200a0
:10ef10001e4290000482fb002e0390000402430076
:10ef2000144278000482fb004822dd00840a780045
:10ef30002e4290000482fb0004024200be029000b8
:10ef4000848242002e4290000482fb0004024200b0
:10ef50003e03900004024300140378001e42900018
:10ef60000482fb000402e800ae0390000482430028
:10ef7000144278000482fb0004027300840a7800c3
:10ef80002e4290000442e800244798001e42900060
:10ef900004c2e800144798001e4fe8001e427800a3
:10efa0000483fb00070020004e029000de02900068
:10efb000840f5300858f5b00d0ff39000080fa007a
:10efc000000006000c00fa002007980031079800a6
:10efd00042079800530798000042eb00144798003e
:10efe0000042eb00244798000042eb00044f7800f9
:10eff000610037002e4290000482fb004222dd00b7
:10f00000be029000048342001e4290000482fb0076
:10f01000ae02900004824200144278000482fb0099
:10f020004822dd00cfa2de00048bbe001e4290000d
:10f030000442e800144798002e4290000482fb002e
:10f040004222dd00be029000048042002e42900069
:10f050000482fb004222dd00be02900004824200d6
:10f060001403be001e4290000482fb00ae0290001a
:10f0700004824200144278000482fb000500200054
:10f0800004027300858273000488be001e42900053
:10f090000442e800144798002e4290000482fb00ce
:10f0a0004222dd00be029000048042002e42900009
:10f0b0000482fb004222dd00be0290000482420076
:10f0c0001403be001e4290000482fb00ae029000ba
:10f0d00004824200144278000482fb0005002000f4
:10f0e000c822dd0004002000040273008582730042
:10f0f0000488be001e4290000442e80014479800b5
:10f100002e4290000482fb004222dd00be029000ed
:10f11000048042002e4290000482fb004222dd0067
:10f12000be029000048242001403be001e42900002
:10f130000482fb00ae029000048242001442780078
:10f140000482fb0005002000c022dd000400200036
:10f1500004027300858273000488be001e42900082
:10f160000442e800144798002e4290000442e80050
:10f17000244798001e4fe8001e4278000483fb00dd
:10f18000070020004e029000de029000840f530022
:10f19000858f5b0097ff39000080fa0000000600b1
:10f1a0001000fa0040079800510798006207980085
:10f1b000730798000042eb00144798000042eb00f0
:10f1c000244798000042eb00044f780053003700ba
:10f1d0006022b80024079800350798001e4290006e
:10f1e0000482fb00ce0290000482420014427800a8
:10f1f0000482fb004822dd00cfa2de002407980035
:10f20000350798001e4290000442e8001447980019
:10f210001e4290000482fb00ce0290000482420055
:10f22000144278000483fb00070020002e029000a7
:10f23000be029000040273008582730024079800c8
:10f24000350798001e4290000442e80014479800d9
:10f250001e4290000482fb00ce0290000482420015
:10f26000144278000482fb0005002000c823dd0062
:10f27000060020002e029000be02900004027300df
:10f280008582730024079800350798001e4290007d
:10f290000442e800144798001e4290000482fb00dc
:10f2a000ce02900004824200144278000482fb00e7
:10f2b00005002000c023dd00060020002e02900083
:10f2c000be02900004027300858273002407980038
:10f2d000350798001e4290000442e8001447980049
:10f2e0002e4290000482fb004222dd00de029000ec
:10f2f00004824200e40247004200200085007800ba
:10f3000004007800a20b0200000000002e429000d2
:10f310000442e800244798001e4fe8001e4278008f
:10f320000483fb00070020006e029000fe029000a4
:10f33000840f5300858f5b00a5ff39000080fa0021
:10f34000000006000c00fa00200798003107980022
:10f3500042079800530798000042eb0014479800ba
:10f360000042eb00244798000042eb00044f780075
:10f37000110037002e4290000482fb00be02900074
:10f38000848242001e4290000482fb002e03900003
:10f390000402430014427800844a78002e42900010
:10f3a0000442e800244798001e4290000442e8000e
:10f3b000144798001e4fe8001e4278000483fb00ab
:10f3c000070020004e029000de029000040242007e
:10f3d00085824a00840f5300858f5b00e5ff39006a
:10f3e0000080fa00000006000000fa00140020006f
:10f3f000040078000080fa00000006000000fa0017
:10f4000014002000040078000080fa0000000600cc
:10f410000200fa00004f7800114798001e42780061
:10f42000e14f520002003a001400200001003700b2
:10f430000002eb00040078000080fa0000000600e3
:10f440000a00fa0020479800314798004247980088
:10f4500033079800440798004e4290000482fb0056
:10f460006123b9000082eb008082eb0006024200bb
:10f4700087824a00f600200007002000860f520015
:10f48000878f5a0053003e00046001000f003700d0
:10f4900019003700230037002d00370037003700f0
:10f4a000410037004b0037004a0037004900370061
:10f4b0004800370047003700460037004500370056
:10f4c000440037002d00370037003700be0290009f
:10f4d0004e02900004824200f00f520003003600fa
:10f4e0000002eb00040f78003d00370014002000fc
:10f4f000040f78003a003700be0290004e029000e0
:10f5000004824200f00f5200030036000002eb00bc
:10f51000040f78003200370014002000040f780038
:10f520002f003700be0290004e029000048242007d
:10f53000ea0f5200030036000002eb00040f7800cf
:10f540002700370014002000040f78002400370043
:10f55000be0290004e02900004824200ea0f520068
:10f56000030036000002eb00040f78001c00370097
:10f5700014002000040f780019003700be0290002c
:10f580004e02900004824200f00f52000300360049
:10f590000002eb00040f7800110037001400200077
:10f5a000040f78000e003700be0290004e0290005b
:10f5b00004824200ea0f5200030036000002eb0012
:10f5c000040f78000600370014002000040f7800b4
:10f5d000030037000002eb00040f78000000000079
:10f5e0001e027800040078000080fa000000060087
:10f5f0000e00fa0040479800514798006247980073
:10f600004307980054079800650798000418800085
:10f61000040078001a0c020000000000280c020010
:10f620000000000000027800670262000508200068
:10f6300004aade00040f78000002eb001407980013
:10f640006e4290000482fb006123b9000082eb004f
:10f650008082eb000602420087824a0036002000ca
:10f6600007002000860f5200878f5a009d003e0041
:10f670000460010003003700230037002b0037002f
:10f680008a003700ce02900064c920000482420044
:10f690005e019000ee00900004007800a473020068
:10f6a0000000000064c9200014427800e14f5200bd
:10f6b00008003a00c402a800c422a800c442a8005e
:10f6c000c462a800c482a800c4a2a800c4c2a80042
:10f6d000c4e2a80064c9200014427800e04f520040
:10f6e0007f003a00c402a900c422a900c442a900b4
:10f6f000c462a900c482a900c4a2a900c4c2a9000e
:10f70000c4e2a90077003700ce02900064ca20004e
:10f71000048242005e019000ee0090000400780038
:10f72000a4730200000000006e0037005e0290002b
:10f73000050020004e039000060343008603780076
:10f7400066cb2000068343000401be00ee0090005b
:10f7500006007800bc74020000000000041880005d
:10f76000b4658800b4658000e00f520005003200e7
:10f77000b565800064092000848f520001003e00be
:10f78000c402a800b565800064092000848f52007f
:10f7900007003600b5658000c4122000848f520037
:10f7a00003003e00c402a800c422a80002003700e3
:10f7b000c422a900c402a900b5658000c4122000bb
:10f7c000848f520008003600b56580006422200056
:10f7d000848f520004003e00c402a800c422a80086
:10f7e000c442a80002003700c422a900c442a900f4
:10f7f000b565800064222000848f52000900360025
:10f80000b5658000c42b2000848f520005003e00a7
:10f81000c402a800c422a800c442a800c462a80070
:10f8200001003700c462a900b5658000c42b200028
:10f83000848f52000b003600b5658000643b2000c9
:10f84000848f520007003e00c402a800c422a80012
:10f85000c442a800c462a800c482a800c4a2a80030
:10f8600002003700c482a900c4a2a900b5658000c7
:10f87000643b2000848f520009003600c402a800b7
:10f88000c422a800c442a800c462a800c482a80080
:10f89000c4a2a800c4c2a800c4e2a8001100370096
:10f8a000c4c2a900c4e2a9000e0037005e029000a5
:10f8b000050020004e0390000603430086037800f5
:10f8c000a6cc2000068343000401be00ee00900099
:10f8d00006007800bc740200000000000100370040
:10f8e000000000000042eb00044078000080fa00b5
:10f8f000000006000a00fa00004f78001147980047
:10f90000224798002307980034079800450798007d
:10f910002e4290000482fb006123b900b4ff2f0047
:10f92000f5ff2f000602420087824a00b600200041
:10f9300007002000860f5200878f5a0023003e00e8
:10f94000046001000b003700130037001f00370070
:10f950001e0037001d0037001c0037001b00370059
:10f960001a0037001900370018003700010037006f
:10f9700009003700ae02900064c9200004824200f2
:10f980003e019000840078004e0090003e7402001a
:10f99000000000000d0037003e029000050020002e
:10f9a0002e039000060343008603780066cb2000f8
:10f9b000068343000401be00860078004e009000dc
:10f9c0006677020000000000000000000042eb002b
:10f9d000044078000080fa00000006000200fa00ef
:10f9e000004f780014002000040078000080fa0026
:10f9f000000006001200fa00004f9800510798001e
:10fa00006207980073079800040f98001400200004
:10fa1000040f7800ba85020000000000228802006e
:10fa2000000000000002eb00140798000002eb0049
:10fa3000240798000002eb00340798008e0a90001b
:10fa40000042eb00844a78000002eb002407980093
:10fa5000330037007c030200000000000002780041
:10fa6000340798001d00370097c0a900fe029000df
:10fa70001e02900084824200b4df2000144278000d
:10fa80000483fb0004a02000040243001442780019
:10fa9000844a7800a4df2000144278000442e90080
:10faa00004407800faedb70097c0a800b4df20004a
:10fab000144278000442e80004407800fbedb700ef
:10fac0001e0290000402e800140798007c03020064
:10fad0000000000000027800340798003e02900009
:10fae000e00f5200040032009e0290005e0290007f
:10faf000848f5200dcff39009e0290005e0290006d
:10fb0000848f52000a003200500020008c910200c5
:10fb1000000000002e0290000402e8002407980074
:10fb20002e029000f30f5200caff3600010037008a
:10fb3000000000009e0290005e029000848f520040
:10fb400007003a006e0290009e029000050a7800bd
:10fb50008e0a90000042eb00844a780005003700ce
:10fb60008e0a900054c0b300844a78000002eb0073
:10fb7000040f78001e027800040078000080fa006c
:10fb8000000006000e00fa00404798003107980078
:10fb9000420798005307980064079800140020005b
:10fba00014079800ba8502000000000022880200b5
:10fbb000000000000042eb0004407800faedb700be
:10fbc0000042eb0004407800fbedb7000042eb0080
:10fbd00004407800fcedb7000002eb00040f780051
:10fbe0000e00370000000000620402000000000068
:10fbf00000427800e04f5200fbff3a005e029000a6
:10fc00001e024200144278000482fb0004007800c7
:10fc100094040200000000001e0fe8003e02900065
:10fc20009e027800848f5200eeff39000000000031
:10fc3000620402000000000000427800e04f520021
:10fc4000fbff3a004e029000be029000050a7800c9
:10fc5000ee0290000042eb00844a78001e02900001
:10fc6000040078000080fa00000006000200fa009c
:10fc7000004f780014002000040078000080fa0093
:10fc8000000006000200fa00004f78000042eb007e
:10fc900004407800faedb7000042eb000440780021
:10fca000fbedb7000042eb0004407800fcedb7002c
:10fcb00014002000040078000080fa000000060014
:10fcc0000400fa00004f78001147980012079800ce
:10fcd0001e009000c8900200000000000080fa00a2
:10fce000000006002600fa00600f9800710f9800cf
:10fcf0000217980013179800446798004e6290000e
:10fd00000482fb003407980000c2eb0024579800df
:10fd100000c2eb003457980000c2eb004457980033
:10fd200000c2eb005457980000c2eb0064579800e3
:10fd300000c2eb00745798000e1290009e129000c3
:10fd4000440f9800550f98006e0a9000fe0a90002c
:10fd500074079800050f98000e0078000400070053
:10fd600000027800040078000080fa00000006001d
:10fd70000200fa00000f780000000000843a020040
:10fd80000000000000027800e00f5200fbff32008c
:10fd90000000eb00083d0200000000001e02780099
:10fda00015002000050a78001e027800058020005a
:10fdb000150298009e02780064c0b300c442980007
:10fdc0009e02780044c0b300d44298009e0278009e
:10fdd0006882420062002000b1d020000400780058
:10fde000a20b0200000000009e037800e6cd200078
:10fdf000164378000680fb00f6cd200016437800fd
:10fe00000683fb004833dd00000373000602780020
:10fe100006ce2000164378000680fb0016ce200098
:10fe2000164378000683fb004833dd0000037300af
:10fe300086027800f4039800850b98001e00780075
:10fe4000500107009e02780072824200c201200029
:10fe500061c0b30004007800423c020000000000d2
:10fe60001e027800c101200004007800443f020017
:10fe700000000000883c0200000000001400200088
:10fe8000040078000080fa00000006000000fa007c
:10fe900000c2eb0004407800b0edb70000c2eb00f8
:10fea00004407800b1edb70000c2eb0004407800d8
:10feb000b2edb70000c2eb0004407800b3edb7002c
:10fec00000c2eb0004407800b4edb70000c2eb00c4
:10fed00004407800b5edb7000082eb008082eb00b3
:10fee000646d8800756d88000080fa0000000600cf
:10fef0001c00fa00b46d8000e00f520003003200d5
:10ff0000e10f5200480032005d0037000e02780019
:10ff1000c101200004007800fa3e02000000000049
:10ff20009c3a0200000000000e0078001501070056
:10ff30001e027800e10f520006003a004e42900087
:10ff4000e64f520003003a005e429000e44f520038
:10ff500002003200140020004a0037003e029000e8
:10ff6000e20f52000c003a004e029000de029000b8
:10ff7000846d8800956d8800ee029000a56d880064
:10ff80007e0290008e0a9000646d8800756d880076
:10ff9000140020003b0037003e029000e10f5200a9
:10ffa00021003a004e0b9000de0b9000deccbf002b
:10ffb0008080fb00dfccbf000080fb004800dd003c
:10ffc0000100700000027800e0ccbf008080fb00e0
:10ffd000e1ccbf000080fb004800dd0001007000a4
:10ffe00080027800840f5300858f5b00020032008e
:10fff00014002000230037007e0290008e0a90003b
:020000040001f9
:10000000c46d8800d56d88004e029000de0290001d
:10001000e46d8800f56d8800ee029000056e8800a2
:1000200014002000b46d88002400200034079800dc
:10003000e46d8000f56d8000140f9800250f980086
:10004000056e8000350f9800c46d8000d56d80006e
:10005000440f9800550f98000e00780044ff0700e9
:1000600000027800e00f520002003a000002eb00ac
:10007000040037000002eb00b46d880000000000af
:1000800014002000040078000080fa000000060040
:100090001e00fa00600f980014002000340798003a
:1000a00000c2eb002457980000c2eb0034579800c0
:1000b00000c2eb004457980000c2eb005457980070
:1000c00000c2eb006457980000c2eb007457980020
:1000d000e6cd2000164378008683fb00f6cd200095
:1000e000164378000683fb004833dd0007037300e6
:1000f0000602780006ce2000164378008683fb00b7
:1001000016ce2000164378000683fb004833dd003e
:1001100007037300860278006e0b90001603be0082
:1001200006036a0087836a00e2ccbf008080fb0080
:10013000e3ccbf000080fb004800dd000100700040
:1001400000027800e4ccbf008080fb00e5ccbf005b
:100150000080fb004800dd00010070008002780094
:100160000600780007037800840378000502780011
:10017000070060000402630005002000c022dd00cb
:10018000040020000403be006102b80004037300f1
:1001900085837300e00f5300e08f5b001500320091
:1001a00066ce2000164378008683fb0076ce2000c2
:1001b000164378000683fb004833dd000703730015
:1001c0000602780086ce2000164378008683fb0066
:1001d00096ce2000164378000683fb004833dd00ee
:1001e0000703730086027800440f9800550f9800ab
:1001f000040037006e0a90001403be00460f9800fa
:10020000570f98000e007800d9fe07000080fa0012
:10021000000006000400fa00000f780011079800a3
:10022000646d8000756d80001e0378001603be00ab
:10023000860f5200878f5a0047003200666d80009b
:10024000776d8000e6ccbf008080fb00e7ccbf006c
:100250000080fb004800dd00010070000002780013
:10026000e8ccbf008080fb00e9ccbf000080fb0031
:100270004800dd000100700080027800840f530008
:10028000858f5b003b003a00e6cd200016437800e6
:100290008683fb00f6cd2000164378000683fb0022
:1002a0004833dd00070373000602780006ce200005
:1002b000164378008683fb0016ce20001643780094
:1002c0000683fb004833dd000703730086027800d5
:1002d0001e0378001603be0006036a0087836a00c7
:1002e000e2ccbf008080fb00e3ccbf000080fb00bd
:1002f0004800dd000100700000027800e4ccbf007f
:100300008080fb00e5ccbf000080fb004800dd00e2
:100310000100700080027800060078000703780072
:10032000840378000502780007006000040263007f
:1003300005002000c022dd00040020000403be00f0
:100340006102b8000403730085837300e00f53005b
:10035000e08f5b00070032001e02900005db2000ea
:1003600005000900355a78006400b100140020002f
:10037000010037000002eb00040078000080fa0062
:10038000000006000200fa00000f78001e0278004c
:10039000140278000400780052710200000000008e
:1003a000000278009e027800840a78001e0278001d
:1003b0001402900004007800527102000000000056
:1003c000000278009e027800940298001e027800d5
:1003d0003402900004007800527102000000000016
:1003e000000278009e027800b40298000080fa00b3
:1003f000000006000000fa00d782a800d382a900fe
:10040000e4c2a900e4e2a800e502a9003413200038
:10041000141388000002eb00241388000002eb0094
:100420000413880061e2a8000080fa0000000600c2
:100430000400fa00008fbe001e02be00646a88003d
:10044000756a88000042eb000440780070edb70048
:100450000002eb00040078000080fa0000000600b3
:100460000000fa0004d7200014427800e04f520048
:100470000f003a00646a8000756a80000302200061
:1004800002d520000400be001d000700646a800041
:10049000756a80000402b0000580b000646a8800bc
:1004a000756a880004c2b3000440780070edb7009c
:1004b00004d72000144278008482fb00060220004a
:1004c0000503530005d520008502430095427800be
:1004d0000442e9000440780070edb700054278005e
:1004e000044078000080fa00000006000000fa00d6
:1004f0000002eb00040078000080fa000000060013
:100500000c00fa0020079800310798004207980075
:100510005307980014138000040f78000413800020
:100520004f22de00044278002447980061e2a900cf
:10053000341320001413880061e2a800d782a900b8
:10054000340020004413880004138000620262001b
:10055000e00f5200fcff3a000413800061026200c9
:10056000e00f5200f8ff320044138000044278008c
:100570003447980064024700144290000482fb0054
:10058000441388000413800062026200e00f5200ee
:10059000fcff3a000413800061026200e00f520089
:1005a000f8ff32004413800004427800344798007a
:1005b00064024700144278000482fb004413880060
:1005c0000413800062026200e00f5200fcff3a0058
:1005d0000413800061026200e00f5200f8ff320055
:1005e0004413800004427800344798001600370016
:1005f0000002eb00441388000413800062026200d2
:10060000e00f5200fcff3a00041380006102620018
:10061000e00f5200f8ff32004413800004427800db
:10062000344798004e029000e00f5200060032005e
:100630003e429000ce029000844a78004e02900024
:100640000402e800440798005e02900004f0a7004e
:100650000402ea000402ea004f22de0004427800ad
:10066000de0290008502e90055079800e04f520035
:10067000dfff3a00d782a80061e2a9001e027800dd
:10068000141388002e429000614262000482fb0035
:100690004f22dd0006138000f5ff2700850263006e
:1006a00004827200041388000002eb00040078004a
:1006b0000080fa00000006000400fa00008fbe006f
:1006c0000042eb000440780070edb7001e02be004f
:1006d000646a8800756a88000002eb0004007800f4
:1006e0000080fa00000006000200fa00004f7800c7
:1006f00004d72000144278000483fb0005d52000b5
:10070000850243009e4a78000442e80004407800d5
:1007100070edb70004d7200014427800ff4f52005c
:1007200002003600340007000e003700646a8000c3
:10073000756a8000044278008482fb0004d72000a0
:10074000144278000482fb00048242008402780094
:10075000f403200004826200e00f520001003a001e
:10076000250007000002eb00040078000080fa007a
:10077000000006000400fa00000f7800110798003e
:10078000050037001e027800144278001e0fe800b2
:1007900004407800d4ff07001e02900004f0a70078
:1007a0000402ea000402ea004f22de00044278005c
:1007b0009e0290008502e90015079800e04f520064
:1007c000f0ff3a00020007000080fa000000060077
:1007d0000000fa0004d7200014427800e04f5200d5
:1007e00001003200040007000002eb000400780062
:1007f0000080fa00000006000600fa0010138000d6
:1008000010079800041380004f22de000442780095
:100810004447980061e2a9003413200014138800b3
:1008200061e2a800d782a900640020004413880078
:100830000413800062026200e00f5200fcff3a00e5
:100840000413800061026200e00f5200f8ff3200e2
:10085000441380000442780054479800d782a800cf
:10086000d782a900240020004413880004138000cc
:1008700062026200e00f5200fcff3a0004138000a5
:1008800061026200e00f5200f8ff32004413800062
:100890000442780054479800c4d4200014429000c9
:1008a0000482fb004413880004138000620262008b
:1008b000e00f5200fcff3a00041380006102620066
:1008c000e00f5200f8ff3200441380000442780029
:1008d00054479800c4d42000144278000482fb00de
:1008e000441388000413800062026200e00f52008b
:1008f000fcff3a000413800061026200e00f520026
:10090000f8ff3200441380000442780054479800f6
:100910000042eb00044f7800130037001e427800bd
:100920008482fb0004d52000048242001442780037
:100930000482fb00441388000413800062026200fa
:10094000e00f5200fcff3a000413800061026200d5
:10095000e00f5200f8ff3200441380000442780098
:10096000544798001e4fe80004d720001442780036
:100970009e42780084cf5200e8ff3900d782a80059
:1009800004d72000144278000483fb0007002000f5
:10099000646a8000756a80000602420087824a000d
:1009a000646a8800756a88000042eb0004407800a1
:1009b00070edb70061e2a9001e02900014138800d8
:1009c0004e429000614262000482fb004f22dd0033
:1009d00006138000f5ff2700850263000482720081
:1009e00004138800000000000500070000027800e2
:1009f000e00f5200fcff3a000080fa000000060001
:100a00000400fa0014138000040f7800041380001f
:100a10004f22de00044278002447980061e2a900da
:100a2000341320001413880061e2a800d782a900c3
:100a30005400200044138800041380006202620006
:100a4000e00f5200fcff3a000413800061026200d4
:100a5000e00f5200f8ff3200441380000442780097
:100a6000344798000002eb00441388000413800010
:100a700062026200e00f5200fcff3a0004138000a3
:100a800061026200e00f5200f8ff32004413800060
:100a90000442780034479800d782a80061e2a90098
:100aa0001e027800141388002e42900061426200fa
:100ab0000482fb004f22dd0006138000f5ff2700b3
:100ac0008502630004827200041388003e42900095
:100ad000614262000482fb00040078000080fa009a
:100ae000000006000000fa000002eb00146e88000f
:100af0000aeda800846e8000e00f520008003a0062
:100b0000086d0200000000000002be000400be00ec
:100b1000566c02000000000014002000846e880063
:100b20001439020000000000467f020000000000af
:100b30007e5b020000000000e215020000000000e1
:100b40000040eb00d046020000000000a4d02000ce
:100b5000144278000444b200e04f520003003a000f
:100b60000040eb001c470200000000000080fa007b
:100b7000000006000a00fa00a4d020001442780009
:100b80000444b200e04f52007a0032006a3a020098
:100b90000000000000027800040f7800746e8000ee
:100ba0009e027800848f5200690032001e00780097
:100bb000706e88001e027800e00f520064003a0058
:100bc00026cf2000164378008683fb0036cf200016
:100bd000164378000683fb004833dd0007037300eb
:100be0000602780046cf2000164378008683fb007b
:100bf00056cf2000164378000683fb004833dd0003
:100c00000703730086027800f60f20008603620057
:100c1000e6cd20001643780060436300074373006d
:100c200006407800deecb700c823de00f6cd2000d9
:100c30001643780060436300074373000640780062
:100c4000dfecb700f60f20008683620006ce20009e
:100c50001643780060436300074373000640780042
:100c6000e0ecb700c82ade0014ce20001442780061
:100c7000604262000542720004407800e1ecb70077
:100c800066cf2000164378008683fb0076cf2000d5
:100c9000164378000683fb004833dd00070373002a
:100ca0000602780086cf2000164378008683fb007a
:100cb00096cf2000164378000683fb004833dd0002
:100cc0000703730086027800f60f20008603620097
:100cd00026ce20001643780060436300074373006c
:100ce00006407800e2ecb700c823de0036ce2000d4
:100cf00016437800604363000743730006407800a2
:100d0000e3ecb700f60f20008683620046ce200099
:100d10001643780060436300074373000640780081
:100d2000e4ecb700c82ade0054ce2000144278005c
:100d3000604262000542720004407800e5ecb700b2
:100d40000aeda8000040eb00d046020000000000c1
:100d5000ee470200000000000040eb006847020080
:100d60000000000000027800e00f52000100320095
:100d70000aeda9008e20020000000000b25c020013
:100d800000000000010037000000000008620200bf
:100d900000000000680247008400780080dc20002a
:100da000f63a02000000000000027800e00f520056
:100db0009f0032000e4a90000482fb00e00f5200b8
:100dc00005003200e60f5200efff3a00787f020084
:100dd00000000000950037000e83e800e90247009c
:100de00064024700860178000501780041dc20009c
:100df00004007800f689020000000000000278007c
:100e0000e00f520001003a00880037001e4a9000af
:100e1000e14f52006c003a002e039000be03900098
:100e2000deccbf008080fb00dfccbf000080fb0079
:100e30004800dd000100700000027800e0ccbf0037
:100e40008080fb00e1ccbf000080fb004800dd009b
:100e50000100700080027800840f5300858f5b00d2
:100e6000530032002e039000be0390000082eb007e
:100e70008082eb00840f5300858f5b004c003200b2
:100e80002e009000be009000e4cd200014427800b7
:100e90008482fb00f4cd2000144278000482fb0021
:100ea0004822dd00050272000403780004ce200011
:100eb000144278008482fb0014ce20001442780093
:100ec0000482fb004822dd000502720084037800e2
:100ed00022ce2000124178008281fb0032ce200019
:100ee000124178000281fb004811dd00030171000e
:100ef0000202780042ce2000124178008281fb007d
:100f000052ce2000124178000281fb004811dd0022
:100f1000030171008202780006017800070378005f
:100f20008403780005027800070161000402630071
:100f300005002000c022dd00040020000403be00e4
:100f40006112b800040373008583730022ce200071
:100f5000124178008281fb0032ce200012417800dd
:100f60000281fb004811dd000301710002027800dc
:100f700042ce2000124178008281fb0052ce200038
:100f8000124178000281fb004811dd00030171006d
:100f9000820278000482ea008582ea00040273007b
:100fa00085827300840f5000858f580005003a0039
:100fb0001e0290008400780040dc2000f8900200bf
:100fc00000000000190037001e4a9000e64f520052
:100fd00008003a009e029000640247000501780074
:100fe0008400780040dc20009e2502000000000004
:100ff0000e0037001e4a9000f14f52000a003a00de
:101000009e02900064024700050178008400780089
:1010100040dc20002862020000000000000278008e
:10102000e00f520004003a000000000057ff3700b4
:101030000000000001003700000000000080fa00fe
:10104000000006000000fa00da880200000000003c
:101050000080fa00000006000200fa006a3a02006e
:101060000000000000027800e00f52004c00320047
:10107000f4652700c3b220000041eb006000b80017
:10108000985b0200000000000042780014479800be
:101090001e429000e14f4200430032000000000079
:1010a0001e4090009e5f02000000000000027800d9
:1010b000e00f5200faff3200f1002000a0cf200024
:1010c0000460020000000000d0c0b300d45f020042
:1010d00000000000a0c0b300d45f020000000000c8
:1010e0000042eb00044f78009e4278000582fb002e
:1010f000c502200084824200f4cd20000482420018
:1011000014427800044078007a7002000000000069
:101110000042780004407800d45f02000000000024
:101120009e4278000582fb00c502200084824200b6
:10113000f4cd20000482420014427800044078007c
:101140009c7002000000000000427800044078001b
:10115000d45f0200000000001e4fe8001e4278002d
:10116000e64f52000a003a00044f290004007800bc
:1011700040600200000000005e600200000000000d
:101180001e409000305f02000000000007003700a2
:10119000d0c2b300d45f020000000000d2ff3700cd
:1011a0000000000001003700000000000080fa008d
:1011b000000006000200fa00346f800005002000e5
:1011c0003600200007002000860f5200878f5a004b
:1011d00084003e0004600100030037001300370064
:1011e0003200370076003700f4652700f3652700ea
:1011f0000041eb006000b800985b020000000000b6
:101200000042780004407800e8edb70084de20005a
:1012100014427800e14f42006b003200346f8000ce
:101220000402e800346f88006e00370084de20007e
:101230001442780004407800586102000000000069
:1012400000027800e00f5200610032000e007800ca
:101250008861020000000000086202000000000037
:101260009e42780044c4b30084cf52005a003a0032
:10127000346f80000402e800346f880084de2000b0
:10128000144278000482fb007822b90084027800be
:1012900004b0200004824200a200200041dc2000b3
:1012a00004007800a20b02000000000084de200091
:1012b00014427800044078009e5f020000000000a5
:1012c00000027800e00f520045003200f1002000db
:1012d000a0cf20000460020000000000d0c0b300d6
:1012e000d45f020000000000a0c0b300d45f020081
:1012f000000000000042eb00044f78001e4278001e
:101300000482fb00c502200084824200f4cd20004c
:101310000482420014427800044078007a7002008f
:10132000000000000042780004407800d45f020012
:10133000000000001e4278000482fb00c50220006d
:1013400084824200f4cd20000482420014427800de
:10135000044078009c700200000000000042780009
:1013600004407800d45f0200000000001e427800b4
:101370000442e800044f78001e427800e64f520015
:101380000b003a00d0c0b300d45f020000000000a0
:10139000a0c0b300d45f0200000000005e60020045
:1013a0000000000014002000346f88000d0037009a
:1013b000d0c2b300d45f020000000000cfff3700ae
:1013c00000000000070037000000000005003700a3
:1013d000000000000300370000000000010037009b
:1013e000000000000080fa00000006001e00fa0065
:1013f000300f9800410f9800520f9800630f98002b
:101400000e82e8004101200004007800fa3e02004c
:10141000000000002e4290008482fb00040f200098
:101420008482620004042000848f52000200320093
:101430000002eb004f003700ce029000f4f12f00c5
:1014400004826200e00f5200020032000002eb0052
:10145000480037002e4290006f42620025002000b5
:101460000522dd0004407800f4edb70044df2000e1
:10147000144278000482fb00840078000000eb0036
:101480003c3d02000000000000027800040f7800dc
:1014900044df2000144278000482fb00040078003e
:1014a000e63c0200000000001e027800e00f52003f
:1014b000020032000002eb002e0037000e82e8002e
:1014c00004007800920007003e0a9000e00f5200ee
:1014d000040032001e0a9000ae0a90003e0b9000fd
:1014e000048bbe007e0390008e0b90004e0a90008d
:1014f000f50f20000500630094427800e0c262000e
:1015000080c27200054a78004830de0094429000a4
:10151000e0c2620080c2720015429800f50f200000
:1015200005806300a4429000e0c2620080c27200a5
:1015300025429800483bde00b4429000e0c26200c1
:1015400086c27200354298003e4a9000de0a900042
:10155000844a7800ae02900044df200014427800f4
:101560000482fb00848252006e0a9000050a780013
:1015700014002000040078000080fa00000006003b
:101580001a00fa00200f980061579800420f980047
:1015900044c1b30004407800f4edb70054c4b30074
:1015a000044f78000042eb00144798004e0a900068
:1015b0007402420014079800946f80000402e8004f
:1015c000946f8800946f8000240798000002eb005d
:1015d0003407980044c6b300044f98006e52900040
:1015e000144f98000002eb0054079800e6cd20004d
:1015f000164378008683fb00f6cd20001643780062
:101600000683fb004833dd00070373000602780001
:1016100006ce2000164378008683fb0016ce2000fd
:10162000164378000683fb004833dd000703730090
:101630008602780064079800750798002e0b9000ca
:10164000164278000480fb00964390008783fb00dd
:10165000c83bdd008083730007027800a64390003a
:101660008783fb00364390000683fb004833dd0090
:101670000703730086027800040f9800150f980086
:101680000e00780022000700410120000e007800c3
:10169000ce7102000000000000027800540798009c
:1016a0004e0a9000f40242002e0a900064024200aa
:1016b000050178008040eb0004007800423c020005
:1016c00000000000410120000e007800443f0200ad
:1016d000000000000002eb00040078000080fa0027
:1016e000000006000200fa00000f780044df20002e
:1016f000144278000482fb001e02420004007800bd
:10170000e63c0200000000000080fa000000060035
:101710000200fa00000f78001e0278001402900008
:1017200004007800527102000000000000027800fe
:101730009e027800940298001e0278002402900015
:1017400004007800527102000000000000027800de
:101750009e027800a40298001e02780054029000b5
:1017600004007800527102000000000000027800be
:101770009e027800d40298000080fa000000060063
:101780000200fa00004f780011479800852d2000d4
:101790000042eb00844a7800c7e2a900d2a2a90067
:1017a000d6a2a9009e42780061c262000482fb00ba
:1017b0004f22dd0056168000f5ff270085026300ea
:1017c0000482720054168800c42d20009e429000ae
:1017d000054a78000000000000000000d682a80042
:1017e00000000000000000000000000000000000f9
:1017f00000000000000000000000000000000000e9
:1018000000000000d682a9000080fa000000060057
:101810000200fa00020220000102200020d720006e
:10182000b00b0200000000000042eb000440780012
:1018300092edb700d682a900d6a2a900852d20007e
:101840000042eb00844a7800d2a2a900c7e2a900b6
:10185000d282a900800220008c91020000000000ca
:10186000cbe2a900c52d200034c0b300844a780023
:1018700000000000000000000042eb00044f780070
:101880000a003700d682a8001000200001002000c6
:10189000c891020000000000d682a90020002000ac
:1018a0008c910200000000001e4fe8001e427800ec
:1018b000e24f5200f3ff360081c3b3000040eb005b
:1018c000afff07005000200001002000c891020077
:1018d0000000000061c0b3000040eb00a8ff07005b
:1018e0005000200001002000c8910200000000000c
:1018f000c1c0b3000040eb00a1ff07005000200072
:1019000001002000c89102000000000011c0b300d7
:101910000040eb009aff0700200020008c9102009d
:10192000000000000080fa00000006000200fa003b
:1019300021c0b3000040eb0091ff07002000200011
:101940008c910200000000000042eb00044f780080
:10195000230037001e4278008482fb0024d7200039
:101960000482420014427800e04f52000f003a0017
:101970001e42780014479800090037001e4290006c
:101980008482fb0024d720008482420004c2b3007a
:10199000844a78001e4290000442e80014479800f0
:1019a0001e429000ef4f5200f4ff36001e427800b6
:1019b0008482fb0024d72000048242001442780075
:1019c0008440780010c0b3006dff07005000200075
:1019d00001002000c8910200000000001e4fe80036
:1019e0001e427800ef4f5200daff360001ccb30000
:1019f0000040eb0062ff07005000200001002000c3
:101a0000c89102000000000004c1b300044f780038
:101a1000230037001e4278008482fb0024d7200078
:101a20000482420014427800e04f52000f003a0056
:101a30001e42780014479800090037001e429000ab
:101a40008482fb0024d720008482420004c2b300b9
:101a5000844a78001e4290000442e800144798002f
:101a60001e429000ff4f5200f4ff36001e427800e5
:101a70008482fb0024d720000482420014427800b4
:101a80008440780010c0b3003dff070050002000e4
:101a900001002000c8910200000000001e4fe80075
:101aa0001e427800ff4f5200daff36000080fa0035
:101ab000000006000000fa0011c0b3000040eb0077
:101ac0002fff0700200020008c9102000000000082
:101ad000020220000102200020d72000b00b0200eb
:0c1ae000000000000080fa00000006007a
:020000040000fa
:020000040001f9
:101aec00ac0d00001600000000000000e60d000028
:101afc000400000000000000fe0d000002000000c9
:101b0c000200000000000000240d0000280000006e
:101b1c0000000000ea0d00000400000002000000bc
:101b2c00ff00070000000000940d000018000000ea
:101b3c0000000000d20d00000a00000000000000b0
:101b4c00ee0d000004000000020000009e9ffe004d
:101b5c0041000000f20d0000040000000000000035
:101b6c00720d000022000000000000004c0d00006f
:101b7c002600000000000000c20d00001000000054
:101b8c0000000000cc0b0000ca00000000000000a8
:101b9c00040e00000200000002000000fefe000027
:101bac00dc0d00000a00000000000000000b00002b
:101bbc00cc00000000000000060e00000200000037
:101bcc0002000000ffff00000a0e000002000000ef
